:0600000076EF06F012008D
:0600080004EF08F01200F5
:100018000CEF08F012001DEE00F02DEE00F0F86A6B
:0600280092EF06F0120049
:1000300000003E0E006E016AFC0E026E036A046A46
:10004000076808680968066A1200D9CFE6FFE1CFA1
:10005000D9FFE65204501EE1040108BF1AD0400E39
:10006000E66E600EE66E000EE66E38EC06F0E552C7
:10007000E552E552010E046EDF6A400EDF5C09E2D4
:10008000DF50EA6AA00FE96E000EEA22EF6ADF2A6B
:10009000F4D717D100016051080A01E10DD10F0A10
:1000A00001E1D3D0010A01E1CAD0030A67E0010AE5
:1000B00058E0070A44E0010A01E003D10001020E02
:1000C000A06F00013A0EA16F0001010EA26F0001A6
:1000D000010EA36F0001A46B100EA56FA66BA76B9A
:1000E00001C0A8F002C0A9F003C0AAF0100E0001E0
:1000F000A95F000E0001AA5B0001AB6B0001030EBB
:10010000AC6F0001F80EAD6FAE69AF6BB06B000164
:10011000080EB16FB26BB36BB46B0001B56904012B
:100120000CBF0CD0400EE66EA00EE66E000EE66E22
:1001300008EC06F0E552E552E552046AC2D000012F
:10014000615107E13F0E006EF80E016E0268036A0E
:1001500006D03E0E006E016AFC0E026E036A046A4F
:10016000B0D0040E056E0028055C06E20400AED88F
:100170009DEC04F0052AF7D7046AA3D0E8680718B5
:1001800005E1E868081802E1E868091806E161C0BD
:1001900007F062C008F063C009F007500001611960
:1001A00008E108500001621904E1095000016319D7
:1001B00000E143E1DF6A00016551DF5C3EE2000ED1
:1001C000075C100E0858000E09582CE300285B6EDF
:1001D0005C6A0A0ED8905B365C36E806FBE15D6A25
:1001E0005CBE5D685B50075C5C5008585D50095808
:1001F00019E23A0E0001D8806555DF24EA6A660FDD
:10020000E96E000EEA22EF50E66E0650E96EEA6AE9
:10021000E9BEEA680A0EE926000EEA22E552E75036
:10022000EF6E062A072A000E0822000E09223A0E57
:10023000065C01E15ED8DF2ABED7046A42D059D8F5
:10024000076808680968046A3CD00001070EA06FBF
:1002500061C0A1F062C0A2F063C0A3F064C0A4F0CA
:1002600065C0A5F061C0F6FF62C0F7FF63C0F8FF8C
:10027000DF6A00016551DF5C0FE209003A0E000100
:10028000D8806555DF24EA6AA60FE96E000EEA22DF
:10029000F5CFEFFFDF2AEDD704010CBF0CD0400EE5
:1002A000E66EA00EE66E000EE66E08EC06F0E55275
:1002B000E552E552046A05D06592656A68D8FF0088
:1002C00000D0E552E552E7CFD9FF1200F66A05509B
:1002D000F76EF86AD890F736F836F736F836140E17
:1002E000A66EF29E550EA76EAA0EA76EA682A694C3
:1002F0001200D9CFE6FFE1CFD9FFE652DF6A000E48
:10030000E76E0618E8AE02D0063403D0E750D88076
:10031000065436E206505B6E5C6A5D6A5BAE02D0E4
:100320005C685D685B50075CF66E5C500858F76E61
:100330005D500958F86EDF50EA6A0A0FE96E000E48
:10034000EA22EF50F56E0D00DF2A0606065009E09E
:10035000DF50EA6A0A0FE96E000EEA22EF50F56EEE
:1003600001D0F5680C00DF2A240EA66EF29E550E11
:10037000A76EAA0EA76EA682065001E00606BFD79A
:10038000A694066AE552E552E7CFD9FF1200D9CF0D
:10039000E6FFE1CFD9FFE652DF6AFF0EDF5C0AE23B
:1003A000E868E85005E0E80600D000D000D0F9D7B2
:1003B000DF2AF3D7E552E552E7CFD9FF12005FD924
:1003C000E652645032E16296040100513C0BE8426F
:1003D000E8420D0828E1180E021923E1040E031962
:1003E00020E1100E026F040E036FDF6ADF505B6EB8
:1003F0005C6A080E5B5C000E5C5813E2DF50EA6A30
:10040000180FE96E040EEA22EF50E66EDF50EA6A3A
:10041000100FE96E040EEA22E552E750EF6EDF2A74
:10042000E5D70ED80AD03DD808D0040E645C03E1AD
:1004300062964DD802D0000E01D0010EE55224D1B3
:100440001ED9E652040104BF046B556A516A526A10
:10045000536A546A4FEC03F0DF6ADF505B6E5C6AEC
:10046000010E5B5C000E5C5819E2525017E1F76A0E
:10047000DF34FE0BF736F66EA40EF6260E0EF722CC
:100480000900F5CF5BF00800F5CF5CF004D05CC04C
:10049000FAFF5B50F96EFBDFDF2ADFD79ED8E5520B
:1004A000F3D0020E515C0EE176D80401180E026FF3
:1004B000040E036F080E016F00BD02D0C80E05D0F8
:1004C000880E03D0BCD8CCD88C0E006F1200040E5E
:1004D000575C0AE112C438FF0F013851000802E2EC
:1004E000050E01D0030E576E51040FE110D8020E15
:1004F000555C03E10401840E06D0040104BD02D062
:10050000C80E01D0880E046F12001FEF03F0B7D899
:10051000020EE126080E535C000E54580DE253C043
:10052000DEFF54C0DDFF555002E1010E03D055043B
:1005300006E1020E556E03D0080EDE6EDD6A040180
:1005400004930491010EDB500413DFCF05F4DE5059
:10055000535EDD50545A0001180EE26F040EE36F33
:1005600058A20CD085D810E0E0C0F6FFE1C0F7FF3C
:100570000800F55068D8F6E2DB06F4D779D804E035
:1005800087D8FCE2DB06FAD7020EE15C02E2E16A00
:10059000E552E16E79D073D8020EE126030E040114
:1005A0000015E76E010EE7CFDBFF01C4DFFFDE5071
:1005B0005326DD5054220001180EE06F040EE16F47
:1005C00057D804E065D8FCE2DB06FAD7020EE15CFE
:1005D00002E2E16AE552E16E57D06598525005E1BA
:1005E0003FD8840E006F040118D0040110AF17D05B
:1005F0005350165D5450175904E216C453F017C4F3
:1006000054F085DF010E516E2BD8800E006F04016F
:10061000180E066F040E076FC80E046F1200020E4C
:10062000516E0401056BC80E046F0401080E016FC2
:10063000180E026F040E036FC80E006F1200516A8D
:100640000401046B1200E2C0E9FFE3C0EAFFEF6EB1
:10065000E22B000EE323E02BE123DF06010E120064
:100660000401080E016F100E026F040E036F1200DA
:10067000D9CFE9FFDACFEAFFEE50ED101200D9CF63
:10068000E6FFE1CFD9FF1200E552E7CFD9FF120014
:10069000E0C0E9FFE1C0EAFFEF5023EF03F00401FF
:1006A0001051600BE842E842E842E842E8420009A3
:1006B00001E012001151070A43E00B0A41E0070A6A
:1006C00034E0010A24E00B0A20E0020A1EE0030ADB
:1006D0001AE0080A10E0010A0CE00F0A08E0030A19
:1006E00001E01200010E526E040E576E1200A1EFCF
:1006F00003F0D7EF03F0010E526E0001590EE06FC8
:10070000000EE16F0ED0F1EF03F01FEF04F0010EC9
:10071000526E14510001E06FE16B5A0EE027000E9B
:10072000E1235892010E536E1200010E526E1451C5
:10073000EA6A5A0FE96E000EEA2212C4EFFF1200B5
:100740001200800E0401105D31E11351030A20E014
:10075000010A0BE0030A29E1010E526E0001E40ECA
:10076000E06F0D0EE16F120E1ED0AAD89A0EF6267B
:100770000E0EB8D8020E0001F76AE025F66EE151C0
:10078000F7220900F5CF53F00A00F5CF54F00DD051
:1007900097D89E0EF6260E0EA5D8E0C0F6FFE1C053
:1007A000F7FF0800F550536E546A58821200010E8C
:1007B000526E0F0EE66E270EE66E0F0E9BD8010EE0
:1007C000E66E5A0EE66E000E95D812C459F004017A
:1007D000125103E1050E576E1200060E576EF3EF2D
:1007E00005F00401186B196B040110511F0B020A6C
:1007F0000EE0030A09E0010A17E1010E526E58A04B
:1008000013D00401188310D0010E526E0DD04AD8B7
:1008100001E0010E5ED8E2C0E9FFEA6EEF50040B82
:1008200003E00401010E186F520408E10001180EE4
:10083000E06F040EE16F5892020E536E1200040135
:1008400012050CE110511F0B000908E1010E526E58
:10085000030E115D02E1588001D05890125121E140
:1008600010511F0B02081DE114510F0B000919E074
:1008700019D801E0010E2DD8030E0401115D02E12B
:10088000840E03D014AF07D0400EE2C0E9FFE3C0EE
:10089000EAFFEF6E1200880EE2C0E9FFE3C0EAFF54
:1008A000EF6E1200010E526E14510F0B080DF35033
:1008B0005C6A000F5B6E040E5C221451800B120008
:1008C000010E526E1251F66EF76AD890F636F73670
:1008D0001200040DF35000015B24E26F000E5C2057
:1008E000E36F1200F7220900F5CFE0F00A00F5CF20
:1008F000E1F01200E66E76EC05F0E552E552E552C5
:10090000120065A60CD8570409E165BA07D0626ADF
:100910000F01366B36813689020E576E1200656AFA
:100920000F01366B6586010E576E1200656A0F0166
:10093000366B576A120096EF04F0575001E112002F
:100940006250040B05E00F013651040B01E083D81F
:1009500065B212006250010B05E00F013651010B28
:1009600001E093D86250100B05E00F013651100BD7
:1009700001E01FD86250200B05E00F013651200B1B
:1009800001E071D8030E575C01E21200566A040EB2
:10099000565C0EE26250080B0BE00F013651080B5B
:1009A00007E0DFEC01F0000901E16296562AEFD77B
:1009B0001200D9CFE6FFE1CFD9FF020EE12636CFF4
:1009C000DFFF0F01040E366F629865828C50040BB6
:1009D00001E0010E5B6E8C50080B01E0010E5B1014
:1009E000E76E010EE7CFDBFF8C968C94A198A08870
:1009F0000300A150100B05E1D050080B02E10300E9
:100A0000F8D7A098DF500F013613010EDB50E8B085
:100A10008C86E8A08C96010EDB50E8B08C84E8A0B0
:100A20008C94D50E4F6E020E506E4FC05BF050C0CE
:100A30005CF04F06000E505A5B505C1002E0040060
:100A4000F4D7020EE15C02E2E16AE552E16EE552A2
:100A5000E7CFD9FF120065920F01369562A402D04C
:100A60006294FCD712000F0126A10DD0800E040164
:100A7000005D07E1840E0401045D03E104018C0EB6
:100A8000006F0F012691629A1200636A626A0F0179
:100A90009F0E376F0F017B0E366F0F01386B0F0EF5
:100AA000E66E270EE66E0F0EE66E20D8E552E55292
:100AB000E5520F01160E266F62A605D0629600D091
:100AC00000D00000F9D765981FEC03F00401080E70
:100AD000016F0401100E026F040E036F04018C0EEF
:100AE000006F5890596A030E576E1200D9CFE6FF77
:100AF000E1CFD9FFFD0EDBCFE9FFFE0EDBCFEAFF32
:100B0000FC0EDB5004E0EE6AFC0EDB06F9D7E55282
:100B1000E7CFD9FF1200040110511F0B010801E0BB
:100B20001200145101E01200060E115D21E1135173
:100B3000230A1DE0010A0DE0030A19E1020E526EBC
:100B4000590405E10001080EE06F0E0EE16F090E79
:100B50000CD0020E526E590405E100017D0EE06FCB
:100B60000E0EE16F590403E11D0E536E546A588254
:100B700004011051600BE842E842E842E842E842D2
:100B8000010801E0120011510B0A26E0080A19E0E1
:100B9000090A12E0080A09E00B0A05E0080A01E068
:100BA0001200F1EF05F0F2EF05F0020E526E0001B7
:100BB0004A0EE06F000E0BD0020E526E13C44AF0C4
:100BC0001200020E526E00014B0EE06F000EE16F3C
:100BD0005892010E536E1200020E526E12C44BF068
:100BE0001200120012004C6A0F011E0E276F040142
:100BF000400E096F200E0A6F040E0B6F880E086FEF
:100C00000401600E0E6F040E0F6F400E0C6F120089
:100C1000D9CFE6FFE1CFD9FFE652FC0EDB5040080A
:100C200005E2400EF36EFC0EF3CFDBFFDF6AFC0E35
:100C3000DB50DF5C0FE2DF504DD8EF50E66EDF5047
:100C4000EA6A600FE96E040EEA22E552E750EF6EA1
:100C5000DF2AEDD7FC0EDBCF0DF4400E04010C179C
:100C60000C7D880E0C13E552E552E7CFD9FF120038
:100C7000D9CFE6FFE1CFD9FF4C6A040108BF25D0E8
:100C8000FC0EDBCF5BF00951D8805B5403E2FC0E15
:100C900009C4DBFF4C6AFC0EDB504C5C0FE24C508D
:100CA000EA6A200FE96E040EEA22EF50E66E4C501D
:100CB00011D8E552E750EF6E4C2AEDD70401400EF3
:100CC000096F0817087D880E08134C50E552E7CFCE
:100CD000D9FF1200E76EFD0EDBCFE9FFFE0EDBCF82
:100CE000EAFFE750E926000EEA2212001DEE00F0AE
:100CF0002DEE00F0F86AF66A100EF76E0800F55057
:100D0000FF0808E1010EF66E100EF76E0800F550B0
:100D1000FF0806E080AE02D000EF08F080AEFED7FC
:100D200001D812000DD8040034D837D8060E575C0D
:100D300005E16550020B02E125EC00F0F4D712004A
:100D4000600ED36E9B8C580E4F6E020E506E4FC0CD
:100D50005BF050C05CF04F06000E505A5B505C10C8
:100D6000F6E165A604D06592656AC7EC01F00F0153
:100D7000140E396F576A586A596A19EC00F04D6AB7
:100D80004E6A8C968C94959695940F01486B496B9E
:100D9000120081EC04F09DEF04F04D504E1004E180
:100DA000100E4D6E270E4E6E4D06000E4E5A060E5C
:100DB000575C02E28C868C94060E575C12E14D5013
:100DC0004E100FE10001E65102E18C868C94030E77
:100DD000E65D02E18C968C84E62BE651030801E285
:100DE000E66B12001201000200000008D8043C006B
:100DF00002000102000109022900010100C03209BC
:100E00000400000203000000092111010001221D5D
:100E100000070581034000010705010340000104AC
:100E200003090434034D006900630072006F00631E
:100E300000680069007000200054006500630068CD
:100E4000006E006F006C006F0067007900200049A1
:100E5000006E0063002E0026034800490044002075
:100E600000550053004200200042006F006F0074E4
:100E7000006C006F0061006400650072000600FFF6
:100E80000901A10119012940150026FF00750895E7
:100E9000408100190129409100C0F60DF60D1F0E8A
:100EA000230E570E160BC00EF36E00EE00F00E0E62
:100EB00001D81200EA6002D0EE6AFCD7F350E96074
:060EC0001200EE6AFCD7EF
:0610000091EF6AF01200FE
:0610080074EF24F0120059
:0610180018EF39F0120090
:10102A0004000DD6000000060000E100000004D60E
:10103A000000B70E00000900000002D60000F1050A
:10104A0000000200000084D50000800200007E003B
:10105A000000020100000000000132000000000050
:10106A000180004D00000002000000000000013273
:10107A00000000000001A700FBFFDFFF015700EF9F
:10108A00FF0400014E00F2FF0700014C00F3FF08C5
:10109A0000014A00F5FF0A00014400F8FF0B0001B5
:1010AA004800FAFF0D00014E00FCFF0F000150003E
:1010BA00FFFF100001320000000A00012E000200AA
:1010CA00090001330002000A00012D000400080093
:1010DA00012D0004000800012F000500080001315D
:1010EA000007000700012E00070006000132000871
:1010FA00000600013300090005000136000A000459
:10110A00000134000A0003000139000B000300014A
:10111A003D000C0002000141000D000100014600E3
:10112A000E0001000146000E00FFFF0141000D0004
:10113A00FFFF013D000C00FEFF013E000C00FDFF19
:10114A000139000B00FDFF0136000A00FCFF0133E4
:10115A00000900FBFF0132000800FAFF0135000810
:10116A0000F9FF012E000600F9FF012E000600F922
:10117A00FF012D000400F8FF012D000400F8FF0113
:10118A002E000200F7FF012E000200F7FF013200D5
:10119A000000F6FF012D000000F7FF012E00FEFF00
:1011AA00F7FF012900FEFFF8FF012B00FDFFF8FF02
:1011BA00012F00FBFFF8FF012B00FBFFF9FF0131B4
:1011CA0000F9FFF9FF012E00F9FFFAFF013200F8DA
:1011DA00FFFAFF013300F7FFFBFF013600F6FFFCC1
:1011EA00FF013900F5FFFDFF013900F5FFFDFF01A1
:1011FA003D00F4FFFEFF014100F3FFFFFF0146003F
:10120A00F2FFFFFF013200F6FF010001C6020000F3
:10121A008E00015B00EEFFFEFF015100F0FFFDFFB3
:10122A00014800F3FFFAFF014100F5FFF9FF013C15
:10123A0000F7FFF8FF013A00FAFFF6FF013600FC5B
:10124A00FFF6FF013C00FFFFF4FF0128000100F850
:10125A00FF0129000200F8FF0126000300F9FF013F
:10126A002B000500F9FF012E000700FAFF012F00ED
:10127A000800FBFF0133000900FBFF013F000C00DF
:10128A00FCFF010000000000000201000000000055
:10129A000132000000000001CE003F006A00020097
:1012AA0000000000000132000000000001120200EC
:1012BA000096FF0141000D000100013E000C0003F1
:1012CA00000134000A000300012F00080005000194
:1012DA0040000A000800013D0007000A00011B0047
:1012EA0002000500011B0002000500013C0001008C
:1012FA000C00013700FFFF0B00012F00FDFF090062
:10130A00013600FAFF0900013500F9FF0800013D26
:10131A0000F6FF0700013C00F5FF0500014400F359
:10132A00FF0400014600F2FF010001000000000076
:10133A00000201000000000001320000000000016C
:10134A00900164FF4AFF0200000000000001320021
:10135A000000000001A200FBFFE0FF012D00F7FFE3
:10136A00FFFF012600F9FFFDFF011D00FBFFFDFF46
:10137A00012000FBFFFCFF012700FBFFFAFF012B06
:10138A0000FDFFF8FF012E00FEFFF7FF013200FF0C
:10139A00FFF6FF0132000100F6FF0133000200F6FA
:1013AA00FF012B000300F8FF0127000500FAFF01E7
:1013BA002A000600FAFF012B000700FBFF012B00A1
:1013CA000800FDFF012F000900FDFF016000130066
:1013DA00FEFF019B001F000000012B00F9FF050022
:1013EA00012A00FAFF0600012700FBFF0600012878
:1013FA0000FCFF0700012400FCFF0600012400FE98
:10140A00FF0700012800FFFF0800012800FFFF086E
:10141A0000012D0001000900012D00010009000151
:10142A002F0003000900012D000400080001280014
:10143A0004000700012E0006000700012E00070025
:10144A000600013200080006000133000900050009
:10145A00013100090004000136000A0004000134C9
:10146A00000A000300016B00150004000173001755
:10147A00000100015000100000000151001000FEA0
:10148A00FF0148000E00FDFF014A000E00FBFF01AC
:10149A004A000E00FBFF0141000B00F9FF0140006A
:1014AA000A00F8FF0139000800F8FF013D000700B3
:1014BA00F6FF013C000500F5FF0138000200F5FFC8
:1014CA000141000100F3FF0128000000F8FF012993
:1014DA0000FEFFF8FF012400FEFFF9FF012800FCCF
:1014EA00FFF9FF012800FCFFF9FF012E00FAFFF9BE
:1014FA00FF012E00F9FFFAFF012B00F9FFFBFF01A4
:10150A0087001B0000000196000000E2FF01DE03D5
:10151A003AFF0000017D00E7FF0000016900EBFFD0
:10152A000200015600EFFF0300014400F3FF04002C
:10153A00013800F6FF0500013D00F6FF07000135FE
:10154A0000F8FF0700013D00F9FF0A00013A00FA1E
:10155A00FF0A00013F00FCFF0C00013D00FEFF0CEA
:10156A0000014600FFFF0E000150000100100001BB
:10157A004E0004000F0001480006000D000144005F
:10158A0008000B00012000040005000127000600E6
:10159A0005000122000600030001260007000300DF
:1015AA000124000700020001290008000200015579
:1015BA00001100010001000000000000020100000B
:1015CA000000000132000000000001EA008A00E584
:1015DA00FF020000000000000132000000000001CC
:1015EA006900EBFFFFFF015B00EEFFFDFF014F000B
:1015FA00F1FFFBFF012200FAFFFDFF012200FAFFC3
:10160A00FDFF013C00F7FFF8FF013900F9FFF7FF82
:10161A00013400FDFFF6FF013300FEFFF6FF01383B
:10162A00000200F5FF0134000300F6FF013900074C
:10163A0000F7FF013C000900F8FF011D000500FD4D
:10164A00FF0126000700FDFF014A000E00FBFF0113
:10165A005B001200FDFF0164001400FFFF0164003B
:10166A001400010001560011000300014F000F0091
:10167A0005000145000C000700013C0009000800B4
:10168A00013900070009000131000400090001378F
:10169A000001000B00013200FFFF0A00013600FCC6
:1016AA00FF0A00013900F9FF0900013C00F7FF08B1
:1016BA0000014300F4FF0600014A00F2FF050001A1
:1016CA005600EFFF0300015F00EDFF01000100007B
:1016DA0000000000020100000000000132000000CA
:1016EA00000001770176FF4EFF02000000000000B3
:1016FA000132000000000001A200FBFFE0FF012D03
:10170A0000F7FFFFFF012600F9FFFDFF011D00FBA7
:10171A00FFFDFF012000FBFFFCFF012700FBFFFA92
:10172A00FF012B00FDFFF8FF012E00FEFFF7FF016E
:10173A003200FFFFF6FF0132000100F6FF0133001D
:10174A000200F6FF012B000300F8FF012700050045
:10175A00FAFF012A000600FAFF012B000700FBFF2F
:10176A00012B000800FDFF012F000900FDFF0160A9
:10177A00001300FEFF019B001F000000012B00F96F
:10178A00FF0500012A00FAFF0600012700FBFF06F9
:10179A0000012400FCFF0600012800FCFF070001ED
:1017AA002400FEFF0700012800FFFF0800012800AF
:1017BA00FFFF0800012D0001000900012D000100B2
:1017CA000900012F00030009000128000400070096
:1017DA00012D0004000800012E0006000700012E5A
:1017EA000007000600013200080006000133000964
:1017FA00000500013100090004000136000A000456
:10180A00000134000A000300016B00150004000106
:10181A007300170001000150001000FFFF01500083
:10182A001000FFFF0148000E00FDFF014A000E00F4
:10183A00FBFF014A000E00FBFF0141000B00F9FF0C
:10184A000140000A00F8FF0139000800F8FF013DD5
:10185A00000700F6FF013C000500F5FF0138000211
:10186A0000F5FF0141000100F3FF0128000000F824
:10187A00FF012900FEFFF8FF012400FEFFF9FF0126
:10188A002800FCFFF9FF012800FCFFF9FF012E00E8
:10189A00FAFFF9FF012E00F9FFFAFF012B00F9FF09
:1018AA00FBFF0187001B0000000196000000E2FF19
:1018BA0001DE033AFF0000017D00E7FF0000016935
:1018CA0000EBFF0200015600EFFF0300014400F3A2
:1018DA00FF0400013800F6FF0500013D00F6FF078E
:1018EA0000013500F8FF0700013D00F9FF0A000179
:1018FA003A00FAFF0A00013F00FCFF0C00013D001C
:10190A00FEFF0C00014600FFFF0E0001500001001F
:10191A001000014E0004000F0001480006000D00EF
:10192A0001440008000B0001200004000500012406
:10193A000006000400012400060004000126000736
:10194A000003000124000700020001290008000228
:10195A000001550011000100010000000000000212
:10196A000100000000000132000000000001EA004E
:10197A008A00E5FF020000000000000132000000BA
:10198A000000016900EBFFFFFF015B00EEFFFDFFB6
:10199A00014F00F1FFFBFF012200FAFFFDFF0122C8
:1019AA0000FAFFFDFF013C00F7FFF8FF013900F9DB
:1019BA00FFF7FF013400FDFFF6FF013800FEFFF5D7
:1019CA00FF0133000200F6FF0134000300F6FF01B5
:1019DA0039000700F7FF013C000900F8FF011D006C
:1019EA000500FDFF0128000700FCFF0149000E0069
:1019FA00FCFF015B001200FDFF0164001400FFFF01
:101A0A000164001400010001560011000300014F97
:101A1A00000F0005000145000C000700013C000909
:101A2A00000800013900070009000131000400091B
:101A3A000001370001000B00013200FFFF0A00011C
:101A4A003600FCFF0A00013900F9FF0900013C00D9
:101A5A00F7FF0800014300F4FF0600014A00F2FF05
:101A6A000500015600EFFF0300015F00EDFF0100D2
:101A7A000100000000000002010000000000013225
:101A8A000000000000018D0189FF32FF0200000002
:101A9A000000000132000000000001960000001E54
:101AAA0000012C063C01000001A5000000DFFF0137
:101ABA00300290FF0000012B000700FBFF012A0003
:101ACA000600FAFF0127000500FAFF0127000500BA
:101ADA00FAFF0126000300F9FF0124000200F9FFC2
:101AEA000124000200F9FF0128000000F8FF012D7F
:101AFA00000000F7FF012900FEFFF8FF012900FEA0
:101B0A00FFF8FF012D00FCFFF8FF012F00FBFFF893
:101B1A00FF012B00FBFFF9FF012E00F9FFFAFF017D
:101B2A002B00F9FFFBFF012F00F8FFFBFF0131003B
:101B3A00F7FFFCFF013600F6FFFCFF013400F6FF59
:101B4A00FDFF013900F5FFFDFF013C00F4FFFFFF37
:101B5A00017800E8FFFEFF014600F2FF000001479E
:101B6A0000F2FF0200013D00F4FF0200013D00F413
:101B7A00FF0200013B00F5FF0400013600F6FF04F6
:101B8A0000013300F7FF0500013300F7FF050001EC
:101B9A003100F9FF0700012E00F9FF0600012B00B2
:101BAA00FBFF0700012B00FBFF0700012D00FCFFD4
:101BBA000800012400FEFF0700012900FEFF0800BB
:101BCA00012D000000090001280000000800012979
:101BDA000002000800012600030007000126000396
:101BEA0000070001270005000600012A000600067A
:101BFA0000012E0007000600012F00080005000161
:101C0A009100E3FF00000201000000000001320021
:101C1A000000000001C10074000000020000000082
:101C2A00000001320000000000015F00EDFFFFFF2D
:101C3A00015000F0FFFFFF014800F2FFFDFF0136EF
:101C4A0000F6FFFCFF012800F9FFFCFF012700FA5C
:101C5A00FFFBFF012000FBFFFCFF012300FBFFFB52
:101C6A00FF012200FDFFFAFF011B00FEFFFBFF013F
:101C7A002000FEFFFAFF0123000000F9FF013200F5
:101C8A000100F6FF0131000400F7FF0139000700E7
:101C9A00F7FF0140000A00F8FF0145000C00F9FFB8
:101CAA000154001000FBFF0156001100FDFF0169FD
:101CBA00001500FFFF01690015000100015B001219
:101CCA00000300014F000F00050001220006000377
:101CDA000001220006000300013C0009000800017F
:101CEA0035000700080001360004000A000132002E
:101CFA0001000A00013200FFFF0A00013600FCFF62
:101D0A000A00013900F9FF0900014000F6FF080046
:101D1A00014300F4FF0600014F00F1FF05000156E0
:101D2A0000EFFF0300016400ECFF01000100000066
:101D3A000000000201000000000001320000000063
:101D4A0000011001FFFF5DFF02000000000000011A
:101D5A00320000000000014B000F00FFFF014600A7
:101D6A000E00FFFF0148000E00FDFF013E000C00BF
:101D7A00FDFF013B000B00FCFF013C000B00FBFFD9
:101D8A000136000900FAFF0135000800F9FF012AAF
:101D9A00000600FAFF012B000500F9FF01280004E4
:101DAA0000F9FF0128000400F9FF012B000300F8E5
:101DBA00FF0129000200F8FF0128000100F8FF01D5
:101DCA002D000000F7FF0132000000F6FF012E008F
:101DDA00FEFFF7FF012E00FEFFF7FF012B00FDFFBC
:101DEA00F8FF012F00FBFFF8FF012B00FBFFF9FFB3
:101DFA00012E00FAFFF9FF013200F8FFFAFF013263
:101E0A0000F8FFFAFF012F00F8FFFBFF013800F688
:101E1A00FFFBFF013400F6FFFDFF013900F5FFFD6E
:101E2A00FF013D00F4FFFEFF014100F3FFFFFF0148
:101E3A004100F3FF0000016900EBFF0000016000B0
:101E4A00EDFF0200015200F0FF0400014A00F2FF18
:101E5A000500014300F4FF0600013D00F6FF0700FC
:101E6A00014000F7FF0900014000F8FF0A00013FA6
:101E7A0000FAFF0B00013C00FBFF0B00013D00FED6
:101E8A00FF0C00013C00FFFF0C0001320000000AB9
:101E9A0000012E0002000900012E000200090001C3
:101EAA002D0004000800012D0004000800012F0085
:101EBA0005000800012E0007000600013100070096
:101ECA00070001320008000600013300090005007E
:101EDA000136000A0004000134000A000300013E32
:101EEA00000C000300013D000C0002000146000E38
:101EFA000001000146000E00010001000000000080
:101F0A000002010000000000013200000000000190
:101F1A0039000000DEFF020000000000000132006C
:101F2A0000000000016900EBFFFFFF015B00EEFF0C
:101F3A00FDFF014F00F1FFFBFF012200FAFFFDFF49
:101F4A00012400FAFFFCFF014000F6FFF8FF013D03
:101F5A0000F9FFF6FF013600FCFFF6FF013C00FF27
:101F6A00FFF4FF013C000100F4FF0136000400F613
:101F7A00FF013D000700F6FF0140000A00F8FF01DB
:101F8A0024000600FCFF0122000600FDFF015400A8
:101F9A001000FBFF015B001200FDFF016900150044
:101FAA00FFFF016400140001000156001100030044
:101FBA00014F000F00050001260007000300012061
:101FCA0000050004000143000A0009000139000766
:101FDA00000900013B0004000B0001370001000B5F
:101FEA0000013C00FFFF0C00013600FCFF0A000163
:101FFA003D00F9FF0A00014000F6FF080001200039
:10200A00FBFF0400012600F9FF0300014F00F1FF66
:10201A000500015B00EEFF0300016400ECFF010014
:10202A00010000000000000201000000000001326F
:10203A00000000000001BC01B0FF02FF0200000026
:10204A000000000132000000000001AC00DEFFFBCE
:10205A00FF014300FDFF0D00013C00FFFF0C0001E2
:10206A0028000100080001230001000700012400E4
:10207A0002000700011D000300050001190003000A
:10208A0004000120000500040001190004000300F7
:10209A00011D0005000300012300070001000133B0
:1020AA00000A0002000191001D000100019402844F
:1020BA00000000017300000017000196001E0000D6
:1020CA00000173000000E9FF011D01390000000151
:1020DA00C9001700DFFF019001B0FF000001A00056
:1020EA000000E0FF019600E2FF000001A0000000EE
:1020FA002000019E027AFF0000014600F2FF000064
:10210A00012300F9FFFFFF011D00FBFFFDFF011581
:10211A0000FDFFFDFF011B00FEFFFBFF011E00FF8C
:10212A00FFFAFF0147000200F2FF01000000000071
:10213A00000201000000000001320000000000015E
:10214A0058075AFF5C040200000000000001320038
:10215A000000000001C701A8FFE9FF0141000000DB
:10216A00F3FF015C014400F1FF014C00F1FFFEFFA7
:10217A00011001CBFFF4FF0141000000F3FF01C78A
:10218A00015800E9FF013C0000000C00010701CDE5
:10219A00FF0D00015700EFFF040001570011000472
:1021AA000001050133000B00013C0000000C000196
:1021BA000601CDFF0C00016100EDFF040001610082
:1021CA001300040001060133000C00014100000065
:1021DA000D000100000000000002010000000000E4
:1021EA000132000000000001FF00A8FF83FF020087
:1021FA0000000000000132000000000001C6015882
:10220A000016000141000000F3FF010501CDFFF5B2
:10221A00FF016200EDFFFBFF0161001300FCFF01FB
:10222A0005013300F5FF0141000000F3FF0105013C
:10223A00CDFFF5FF015700EFFFFCFF01570011002A
:10224A00FCFF0107013300F3FF013C000000F4FF2B
:10225A0001C701A8FF170001410000000D0001108D
:10226A000135000C00014C000F000300015C01BCA9
:10227A00FF0F0001410000000D00020100000000F4
:10228A00000132000000000001AC00000099FF02CA
:10229A000000000000000132000000000001C60139
:1022AA0058001600013C000000F4FF010601CDFFB2
:1022BA00F4FF016200EDFFFBFF0160001300FDFF68
:1022CA000106013300F4FF0141000000F3FF01059C
:1022DA0001CDFFF5FF015700EFFFFCFF0157001189
:1022EA0000FCFF0107013300F3FF013C000000F48A
:1022FA00FF01C701A8FF170001410000000D0001FE
:10230A00100135000C00014C000F000300015C01B4
:10231A00BCFF0F0001410000000D00020100000097
:10232A00000001320000000000019B000000A3FF32
:10233A000200000000000001320000000000015508
:10234A0000110000000146000000F2FF015500EFF5
:10235A00FF000001460000000E000201000000001C
:10236A0000013200000000000197001C00AAFF02D1
:10237A0000000000000001320000000000014100DE
:10238A00FFFFF3FF012400F9FF0200012000FAFF1A
:10239A000200011900FCFF0300012000FBFF0400FA
:1023AA00011D00FDFF0500011B00FEFF0500011BCA
:1023BA0000FEFF0500011E000000060001280001C2
:1023CA00000800012400020007000124000400069E
:1023DA000001230005000500012400060004000195
:1023EA002B0008000300012E000900020001320040
:1023FA000A0000000137000B000000012E0009004E
:10240A00FEFF012B000800FDFF0128000700FCFF6A
:10241A000123000500FBFF0124000400FAFF012646
:10242A00000300F9FF0123000000F9FF0123000067
:10243A0000F9FF012200FDFFFAFF012200FDFFFA69
:10244A00FF012700FAFFFBFF012400FAFFFCFF014E
:10245A002B00F8FFFDFF012E00F7FFFEFF013700FA
:10246A00F5FFFFFF011500FCFF0100011301000049
:10247A003700012300F9FFFFFF012000FAFFFEFFEA
:10248A00011B00FBFFFEFF011600FCFFFEFF011906
:10249A0000FDFFFCFF011500FDFFFDFF011500FF18
:1024AA00FFFCFF011900FFFFFBFF011E000100FAFC
:1024BA00FF0120000400FBFF0123000500FBFF01D0
:1024CA002B000800FDFF01000000000000020100CF
:1024DA000000000001320000000000015000190055
:1024EA002900020000000000000132000000000084
:1024FA0001CD000000D7FF012D00090001000126CF
:10250A000007000300011C00040004000115000379
:10251A000003000116000200040001190000000572
:10252A000001140000000400011600FEFF0400016F
:10253A001200FEFF0300011500FDFF030001190050
:10254A00FCFF0300011600FCFF0200011900FBFF5B
:10255A000100011900FBFF0100010000000000005A
:10256A000201000000000001320000000000019793
:10257A0000C4FFBCFF02000000000000013200009E
:10258A00000000013E00FDFFF4FF011900FBFFFF00
:10259A00FF011900FCFFFDFF011D00FDFFFBFF010C
:1025AA002900FEFFF8FF0124000200F9FF012200C2
:1025BA000300FAFF0120000500FCFF0120000600CD
:1025CA00FEFF0123000700FFFF0141000D0000008C
:1025DA00012400FAFF0400011D00FDFF0500011B94
:1025EA0000FEFF0500011E00FFFF06000123000197
:1025FA000007000124000200070001200004000572
:10260A00000127000600050001260007000300015B
:10261A002B000800030001280008000100012D001A
:10262A0009000100013C000C00FFFF0139000B000A
:10263A00FDFF0138000A00FBFF012E000700FAFF28
:10264A000116000200FCFF0116000200FCFF011542
:10265A00000100FCFF0119000000FBFF011E000041
:10266A0000FAFF012200FDFFFAFF012000FCFFFB38
:10267A00FF012300FBFFFBFF0132000A00000001FB
:10268A0037000000F5FF017C01B4FF0000015A0089
:10269A00EEFF0100011E00FAFF0100011900FBFF15
:1026AA000100012F00F8FF0500012E00FAFF0700C4
:1026BA00012D00FCFF0800013200FFFF0A00012380
:1026CA00000100070001190001000500011B0002BA
:1026DA00000500011D0003000500011900040003A4
:1026EA0000011D0005000300011E00060001000193
:1026FA0023000700000001000000000000020100A2
:10270A000000000001320000000000015A003500FC
:10271A00F6FF020000000000000132000000000085
:10272A00012800F8FF0000012300F9FFFFFF012044
:10273A0000FAFFFEFF011D00FBFFFDFF011500FD72
:10274A00FFFDFF011500FDFFFDFF011500FFFFFC66
:10275A00FF011500FFFFFCFF0115000100FCFF014E
:10276A0015000100FCFF0115000300FDFF0119001F
:10277A000300FCFF011B000500FEFF01200006000C
:10278A00FEFF011E000600FFFF01280008000000EE
:10279A0001280008000000011E00060001000120B7
:1027AA000006000200011D000500030001150003D8
:1027BA0000030001150003000300011500010004D5
:1027CA000001150001000400011500FFFF040001CB
:1027DA001500FFFF0400011500FDFF0300011500AD
:1027EA00FDFF0300011D00FBFF0300011B00FBFFAF
:1027FA000200012300F9FF0100012300F9FF000094
:10280A000100000000000002010000000000013287
:10281A000000000000019100CBFFBBFF0200000096
:10282A0000000001320000000000013E00FDFFF43C
:10283A00FF011900FBFFFFFF011900FCFFFDFF016B
:10284A002200FDFFFAFF012400FEFFF9FF01290023
:10285A000200F8FF011D000300FBFF012000050034
:10286A00FCFF0122000600FDFF0123000700000013
:10287A000141000D00FFFF012700FAFF0500011DBD
:10288A0000FDFF0500011B00FEFF0500011E00FF01
:10289A00FF060001230001000700012000020006D4
:1028AA0000012400040006000124000600040001BF
:1028BA00280007000400012B00080003000128007B
:1028CA0008000100012D0009000100013C000C0074
:1028DA00FFFF0139000B00FDFF0138000A00FBFF72
:1028EA00012E000700FAFF0116000200FCFF011684
:1028FA00000200FCFF0115000100FCFF01190000A5
:10290A0000FBFF011E000000FAFF012200FDFFFA92
:10291A00FF012000FCFFFBFF012300FBFFFBFF017F
:10292A0032000A0000000137000000F5FF017C01B7
:10293A00B4FF0000015A00EEFF0100011E00FAFF79
:10294A000100011900FBFF0100012F00F8FF05003B
:10295A00012A00FAFF0600013100FCFF09000132DA
:10296A0000FFFF0A00011E0001000600011E00010F
:10297A00000600011B000200050001190003000403
:10298A0000011C0004000400011B000500020001F4
:10299A0020000600020001230007000000010000D9
:1029AA0000000000020100000000000132000000E7
:1029BA000000015A003500F6FF0200000000000086
:1029CA0001320000000000012800F8FF0000012485
:1029DA0000F9FFFEFF011E00FAFFFFFF011D00FBC9
:1029EA00FFFDFF011500FDFFFDFF011500FDFFFDC5
:1029FA00FF011500FFFFFCFF011500FFFFFCFF01AF
:102A0A0015000100FCFF0115000100FCFF0119007F
:102A1A000300FCFF0115000300FDFF011B00050078
:102A2A00FEFF0120000600FEFF011E000600FFFF58
:102A3A000128000800FFFF01280008000100011E0C
:102A4A00000600010001200006000200011B00052B
:102A5A00000200011900030004000115000300032D
:102A6A000001150001000400011500010004000125
:102A7A001500FFFF0400011500FFFF040001150007
:102A8A00FDFF0300011500FDFF0300011D00FBFF10
:102A9A000300011900FBFF0100012400F9FF0200F5
:102AAA00012300F9FF0000010000000000000201FC
:102ABA00000000000001320000000000016F00F772
:102ACA00FFBEFF020000000000000132000000000B
:102ADA0000014B000F00000001C3000000D9FF01F4
:102AEA004B00F1FF000001C30000002700020100B3
:102AFA000000000001320000000000017B00DBFF43
:102B0A00C0FF0200000000000001320000000000C7
:102B1A0001370000000B000162027A000000013C4C
:102B2A00000000F4FF01DC00D4FF000001240006CD
:102B3A0000FCFF011D000300FBFF011D000300FB59
:102B4A00FF011E000000FAFF0123000000F9FF0147
:102B5A002200FDFFFAFF012400FCFFFAFF0120001A
:102B6A00FBFFFCFF012800F9FFFCFF012900F8FF29
:102B7A00FEFF012900F8FFFEFF012D00F7FFFFFF0E
:102B8A00013700F5FF0100013300F6FF0200012BB7
:102B9A0000F8FF0300012800F9FF0400012300FBED
:102BAA00FF0500012000FCFF0500012000FEFF06D2
:102BBA0000011E00FFFF0600011E000100060001C1
:102BCA002000020006000120000400050001240084
:102BDA0006000400013700F5FF00000201000000B2
:102BEA00000001320000000000014B002D0000002F
:102BFA00020000000000000132000000000001464F
:102C0A0000F2FFFFFF012F00F7FFFDFF011D00FB90
:102C1A00FFFDFF011C00FCFFFCFF011600FEFFFC8C
:102C2A00FF011900FFFFFBFF0115000100FCFF0176
:102C3A0010000100FDFF0119000300FCFF0119004B
:102C4A000400FDFF011B000500FEFF011B0005003B
:102C5A00FEFF0123000700FFFF0128000800FFFF15
:102C6A000128000800010001230007000100011EDD
:102C7A000006000100011D00050003000115000304
:102C8A0000030001150003000300011600020004FE
:102C9A0000011400000004000114000000040001F7
:102CAA001200FEFF0300011900FDFF0400011500D8
:102CBA00FDFF0300011D00FBFF0300011E00FAFFD8
:102CCA000100012400F9FF0200012300F9FF0000BE
:102CDA0001000000000000020100000000000132B3
:102CEA000000000000016900FFFFC1FF02000000B0
:102CFA0000000001320000000000013C000C00FF4F
:102D0A00FF0133000A00FEFF012D000800FCFF014D
:102D1A002B000700FBFF0120000400FBFF011D0040
:102D2A000300FBFF0120000200FAFF01230000005C
:102D3A00F9FF0123000000F9FF012600FDFFF9FF5A
:102D4A00011D00FDFFFBFF012A00FAFFFAFF012423
:102D5A0000FAFFFCFF012B00F8FFFDFF012E00F730
:102D6A00FFFEFF013200F6FF0000014B00F1FF01F8
:102D7A0000011E00FAFF0100011B00FBFF02000117
:102D8A003300F7FF0500013100F9FF0700013100A8
:102D9A00FCFF0900012D00FFFF09000128000100C6
:102DAA0008000120000200060001240004000600B9
:102DBA000123000500050001240006000400012B80
:102DCA0000080003000133000A0002000132000A71
:102DDA0000010001000000000000020100000000E4
:102DEA0000013200000000000116000000F3FF029B
:102DFA00000000000000013200000000000128006D
:102E0A00F8FF0000012400F9FFFEFF011E00FAFF8F
:102E1A00FFFF011900FCFFFDFF011900FCFFFDFF88
:102E2A00011900FDFFFCFF011500FFFFFCFF01195E
:102E3A0000FFFFFBFF0115000100FCFF0115000167
:102E4A0000FCFF0119000300FCFF0119000400FD4A
:102E5A00FF011D000500FDFF011B000500FEFF012B
:102E6A0028000800FFFF01280008000000012300D5
:102E7A0007000000012300070001000120000600EE
:102E8A000200011D000500030001150003000300F4
:102E9A0001190003000400011500010004000115D6
:102EAA000001000400011900FFFF0500011500FFE1
:102EBA00FF0400011900FDFF0400011500FDFF03D6
:102ECA0000011D00FBFF0300011E00FAFF010001C3
:102EDA002400F9FF0200012800F8FF0000010000A9
:102EEA0000000000020100000000000132000000A2
:102EFA00000001AB00E1FF9EFF020000000000009D
:102F0A0001320000000000014200F3FFFEFF012D24
:102F1A0000FFFF0900011E0000000600011B00025D
:102F2A000005000115000300030001160004000259
:102F3A0000012300070001000137000B0001000116
:102F4A00FF0033000000012D0000000900013700D6
:102F5A000B000000012D000000F7FF016E001600B3
:102F6A000000014F000900F3FF019B00E1FF000090
:102F7A00013C000000F4FF013700F5FF0000013CAE
:102F8A000000000C00010401CCFF0000012800F839
:102F9A00FF0000011500FDFFFDFF011500FFFFFC0A
:102FAA00FF0119000000FBFF010000000000000201
:102FBA0001000000000001320000000000012200B0
:102FCA00F3FFF0FF020000000000000132000000E1
:102FDA000000015500110000000146000000F2FF48
:102FEA00015500EFFF000001460000000E0002013B
:102FFA0000000000000132000000000001960020DD
:10300A0000ACFF02000000000000013200000000D6
:10301A0000013D00FEFFF4FF012300F9FF0100015A
:10302A002000FAFF0200012200FAFF0300011C003F
:10303A00FCFF0400011C00FCFF0400011D00FDFF51
:10304A000500012000FEFF0600011900000005002E
:10305A0001280001000800012000020006000124E6
:10306A0000040006000123000500050001240006F3
:10307A00000400012B0008000300012D00090001D3
:10308A00000137000B0001000141000D00FFFF01A4
:10309A003E000C00FDFF011B000500FEFF011900A8
:1030AA000400FDFF0119000400FDFF0119000300DF
:1030BA00FCFF012D000400F8FF0132000100F6FFB9
:1030CA000119000000FBFF011E00FFFFFAFF0119B2
:1030DA0000FDFFFCFF011900FDFFFCFF011C00FCC5
:1030EA00FFFCFF011D00FBFFFDFF011B00FBFFFEB4
:1030FA00FF012300F9FFFFFF013D00FEFF0C000165
:10310A0029000800020001240006000400011D0035
:10311A0003000500011E0001000600011400000062
:10312A000400011600FEFF0400011900FDFF04005F
:10313A00011500FDFF0300011D00FBFF0300012034
:10314A0000FAFF0200012300F9FF0100012800F83C
:10315A00FF0000012800F8FF0000012300F9FFFF2B
:10316A00FF012000FAFFFEFF011D00FBFFFDFF012A
:10317A001500FDFFFDFF011500FDFFFDFF01150014
:10318A00FFFFFCFF011500FFFFFCFF012400020006
:10319A00F9FF0124000400FAFF0112000300FEFFF8
:1031AA000116000400FEFF012E000900FEFF0100C7
:1031BA0000000000000201000000000001320000CF
:1031CA000000000124000C00EEFF020000000000D5
:1031DA000001320000000000013C000C00FFFF016A
:1031EA0033000A00FEFF012D000800FCFF012B003E
:1031FA000700FBFF0120000400FBFF011D00030084
:10320A00FBFF0120000200FAFF0123000000F9FF82
:10321A000123000000F9FF012600FDFFF9FF01224A
:10322A0000FDFFFAFF012700FAFFFBFF012400FA65
:10323A00FFFCFF012B00F8FFFDFF012E00F7FFFE48
:10324A00FF013200F6FF0000014B00F1FF0100010F
:10325A001E00FAFF0100011B00FBFF020001330000
:10326A00F7FF0500013100F9FF0700013100FCFFFB
:10327A000900012D00FFFF090001230001000700DA
:10328A0001240002000700012400040006000123B3
:10329A00000500050001240006000400012B0008B7
:1032AA000003000133000A0002000132000A000193
:1032BA0000010000000000000201000000000001FF
:1032CA003200000000000116000000F3FF020000B7
:1032DA000000000001320000000000012800F8FF91
:1032EA00FFFF012300F9FFFFFF012000FAFFFEFFA5
:1032FA00011600FCFFFEFF011C00FCFFFCFF01158C
:10330A0000FDFFFDFF011500FFFFFCFF011900FF93
:10331A00FFFBFF0115000100FCFF0115000100FC85
:10332A00FF0119000300FCFF0119000400FDFF0161
:10333A001D000500FDFF011B000500FEFF0128001E
:10334A000800FFFF0128000800FFFF012300070013
:10335A00010001230007000100012000060002000D
:10336A00011D0005000300011500030003000119F7
:10337A00000300040001150001000400011500010A
:10338A00000400011900FFFF0500011500FFFF04FA
:10339A0000011500FDFF0300011900FDFF040001F3
:1033AA001B00FBFF0200012000FAFF0200012300BC
:1033BA00F9FF0100012800F8FF01000100000000E8
:1033CA0000000201000000000001320000000000BD
:1033DA00018B00D4FFB9FF02000000000000013297
:1033EA00000000000001B801580000000137000089
:1033FA0000F5FF013C00F4FF00000124000600FC78
:10340A00FF0124000400FAFF0122000300FAFF0171
:10341A0023000100F9FF012300FFFFF9FF01220049
:10342A00FDFFFAFF012300FBFFFBFF012000FAFF6B
:10343A00FEFF012B000700FBFF0127000500FAFF32
:10344A000120000200FAFF011E000100FAFF011923
:10345A00000000FBFF011900FFFFFBFF011900FD3F
:10346A00FFFCFF011500FDFFFDFF011900FCFFFD38
:10347A00FF011B00FBFFFEFF011E00FAFFFFFF0119
:10348A002300F9FF0000013101C3FF0000013C00E5
:10349A0000000C0001180138000000012300070099
:1034AA000100011E000600010001100003000100D6
:1034BA0001150003000300011600020004000114B4
:1034CA000000000400010F0000000300011500FFC6
:1034DA00FF0400011200FEFF0300011200FDFF02BB
:1034EA0000011500FDFF0300011900FBFF010001A7
:1034FA003D00F4FF020001FF00CDFF0000013C0087
:10350A0000000C00011D0139000000012D00090016
:10351A00010001200006000200011200030002005F
:10352A00010B0001000200011E0001000600011942
:10353A000000000500011D00FDFF0500011C00FC44
:10354A00FF0400012000FAFF0200012900F8FF022F
:10355A0000013200F6FF000001E600D2FF00000180
:10356A00410000000D0002010000000000013200CD
:10357A000000000001ED05CB0089FC0200000000FC
:10358A0000000132000000000001A400F5FFE1FF85
:10359A0001A100F7FFE1FF012201F1FFC8FF0105C8
:1035AA0001F5FFCDFF01DA00F9FFD5FF01B100FBFC
:1035BA00FFDDFF018700FEFFE5FF016E00FEFFEA67
:1035CA00FF020100000000000132000000000001BB
:1035DA00F8013E002801020000000000000132004C
:1035EA000000000001800280FF00000201000000CC
:1035FA00000001320000000000010C02EC0030FF64
:10360A00020000000000000132000000000001ABCF
:10361A0000F7FF2100019500F6FF1C00019600F556
:10362A00FF1C00019D00F4FF1D0001C000F0FF23F4
:10363A000001CE00ECFF2400016300F6FF11000137
:10364A006100F5FF1000016400F4FF100001600042
:10365A00F4FF0F00012A00FAFF0600012700FAFF13
:10366A000500012400FAFF0400012000FAFF02000D
:10367A00012000FAFF0200011E00FAFF0000013CCF
:10368A0000F4FF0000013D00F4FFFEFF014200F3D9
:10369A00FFFEFF014200F3FFFEFF014600F2FF00BA
:1036AA0000013700F5FF0000012D00F7FFFFFF01C1
:1036BA002B00F8FFFDFF012000FBFFFCFF010E00BD
:1036CA00FEFFFEFF010F000000FDFF011000FFFFDB
:1036DA00FDFF0115000100FCFF012D000400F8FFA9
:1036EA000140000800F6FF0120000400FBFF01244E
:1036FA00000200F9FF012E000200F7FF012D000071
:10370A0000F7FF012D00FFFFF7FF012E00FEFFF774
:10371A00FF012800FCFFF9FF012700FBFFFAFF0267
:10372A0001000000000001320000000000019E02BA
:10373A00FF00C9FE02000000000000013200000084
:10374A000000011E0006000000011500040001002F
:10375A000112000300020001160002000400011B0E
:10376A00000200050001190001000500014600FFE2
:10377A00FF0E00014C00FEFF0F00014C00FDFF0F81
:10378A0000018E00FBFF1C00018F00FAFF1C0002E3
:10379A0001000000000001320000000000012902BF
:1037AA00E9FEB4000200000000000001320000003F
:1037BA000000015D00EEFFFBFF014700F2FFFEFF84
:1037CA00013700F5FF0000012F00F7FF0300012772
:1037DA0000FAFF0500012700FBFF0600012600FD95
:1037EA00FF0700012E00FEFF0900015600FDFF1130
:1037FA0000012D00FFFF0900012900FEFF0800015A
:10380A002600FDFF0700012000FCFF05000124003F
:10381A00FAFF0400012800F8FF0100018A01EFFF06
:10382A00B3FF011E000000FAFF0119000100FBFFAF
:10383A000136000400F6FF013A000600F6FF0136E1
:10384A00000600F7FF0160000C00F1FF01280004E8
:10385A0000F9FF0120000200FAFF010B00FFFFFE42
:10386A00FF011000FFFFFDFF012E00F9FFFAFF0123
:10387A008A00EBFFEEFF014B00F4FFF7FF014A005D
:10388A00F6FFF5FF014300F7FFF6FF011D00FDFFFC
:10389A00FBFF011B00FEFFFBFF014B01F3FFBFFF14
:1038AA00010401F6FFCDFF0119000500000001190E
:1038BA0000050001000116000400020001160004C0
:1038CA0000020001350007000800013A0006000A5C
:1038DA00000194000C001B00015E000800110001A9
:1038EA00600009001100011D0003000500011C0011
:1038FA00040004000144000B000800014A000D0006
:10390A000700014A000E0005000147000E000200F0
:10391A00012300070000000123000700FFFF012028
:10392A00000600FEFF011D000500FDFF0120000545
:10393A0000FCFF0124000400FAFF0131000400F733
:10394A00FF013E000300F4FF0141000100F3FF0103
:10395A0046000000F2FF02010000000000013200F0
:10396A0000000000010A000600000002000000003A
:10397A00000001320000000000016600140004008B
:10398A0001510010000200013C000C00000001334C
:10399A00000A00FEFF012D000800FCFF01320008AA
:1039AA0000FAFF0135000800F9FF0143000900F69B
:1039BA00FF014E000A00F4FF014E000A00F4FF0165
:1039CA009E001200E6FF0138012100CBFF015500DD
:1039DA000800F1FF015C000900F0FF01BE000F00C2
:1039EA00DDFF01BF000D00DCFF01B1000A00DEFFB0
:1039FA0001F7000C00D0FF01F5000A00D0FF015AC0
:103A0A00000100EEFF011E00FFFFFAFF011500FF93
:103A1A00FFFCFF011200FEFFFDFF011200FDFFFE89
:103A2A00FF011000FDFFFFFF011000FDFF01000173
:103A3A002E00F7FF0200012F00F7FF0300013900F3
:103A4A00F5FF0300013200F6FF0100013200F6FF24
:103A5A000000012E00F7FF0200013100F7FF040009
:103A6A00013600F7FF0600013900F7FF0700013CA5
:103A7A0000F8FF0900014300F7FF0A00014400F8BB
:103A8A00FF0B00018900F1FF1700019200F1FF19F5
:103A9A0000018B00F2FF1800018000F3FF160002FC
:103AAA0001000000000001320000000000019B013B
:103ABA00C4FFEF0002000000000000013200000015
:103ACA000000015F00EDFF0000015100F0FFFEFF62
:103ADA00013D00F4FFFEFF013100F7FFFCFF011575
:103AEA0000FDFFFDFF011500FDFFFDFF011600FEB1
:103AFA00FFFCFF011500FFFFFCFF013C00FFFFF484
:103B0A00FF014C000200F1FF0156000300EFFF0124
:103B1A0061000400EDFF0162000500EDFF01650090
:103B2A000700EDFF0165000900EEFF013200060003
:103B3A00F8FF0132000600F8FF0135000700F8FF20
:103B4A000131000700F9FF0132000800FAFF0133D2
:103B5A00000900FBFF020100000000000132000022
:103B6A00000000011D00F1FF090002000000000032
:103B7A00000132000000000001FF00F6FFCEFF0145
:103B8A005601F2FFBDFF02010000000000013200F1
:103B9A00000000000186023D01DF00020000000073
:103BAA00000001320000000000019300F7FFE4FF6B
:103BBA00018200F9FFE7FF010701F3FFCDFF019F33
:103BCA0000F9FFE1FF01C500FAFFD9FF01D400FAAD
:103BDA00FFD6FF01DD00FCFFD4FF02010000000058
:103BEA000001320000000000018F01F7FFEF000220
:103BFA0000000000000001320000000000017F0008
:103C0A000B00E9FF014600F2FFFFFF017D00F6FF0E
:103C1A0017000141000D0001000100000000000032
:103C2A00020100000000000132000000000001173C
:103C3A0000F2FF0000020000000000000132000054
:103C4A00000000016A00FDFFEBFF0172000900EBB2
:103C5A00FF015D00050012000201000000000001E2
:103C6A00320000000000012700F4FF1400020000E7
:103C7A000000000001320000000000014F01BDFFFA
:103C8A00FFFF0201000000000001320000000000F6
:103C9A00016E004000EFFF02000000000000013248
:103CAA000000000000010901CBFF00000201000032
:103CBA0000000001320000000000016F003F00EB2D
:103CCA00FF020000000000000132000000000001B5
:103CDA00FA00CEFF000002010000000000013200DD
:103CEA00000000000179003A002C000200000000E8
:103CFA0000000132000000000001F2021D009400E1
:103D0A00020100000000000132000000000001046E
:103D1A0001D5FF6AFF020000000000000132000026
:103D2A0000000001F7021D009500020100000000DA
:103D3A000001320000000000011D01FCFF55FF02D6
:103D4A000000000000000132000000000001BF0274
:103D5A001B008A000201000000000001320000007E
:103D6A000000012B0002001A0002000000000000FF
:103D7A0001320000000000012800FFFF08000124B2
:103D8A0000FEFF0700010700FFFF0100010700FF17
:103D9A00FF0100010E00FEFFFEFF012800FCFFF9F3
:103DAA00FF020100000000000132000000000001D3
:103DBA001800F2FFFEFF02000000000000013200BE
:103DCA0000000000012400020007000115000300A2
:103DDA000300010B00020001000141000D00000078
:103DEA00020100000000000132000000000001EFA3
:103DFA00007AFF33000200000000000001320000D8
:103E0A000000000126000700FDFF0126000700FD53
:103E1A00FF0132000800FAFF012E000700FAFF0135
:103E2A0035000700F8FF0136000600F7FF013600EB
:103E3A000600F7FF013A000600F6FF013800050008
:103E4A00F6FF013B000400F5FF0139000300F5FF0E
:103E5A000133000200F6FF0137000100F5FF012DD2
:103E6A00000000F7FF013200FFFFF6FF012D00FC02
:103E7A00FFF8FF012600FDFFF9FF012300FBFFFB0E
:103E8A00FF011D00FBFFFDFF012200FAFFFDFF01FC
:103E9A001E00FAFFFFFF011E00FAFFFFFF011E00CE
:103EAA00FAFF0100012300F9FF0100013F00F4FFBE
:103EBA000400014300F4FF0600013900F7FF070080
:103ECA00013500F8FF07000201000000000001327E
:103EDA00000000000001F30085003C000200000021
:103EEA000000000132000000000001D600D7FFF4F4
:103EFA00FF02010000000000013200000000000182
:103F0A0040002500F5FF0200000000000001320019
:103F1A000000000001C100DBFF0B000201000000ED
:103F2A00000001320000000000016B003F000C009D
:103F3A000200000000000001320000000000014001
:103F4A0001400000000136013E0000000176027EB9
:103F5A0000FDFF014C000F00FEFF012D000900FFCC
:103F6A00FF0110000300FFFF010B000100FEFF012B
:103F7A0010000100FDFF0119000000FBFF012800ED
:103F8A00FFFFF8FF010B00FFFFFEFF010B00FEFF22
:103F9A00FFFF012D00F7FFFFFF015000F0FFFFFFB9
:103FAA00017B0281FF0100013B01C1FF01000140C9
:103FBA0001C0FF0300010B00FEFF0100010E00FE1D
:103FCA00FF0200011500FFFF0400011900000005AF
:103FDA00000119000100050001150001000400019B
:103FEA00120002000300011000030001000100009A
:103FFA000000000002010000000000013200000081
:10400A0000000147001500DBFF020000000000006D
:10401A000132000000000001BA00EFFFDFFF015982
:10402A0000F8FFF0FF015E00F8FFEFFF0201000059
:10403A0000000001320000000000016D00EBFFC229
:10404A00FF02000000000000013200000000000131
:10405A006200FBFFEDFF016000FEFFEDFF01600063
:10406A00FEFFEDFF015F00FFFFEDFF01C30001004E
:10407A00D9FF01B9000100DBFF02010000000000C6
:10408A0001320000000000015B014300C50002008C
:10409A0000000000000132000000000001C800D842
:1040AA00FFFFFF02010000000000013200000000D3
:1040BA0000015002EBFE22FF020000000000000196
:1040CA00320000000000012800080001000126005B
:1040DA000700030001270006000500012300050070
:1040EA00050001550008000F0001620008001200D7
:1040FA0001B6000D0022000201000000000001329A
:10410A00000000000001F20156001E01020000003A
:10411A0000000001320000000000010C01E8FF303D
:10412A00000201000000000001320000000000014E
:10413A0054002100DAFF02000000000000013200F2
:10414A000000000001FF00EAFF2E0002010000004B
:10415A00000001320000000000019B00B4FFCAFF0A
:10416A0002000000000000013200000000000111FE
:10417A0001E6FF30000201000000000001320000E9
:10418A0000000001EC008A001F000200000000008D
:10419A000001320000000000011C01E9FF340002A6
:1041AA0001000000000001320000000000017C0054
:1041BA00E6FFBAFF02000000000000013200000022
:1041CA00000001C201A6FF01000201000000000078
:1041DA0001320000000000019C005C00F0FF0200B8
:1041EA0000000000000132000000000001C701A524
:1041FA00FF0200020100000000000132000000007E
:10420A000001E60068005B000200000000000001F7
:10421A0032000000000001BD01A7FF0100020100F9
:10422A000000000001320000000000019400590063
:10423A00FFFF020000000000000132000000000041
:10424A00018C01F2FFB2FF020100000000000132FE
:10425A000000000000017C00190046000200000076
:10426A0000000001320000000000018701F2FFB3E4
:10427A00FF020100000000000132000000000001FE
:10428A00CB00AAFF56000200000000000001320025
:10429A0000000000018E01F0FFB2FF0201000000E1
:1042AA0000000132000000000001DD007400C0FFC0
:1042BA00020000000000000132000000000001BD01
:1042CA0001A7FF0100020100000000000132000006
:1042DA00000000019B004B003700020000000000B4
:1042EA000001320000000000014100F5FF07000252
:1042FA000100000000000132000000000001170068
:10430A000000F2FF0200000000000001320000007D
:10431A000000014600FFFF0E00020100000000003D
:10432A00013200000000000119000100F1FF020043
:10433A000000000000013200000000000144000BF0
:10434A000008000201000000000001320000000025
:10435A000001B60093FF0100020000000000000106
:10436A0032000000000001350007000800020100C9
:10437A000000000001320000000000011B000200E2
:10438A00F0FF0200000000000001320000000000FF
:10439A00013900F7FF0700020100000000000132A6
:1043AA00000000000001F2007B004D000200000046
:1043BA0000000001320000000000014400F5FF087F
:1043CA0000020100000000000132000000000001AC
:1043DA00A000A0FFF9FF0200000000000001320067
:1043EA0000000000018A01EFFFB3FF020100000094
:1043FA00000001320000000000015C001A00CFFF3B
:10440A000200000000000001320000000000011359
:10441A0001E7FF3100020100000000000132000044
:10442A00000000016D002200C8FF02000000000029
:10443A000001320000000000013900F7FF07000206
:10444A000100000000000132000000000001A40089
:10445A006200F9FF020000000000000132000000C3
:10446A000000014E0007000E0002010000000000DB
:10447A000132000000000001D40086FF240002007F
:10448A0000000000000132000000000001410000AD
:10449A00000D0002010000000000013200000000CF
:1044AA000001770008004700020000000000000138
:1044BA00320000000000013100070007000201007D
:1044CA000000000001320000000000014302620007
:1044DA00B3FE0200000000000001320000000000EC
:1044EA00015101F2FFBEFF0201000000000001328B
:1044FA000000000000016B0019003B0002000000F0
:10450A0000000001320000000000014B01F3FFBF70
:10451A00FF0201000000000001320000000000015B
:10452A0045002300160002000000000000013200CE
:10453A0000000000014B01F3FFBFFF020100000071
:10454A0000000132000000000001FD009EFF74001F
:10455A0002000000000000013200000000000155C6
:10456A0001F3FFBDFF02010000000000013200005C
:10457A000000000118000300F2FF02000000000022
:10458A00000132000000000001FB001A00D5FF0202
:10459A0001000000000001320000000000017B0061
:1045AA003000380002000000000000013200000064
:1045BA000000018101B3FF010002010000000000B8
:1045CA00013200000000000186004F00F2FF0200E5
:1045DA00000000000001320000000000017C01B46C
:1045EA00FF0000020100000000000132000000008C
:1045FA0000017F004C0000000200000000000001E2
:10460A0032000000000001F4001700D5FF0201008B
:10461A000000000001320000000000015600F3FF14
:10462A003200020000000000000132000000000019
:10463A0001ED001600D6FF02010000000000013261
:10464A00000000000001C400ECFF7400020000003A
:10465A0000000001320000000000018101B3FF00E8
:10466A000002010000000000013200000000000109
:10467A00FD00580084FF0200000000000001320023
:10468A0000000000016D01B7FF00000201000000F8
:10469A0000000132000000000001E400490074003B
:1046AA00020000000000000132000000000001EDDD
:1046BA00001600D6FF0201000000000001320000CF
:1046CA00000000015B00D3FFE1FF020000000000D0
:1046DA000001320000000000013D000A000700024C
:1046EA000100000000000132000000000001160075
:1046FA00F4FF060002000000000000013200000082
:10470A0000000143000C00FAFF0201000000000053
:10471A0001320000000000011700F4FF0700020048
:10472A000000000000013200000000000147000202
:10473A0000F2FF0201000000000001320000000048
:10474A0000018500B1FF0D00020000000000000119
:10475A00320000000000013E000300F4FF020100E5
:10476A000000000001320000000000017F00040088
:10477A004C000200000000000001320000000000AE
:10478A00015001F3FFBEFF020100000000000132E8
:10479A0000000000000102000000FFFF020000000C
:1047AA00000000013200000000000143000900F689
:1047BA00FF020100000000000132000000000001B9
:1047CA001600F7FF0A000200000000000001320094
:1047DA00000000000124000600040002010000009D
:1047EA00000001320000000000010D00FAFFFBFF8B
:1047FA000200000000000001320000000000010277
:10480A00011B00D4FF020100000000000132000079
:10481A000000000102000000FFFF0200000000008B
:10482A0000013200000000000135000800F9FF0213
:10483A000100000000000132000000000001CB006E
:10484A00EBFF7800020000000000000132000000C7
:10485A000000012000050004000201000000000021
:10486A00013200000000000182004E000000020038
:10487A000000000000013200000000000141000BAE
:10488A0000F9FF02010000000000013200000000F0
:10489A000001C30001008BFF0200000000000001BC
:1048AA00320000000000013900080008000201007F
:1048BA00000000000132000000000001AF0E3200CB
:1048CA00CF080201000000000001320000000000D1
:1048DA000201000000000000000000000000E9CF13
:1048EA00E4FFEACFE4FFE652D9CFE6FFDACFE6FFEC
:1048FA00E1CFD9FFE2CFDAFFE6529EA0E9D29E903D
:10490A00FE0ECF6E3D0ECE6E19C530F50501316B28
:10491A000501010E326F05011A511B111C111D11DF
:10492A0017E0D880000E05011A55000E1B55190E06
:10493A001C55000E1D5506E205011A6B1B6B1C6BFC
:10494A001D6B06D005011A07000E1B5B1C5B1D5B65
:10495A0005011A511B111C111D1102E00501326BD0
:10496A000501000501E03DD1050111511211131194
:10497A00141107E10501155116111711181101E15A
:10498A002FD10501D7510DE1050119A302D08C8E53
:10499A0001D08C9E050119A702D08C8A01D08C9A6D
:1049AA000FD00501D7050CE1050119A302D08B84AC
:1049BA0001D08B94050119A702D0898401D089946A
:1049CA000501115112111311141164E0010EE96E5F
:1049DA00050EEA6E0E01B751EE240E01B76F0E01F5
:1049EA00B851EE200E01B86F0E01B951EE200E013A
:1049FA00B96F0E01BA51EE200E01BA6FB7CE4CF064
:104A0A00B8CE4DF0B9CE4EF0BACE4FF04C6A4D6AE0
:104A1A004E6A800E4F164C504D104E104F1028E023
:104A2A00B7CEB7FEB8CEB8FEB9CEB9FEBACEBAFE88
:104A3A000E01BA9F010E050130110501306F050103
:104A4A00010E316F05011107000E125B135B145B37
:104A5A00050119A307D005012807000E295B2A5B67
:104A6A002B5B06D00501282B000E29232A232B2392
:104A7A00050109510501012705010A510501022312
:104A8A0005010B510501032305010C5105010423FE
:104A9A000501326B0501155116111711181164E041
:104AAA00050EE96E050EEA6E0E01BB51EE240E01EB
:104ABA00BB6F0E01BC51EE200E01BC6F0E01BD5141
:104ACA00EE200E01BD6F0E01BE51EE200E01BE6F2B
:104ADA00BBCE4CF0BCCE4DF0BDCE4EF0BECE4FF0AC
:104AEA004C6A4D6A4E6A800E4F164C504D104E104D
:104AFA004F1028E0BBCEBBFEBCCEBCFEBDCEBDFE79
:104B0A00BECEBEFE0E01BE9F040E05013011050188
:104B1A00306F0501010E316F05011507000E165B96
:104B2A00175B185B050119A707D005012C07000EB2
:104B3A002D5B2E5B2F5B06D005012C2B000E2D233F
:104B4A002E232F2305010D510501052705010E51BD
:104B5A000501062305010F5105010723050110511F
:104B6A00050108230501326B0501315139E00501C0
:104B7A00D75107E1050130B18C8C050130B58C881D
:104B8A0009D00501D70506E1050130B18B8C050175
:104B9A0030B5898A00000000000000000000000013
:104BAA0000000000000000000000000000000000FB
:104BBA0000000000000000000000000000000000EB
:104BCA00000000000000000000000501D75103E1C9
:104BDA008C9C8C9805D00501D70502E18B9C899A9B
:104BEA00D7D0030E0501005D01E0A0D00501E45114
:104BFA0001E179D005012105DF6E05011E511F1162
:104C0A0037E1DF50EA6A310FE96E0E0EEA22EF5001
:104C1A000E01EA6AAC25E96EAD51EA22EF6AEA6A48
:104C2A00DF34FE0BEA36E96E790EE9260E0EEA2229
:104C3A00EE6AED6AEA6ADF34FE0BEA36E96E490E7D
:104C4A00E9260E0EEA22EE6AED6ADF50EA6A310FB1
:104C5A00E96E0E0EEA22EF6AEA6ADF34FE0BEA36E2
:104C6A00E96E010EE9260E0EEA22EE6AED6A3BD0E3
:104C7A00EA6ADF34FE0BEA36E96E790EE9260E0E91
:104C8A00EA2222C5EEFF23C5EDFFEA6ADF34FE0BF6
:104C9A00EA36E96E490EE9260E0EEA221EC5EEFF35
:104CAA001FC5EDFFDF50EA6A310FE96E0E0EEA22E8
:104CBA0020C5EFFFEA6ADF34FE0BEA36E96E010E21
:104CCA00E9260E0EEA22EE50ED100DE1EA6ADF3413
:104CDA00FE0BEA36E96E010EE9260E0EEA221EC521
:104CEA00EEFF1FC5EDFF0E01B6510501205D1DE166
:104CFA000E01B05105011E1904E10E01B151050161
:104D0A001F190AE10501010ED86F0501D46B0501CF
:104D1A00E35101E08A9809D00501D86B0501010E1B
:104D2A00D46F0501E35101E08A8832D0040E0501EF
:104D3A00005D2EE10501245124E025C54CF026C56D
:104D4A004DF0D8904D324C32D8904D324C324C50B6
:104D5A00BB6EE1C54EF0E2C54FF0040ED8904E3658
:104D6A004F36E804FBE1300E4E16000E4F16CF0EFA
:104D7A00BA1400014E104C6E4FC04DF04C50BA6E32
:104D8A0004D0BB6ACF0EBA14BA6E0501010E326F97
:104D9A000501325101E190D005011A511B111C1174
:104DAA001D1101E089D00501006B0501275101E0C1
:104DBA007ED034C500F535C501F536C502F537C5CF
:104DCA0003F538C504F539C505F53AC506F53BC5F9
:104DDA0007F53CC508F53DC509F53EC50AF53FC5C9
:104DEA000BF540C50CF541C50DF542C50EF543C599
:104DFA000FF544C510F545C511F546C512F547C569
:104E0A0013F548C514F549C515F54AC516F54BC538
:104E1A0017F54CC518F54DC519F54EC51AF54FC508
:104E2A001BF550C51CF551C51DF552C51EF553C5D8
:104E3A001FF554C520F555C521F556C522F557C5A8
:104E4A0023F558C524F559C525F55AC526F5050192
:104E5A00346B0501356B366B376B386B0501396B73
:104E6A003A6B3B6B3C6B0501456B466B476B486B7A
:104E7A000501496B4A6B4B6B4C6B05014D6B050188
:104E8A004E6B4F6B506B516B0501526B536B0501A7
:104E9A00546B0501556B0501566B576B0501586B31
:104EAA000501596B5A6B0501010E276F05D00501E3
:104EBA001A6B1B6B1C6B1D6B8050800B06E0050187
:104ECA00DF5106E08150010B03E10501010EDE6F9F
:104EDA00E552E552E5CFDAFFE7CFD9FFE552E5CF54
:104EEA00EAFFE5CFE9FF1100D9CFE6FFDACFE6FF07
:104EFA00E1CFD9FFE2CFDAFFE652DF6ADFCF00F077
:104F0A00020EE76E0018E8AE02D0E73402D0E7508E
:104F1A00005C3CE2DFCFE9FFEA6AE9BEEA68D890C2
:104F2A00E936EA36D890E936EA36010EE926050E60
:104F3A00EA22010EEE6EEE6AEE6AEE6ADFCFE9FF52
:104F4A00EA6AE9BEEA68D890E936EA36D890E936DC
:104F5A00EA36110EE926050EEA22EE6AEE6AEE6AD2
:104F6A00EE6ADFCFE9FFEA6AE9BEEA68D890E93675
:104F7A00EA36D890E936EA36090EE926050EEA221B
:104F8A00EE6AEE6AEE6AEE6ADF2AB8D70501006BAE
:104F9A000501196B05011A6B1B6B1C6B1D6B050157
:104FAA001E6B1F6B0501206B0501216B0501226B2E
:104FBA00236B0501010E276FCD82CD9ECD9CCD9A24
:104FCA00CD98CD96CD94FE0ECF6E3D0ECE6ECD8091
:104FDA009F809E909D8092809F9C010EE66EE66A5D
:104FEA002BEC41F0E552E552010EE66E0B0EE66E31
:104FFA002BEC41F0E552E5528D8496948D8296927F
:10500A00898C929C8D8096908B8294928C9C959C94
:10501A008C9E959E8C9895988C9A959A949E828E41
:10502A000000000000000000000000000000000076
:10503A000000000000000000000000000000000066
:10504A00000000000000948E829E0501010EE36FAD
:10505A000501010EE46F8A9893980501010ED46F39
:10506A000501D76B0501010ED86F0501DD6B05013E
:10507A00D96BDA6BDB6BDC6B0501DE6B9380F19E1F
:10508A000501010EDF6F93968196C5EC34F0E55267
:10509A00E552E5CFDAFFE7CFD9FF120017EC35F07A
:1050AA00BAEC36F0F3EC35F015EC39F0E66AD95083
:1050BA00FEEC38F00701B45101E0B3D0DF0424E17B
:1050CA00C3EC36F00CE10501010EE36FE46B6EEC04
:1050DA0036F002E2E16AE552E16E00500DD01CECB6
:1050EA0037F006E1ED5004E10501E36B010E03D050
:1050FA000501010EE36FE46F000EE66EE66AD8C59D
:10510A00E6FF4CEC37F08BD0020EDF5C2EE1C3ECED
:10511A0036F009E10501D76B96909492959C959E7D
:10512A009598959A1BD01CEC37F00DE1ED500BE1E8
:10513A000501010E5AEC37F094949294949C929A39
:10514A00959292926CD0ECEC38F0020EEE1867E170
:10515A00ED5065E10501020E5AEC37F09484928411
:10516A00948C928A958292825AD0040EDF5C07E16F
:10517A00010EDBCFB0FE020EDBCFB1FE50D0050E22
:10518A00DF5C07E1010EDBCFAEFE020EDBCFAFFE26
:10519A0046D0080EDF5C0FE1ECEC38F0180ED88030
:1051AA00EE54000EED5403E2180E66EC37F0010ED1
:1051BA00DBCFAAFE34D0090EDF5C0FE1ECEC38F04D
:1051CA00060ED880EE54000EED5403E2060E66EC8D
:1051DA0037F0010EDBCFABFE22D00A0EDF5C03E113
:1051EA006DEC37F009D00B0EDF5C03E16DEC37F0A4
:1051FA0016D00C0EDF5C07E1010EDBCFB4FE020E07
:10520A00DBCFB5FE0CD00D0EDF5C09E1C3EC36F046
:10521A0004E00501010EDF6F02D00501DF6B97EC98
:10522A0040F0FAEC38F02BEF35F017EC35F0200EA1
:10523A00E12402E3E168E6520AEC38F020EC37F0A8
:10524A00E66AD950040F0DEC39F0060F0DEC39F06F
:10525A00080FF0EC38F00C0F96EC37F0D950040F29
:10526A0008EC37F004E22E0E006EBB0E83D2D95042
:10527A00060F08EC37F004E2000E006EBB0E7AD27D
:10528A00FAEC36F0040E005C000E015804E2D60E69
:10529A00006EBA0E6FD2060EDBCF00F0070EDBCF20
:1052AA0001F0040E005C000E015804E2AE0E006E1E
:1052BA00BA0E60D20701B45101E065D2080EDBCF05
:1052CA0010F0090EDBCF11F00A0EDBCF12F00B0E35
:1052DA00DBCF13F010C038F011C039F012C03AF029
:1052EA0013C03BF0080EDBCF3DF0090EDBCF3EF0DA
:1052FA000A0EDBCF3FF00B0EDBCF40F0A2EC69F0D9
:10530A0034C00CF035C00DF036C00EF037C00FF0C7
:10531A000C0EDBCF14F00D0EDBCF15F00E0EDBCF2B
:10532A0016F00F0EDBCF17F014C038F015C039F0A5
:10533A0016C03AF017C03BF00C0EDBCF3DF00D0E55
:10534A00DBCF3EF00E0EDBCF3FF00F0EDBCF40F08F
:10535A00A2EC69F00C503424086E0D503520096E09
:10536A000E5036200A6E0F5037200B6E01EC37F0C4
:10537A003B6E25EC59F0D7EC35F039C0E6FF3AC060
:10538A00E6FF3BC0E6FF3CC0E6FFA6EC5EF0FAECA7
:10539A0038F0E5528BEC38F038C039F0BBEC38F015
:1053AA0095EC5AF0140E38C0DBFF150E39C0DBFF3E
:1053BA00160E3AC0DBFF170E3BC0DBFF0501275173
:1053CA00FDE04E6B4F6B506B516B4D6B8D908B921A
:1053DA00D950080FAFEC38F002E698EC35F006E247
:1053EA00020E4D6FB7EC37F0F6EC35F0D9500C0FD2
:1053FA00AFEC38F002E698EC35F012E2080E05013F
:10540A004D114D6F0C0EDBCF38F00D0EDBCF39F09E
:10541A000E0EDBCF3AF00F0E31EC35F003EC36F01E
:10542A00C3EC37F002E677EC35F004E2800E006E4A
:10543A00BA0EA0D1CFEC37F002E677EC35F004E2F1
:10544A00520E006EBA0E96D1C7EC36F0D7EC35F094
:10545A00AC0E3E6EC50E3F6EA70E406E470E416EF5
:10546A0091EC59F00FEC37F0DBCF0CF0150EDBCFD7
:10547A000DF0160EDBCF0EF0170EDBCF0FF00CC0BF
:10548A0038F00DC039F00EC03AF00FC03BF023ECF3
:10549A0059F029EC37F060EC35F03EEC59F0180E73
:1054AA0039C0DBFF190E3AC0DBFF1A0E3BC0DBFF27
:1054BA001B0E3CC0DBFFE0EC36F0080EDBCF08F039
:1054CA00090EDBCF09F00A0EDBCF0AF00B0EF3EC64
:1054DA0037F038C035F539C036F53AC037F53BC034
:1054EA0038F5080EDBCF45F5090EDBCF46F50A0E77
:1054FA00DBCF47F50B0EDBCF48F532EC37F029EC62
:10550A0037F032EC37F039C00CF03AC00DF03BC03E
:10551A000EF03CC00FF0A5EC37F008C039F009C016
:10552A003AF00AC03BF00BC03CF091EC59F0D7ECD2
:10553A0035F0C7EC36F039C014F03AC015F03BC06C
:10554A0016F03CC017F0C7EC36F039C018F03AC074
:10555A0019F03BC01AF03CC01BF0A5EC37F014C0A0
:10556A0039F015C03AF016C03BF017C03CF091EC88
:10557A0059F039C010F03AC011F03BC012F03CC0EB
:10558A0013F0A5EC37F004C039F005C03AF006C0B4
:10559A003BF007C03CF0FEEC59F00FEC37F0DBCFE4
:1055AA0028F0150EDBCF29F0160EDBCF2AF0170EE6
:1055BA00DBCF2BF028C038F029C039F02AC03AF0E6
:1055CA002BC03BF023EC59F039C024F03AC025F047
:1055DA003BC026F03CC027F0140EDBCF30F0150E8E
:1055EA00DBCF31F0160EDBCF32F0170EDBCF33F004
:1055FA0030C038F031C039F032C03AF033C03BF035
:10560A0023EC59F039C02CF03AC02DF03BC02EF0F3
:10561A003CC02FF0A5EC37F024C039F025C03AF091
:10562A0026C03BF027C03CF091EC59F039C020F07D
:10563A003AC021F03BC022F03CC023F03E6A3F6AE8
:10564A00406A400E416E91EC59F039C01CF03AC0E4
:10565A001DF03BC01EF03CC01FF060EC35F03EEC84
:10566A0059F01C0E39C0DBFF1D0E3AC0DBFF1E0EBF
:10567A003BC0DBFF1F0E3CC0DBFF080EDBCF04F094
:10568A00090EDBCF05F00A0EDBCF06F00B0E39EC64
:10569A0035F038C03DF539C03EF53AC03FF53BC05C
:1056AA0040F5E0EC36F00C0EDBCF08F00D0EDBCF48
:1056BA0009F00E0EDBCF0AF00F0EF3EC37F038C00C
:1056CA0039F539C03AF53AC03BF53BC03CF50C0E0A
:1056DA00DBCF49F50D0EDBCF4AF50E0EDBCF4BF5CE
:1056EA000F0EDBCF4CF59AEC37F039EC35F038C0B9
:1056FA0041F539C042F53AC043F53BC044F5FAECEE
:10570A0036F0060EDB50001803E1070EDB500118D5
:10571A0014E005013D513E113F1140110EE1D880C0
:10572A00000E4555000E4655000E4755000E4855C9
:10573A0004E2270E006EBA0E1DD0FAEC36F0060E01
:10574A00DB50001803E1070EDB50011816E00501D3
:10575A00415142114311441110E1D880000E4955BC
:10576A00000E4A55000E4B55000E4C5506E2FC0E33
:10577A00006EB90E0FEC38F006D00501010E346F39
:10578A00276B97EC40F0200EE15C02E2E16AE552F9
:10579A00E16E2BEF35F017EC35F03F0EE12402E312
:1057AA00E168E652E16EE5EC37F0E1EC38F0100F13
:1057BA00F0EC38F0040FF0EC38F0080F0DEC39F08B
:1057CA00140FF0EC38F00C0F96EC37F00701B451D7
:1057DA0001E06FD128EC35F00DE1040EDBCF04F0C7
:1057EA00050EDBCF05F0060EDBCF06F0070EA8ECA0
:1057FA0035F011E0100EDBCF08F0110EDBCF09F007
:10580A00120EDBCF0AF0130EDBCF0BF00850091093
:10581A000A100B1035E1080EDBCF0CF0090EDBCFB6
:10582A000DF00A0EDBCF0EF00B0EDBCF0FF00C5093
:10583A000D100E100F1012E10C0EDBCF10F00D0E32
:10584A00DBCF11F00E0EDBCF12F00F0EDBCF13F011
:10585A00105011101210131001E12BD1140EDBCFCE
:10586A0014F0150EDBCF15F0160EDBCF16F0170E5F
:10587A00DBCF17F0145015101610171001E119D1CB
:10588A00320EDB6A330EDB6A340EDB6A350EDB6AF4
:10589A00310EDB6A8D908B92D950100FAFEC38F035
:1058AA0002E698EC35F01FE2310EDB500209E76E92
:1058BA00310EE7CFDBFF100EDBCF38F0110EDBCF56
:1058CA0039F0120EDBCF3AF0130E31EC35F0100E30
:1058DA0034C0DBFF110E35C0DBFF120E36C0DBFF12
:1058EA00130E37C0DBFFD950140FAFEC38F002E6C5
:1058FA0098EC35F015E2310EDB500809E76E310EEF
:10590A00E7CFDBFF140EDBCF38F0150EDBCF39F013
:10591A00160EDBCF3AF0170E31EC35F010EC36F0FC
:10592A00DCEC38F0190EEECFDBFF1A0EEECFDBFF00
:10593A001B0EEECFDBFF1C0EB7EC38F0100F91EC0C
:10594A0037F0290EEECFDBFF2A0EEECFDBFF2B0E50
:10595A00EECFDBFF2C0EB7EC38F0040FE96E000E29
:10596A007DEC36F0D950080F91EC37F01D0EEECFD2
:10597A00DBFF1E0EEECFDBFF1F0EEECFDBFF200E8E
:10598A00B7EC38F0140F91EC37F02D0EEECFDBFFA9
:10599A002E0EEECFDBFF2F0EEECFDBFF300EB7EC75
:1059AA0038F00C0FE96E000E8CEC36F0010EF36E37
:1059BA00180EF3CFDBFF05012751FDE0180EDBCFF0
:1059CA0034F5190EDBCF35F51A0EDBCF36F51B0E83
:1059DA00DBCF37F51C0EDBCF38F51D0EDBCF39F5E3
:1059EA001E0EDBCF3AF51F0EDBCF3BF5200EDBCFC9
:1059FA003CF5210EDBCF3DF5220EDBCF3EF5230E23
:105A0A00DBCF3FF5240EDBCF40F5250EDBCF41F58A
:105A1A00260EDBCF42F5270EDBCF43F5280EDBCF70
:105A2A0044F5290EDBCF45F52A0EDBCF46F52B0EC2
:105A3A00DBCF47F52C0EDBCF48F52D0EDBCF49F532
:105A4A002E0EDBCF4AF52F0EDBCF4BF5300EDBCF18
:105A5A004CF5310EDBCF4DF5320EDBCF4EF5330E62
:105A6A00DBCF4FF5340EDBCF50F5350EDBCF51F5DA
:105A7A00360EDBCF52F5370EDBCF53F5380EDBCFC0
:105A8A0054F5390EDBCF55F53A0EDBCF56F53B0E02
:105A9A00DBCF57F53C0EDBCF58F53D0EDBCF59F582
:105AAA003E0EDBCF5AF5276B0701E35102E097EC74
:105ABA0040F03F0EE15C02E2E16AE552E16E2BEF53
:105ACA0035F017EC35F0100EE12402E3E168E652F6
:105ADA000AEC38F0F3EC35F0EEEC37F0040F96EC04
:105AEA0037F062EC37F0080F96EC37F00E01BF5131
:105AFA006FE028EC35F002E10701B48D0701B451DB
:105B0A0073E1CFEC36F004E2C90E006EB90E5DD037
:105B1A0017EC38F002E6EEEC35F005E2D950040F46
:105B2A004DEC36F004D023EC38F003EC36F0CFEC31
:105B3A0037F002E677EC35F004E2800E006EBA0E1A
:105B4A0044D02FEC38F004E2990E006EB90E3DD025
:105B5A00D9EC34F00C0F81EC35F009E39AEC37F00C
:105B6A00A8EC35F004E0730E006EB90E2ED0C3EC2B
:105B7A0037F002E6EEEC35F005E2D950080F4DECAD
:105B8A0036F004D0B7EC37F003EC36F0CFEC37F050
:105B9A0002E677EC35F004E2520E006EBA0E15D02A
:105BAA002FEC38F004E2430E006EB90E0ED0D9EC99
:105BBA0034F00C0F81EC35F00BE39AEC37F0A8ECDB
:105BCA0035F006E01D0E006EB90E0FEC38F00CD061
:105BDA0000EC38F002E2E16AE552E16E005007019A
:105BEA00E35102E097EC40F0100EE15C02E2E16A58
:105BFA00E552E16E2BEF35F017EC35F0180EE12483
:105C0A0002E3E168E6520AEC38F020EC37F0E1EC06
:105C1A0038F00C0FF0EC38F0100F96EC37F028EC57
:105C2A0035F002E10701B48D100EDBCF00F0110E42
:105C3A00DBCF01F0120EDBCF02F0130EDBCF03F045
:105C4A00D9500C0F91EC37F0EE500026EE5001229D
:105C5A00EE500222EE500322040E00C0DBFF050EB6
:105C6A0001C0DBFF060E02C0DBFF070E03C0DBFF2D
:105C7A009AEC37F0DBCF07F0D950100F91EC37F0E0
:105C8A00EE50045C006EEE500558016EEE50065858
:105C9A00026EEE500758036E080E00C0DBFF090EB5
:105CAA0001C0DBFF0A0E02C0DBFF0B0E03C0DBFFE5
:105CBA0017EC38F002E6EEEC35F005E2D950040FA5
:105CCA005BEC36F004D023EC38F010EC36F0CFEC75
:105CDA0036F004E2C90E006EB90E4AD03BEC38F039
:105CEA0002E677EC35F004E2800E006EBA0E40D080
:105CFA0047EC38F004E2990E006EB90E39D0D9ECAF
:105D0A0034F0140F81EC35F007E353EC38F004E07B
:105D1A00730E006EB90E2CD0C3EC37F002E6EEEC2F
:105D2A0035F005E2D950080F5BEC36F004D0B7EC39
:105D3A0037F010EC36F03BEC38F002E677EC35F051
:105D4A0004E2520E006EBA0E13D047EC38F004E2A9
:105D5A00430E006EB90E0CD0D9EC34F0140F81EC5E
:105D6A0035F009E353EC38F006E01D0E006EB90E6B
:105D7A000FEC38F00CD00701B45109E100EC38F00F
:105D8A0002E2E16AE552E16E005097EC40F0180E2B
:105D9A00E15C02E2E16AE552E16E2BEF35F017ECC5
:105DAA0035F0370EE12402E3E168E6520AEC38F0F6
:105DBA008BEC35F010EC39F017E15FEC38F014E1B8
:105DCA00020EF36E100EF3CFDBFFBCEC35F02A0E99
:105DDA0034C0DBFF2B0E35C0DBFF2C0E36C0DBFFD9
:105DEA002D0E37C0DBFF64D12A0EDB6A2B0EDB6A6D
:105DFA002C0EDB6A2D0EDB6A290EDB6A8D908B92E4
:105E0A00D950F60FB3EC38F002E698EC35F01FE201
:105E1A00290EDB500209E76E290EE7CFDBFFF60EEB
:105E2A00DBCF38F0F70EDBCF39F0F80EDBCF3AF0E4
:105E3A00F90E31EC35F0F60E34C0DBFFF70E35C043
:105E4A00DBFFF80E36C0DBFFF90E37C0DBFFD95097
:105E5A00F20FB3EC38F002E698EC35F01FE2290EA7
:105E6A00DB500809E76E290EE7CFDBFFF20EDBCF26
:105E7A0038F0F30EDBCF39F0F40EDBCF3AF0F50E43
:105E8A0031EC35F0F20E34C0DBFFF30E35C0DBFF28
:105E9A00F40E36C0DBFFF50E37C0DBFFD950F60F24
:105EAA00B3EC38F002E63AEC37F030E2BCEC35F00D
:105EBA00040E34C0DBFF050E35C0DBFF060E36C00C
:105ECA00DBFF070E37C0DBFF8BEC35F00F0E1F0B25
:105EDA0003E0AFEC35F0FDE1E6EC34F0CCEC35F064
:105EEA008BEC35F00F0E1F0B03E0AFEC35F0FDE144
:105EFA00C2EC38F014E29BEC36F003E0AFEC35F07C
:105F0A00FDE1E6EC34F0EDEC36F009D08BEC35F03F
:105F1A00E0EC35F074EC37F0FDE1F4EC38F0DAEC53
:105F2A0036F00CE265EC35F0E80E006EB80E6FEC58
:105F3A0038F002E2E16AE55212EC37F028EC35F06B
:105F4A0012E1F60EDBCF04F0F70EDBCF05F0F80E08
:105F5A00DBCF06F0F90EA8EC35F005E0BD0E006EB9
:105F6A00B80E03EC39F067EC35F009E2AAEC36F02A
:105F7A0003E07BEC37F0FDE137EC36F006D0B6EC07
:105F8A0036F003E0AFEC35F0FDE161EC36F0110ECE
:105F9A00EECFDBFF120EEECFDBFF130EEECFDBFFF1
:105FAA00140EB7EC38F0F60FE96EFF0E7DEC36F002
:105FBA00190EDB6A1A0EDB6A1B0EDB6A1C0EDB6A21
:105FCA00D950F20FB3EC38F002E63AEC37F022E29D
:105FDA001DEC36F00F0E1F0B03E0AFEC35F0FDE1C0
:105FEA00E6EC34F0CCEC35F01DEC36F00F0E1F0B5E
:105FFA0003E0AFEC35F0FDE1C2EC38F014E29BECC3
:10600A0036F003E0AFEC35F0FDE1E6EC34F0EDEC10
:10601A0036F009D01DEC36F0E0EC35F074EC37F0D0
:10602A00FDE1F4EC38F0DAEC36F00CE265EC35F030
:10603A00880E006EB80E6FEC38F002E2E16AE552A3
:10604A0012EC37F028EC35F008E15FEC38F005E0A7
:10605A005D0E006EB80E03EC39F067EC35F009E21C
:10606A00AAEC36F003E07BEC37F0FDE137EC36F0D2
:10607A0006D0B6EC36F003E0AFEC35F0FDE161ECAA
:10608A0036F078EC38F0180EB7EC38F0F20FE96E0B
:10609A00FF0E8CEC36F01D0EDB6A1E0EDB6A1F0E3D
:1060AA00DB6A200EDB6A010EF36E100EF3CFDBFF04
:1060BA0005012751FDE0100EDBCF34F5110EDBCFC1
:1060CA0035F5120EDBCF36F5130EDBCF37F5140E8E
:1060DA00DBCF38F5150EDBCF39F5160EDBCF3AF5E7
:1060EA00170EDBCF3BF5180EDBCF3CF5190EDBCFD5
:1060FA003DF51A0EDBCF3EF51B0EDBCF3FF51C0E2E
:10610A00DBCF40F51D0EDBCF41F51E0EDBCF42F58E
:10611A001F0EDBCF43F5200EDBCF44F5210EDBCF7C
:10612A0045F5220EDBCF46F5230EDBCF47F5240ECD
:10613A00DBCF48F5250EDBCF49F5260EDBCF4AF536
:10614A00270EDBCF4BF5280EDBCF4CF5290EDBCF24
:10615A004DF52A0EDBCF4EF52B0EDBCF4FF52C0E6D
:10616A00DBCF50F52D0EDBCF51F52E0EDBCF52F5DE
:10617A002F0EDBCF53F5300EDBCF54F5310EDBCFCC
:10618A0055F5320EDBCF56F5330EDBCF57F5340E0D
:10619A00DBCF58F5350EDBCF59F5360EDBCF5AF586
:1061AA00276B370EE15C02E2E16AE552E16E2BEF02
:1061BA0035F017EC35F0110EE12402E3E168E652FE
:1061CA0043EC37F005EC35F0100EDB6A0501275178
:1061DA0002E1340502E0000502E1010EDF6E34053A
:1061EA002BE1346B090E45C5DBFF0A0E46C5DBFF02
:1061FA000B0E47C5DBFF0C0E48C5DBFF0D0E49C56C
:10620A00DBFF0E0E4AC5DBFF0F0E4BC5DBFF100E80
:10621A004CC5DBFF456B466B476B486B496B4A6B5A
:10622A004B6B4C6B3D6B3E6B3F6B406B416B426BF8
:10623A00436B446B010E276F000529E1006B010EC9
:10624A0011C5DBFF020E12C5DBFF030E13C5DBFF10
:10625A00040E14C5DBFF050E15C5DBFF060E16C5B9
:10626A00DBFF070E17C5DBFF080E18C5DBFF116B36
:10627A00126B136B146B156B166B176B186B096B20
:10628A000A6B0B6B0C6B0D6B0E6B0F6B106BD95093
:10629A00050FCEDBD950010FCBDBD9500D0FC8DB70
:1062AA00D950090FC5DBDFCFE6FFE66A480E006E5C
:1062BA00B80EC0DB036E150EE15C02E2E16AE5523C
:1062CA0056EC37F0110EE15C02E2E16AE552E16E4A
:1062DA00BDD3D8C500F0016A00BE016882EC37F070
:1062EA00430E026EB80E2AEC36F002E2E16AE5527B
:1062FA00E16E055097EF40F06BEC38F0DE6ADD6A2C
:10630A00010EE66ED3EC38F0030E47DB0701B451F9
:10631A000FE10501D80504E187EC37F0E66A04D0FD
:10632A0087EC37F0010EE66E4CEC37F097EC40F054
:10633A00E552E5528BD36BEC38F0BAEC36F050EC00
:10634A0037F012EC38F094EC38F08CEC37F00701A7
:10635A00B45129E1030EDB50070802E250EC37F092
:10636A00DF50010802E2010EDF6E030EDB50030F5D
:10637A000E01B65D0CE06EEC36F002E2E16AE5521F
:10638A00E16E0050030EDB50030F0E01B66F010ED3
:10639A00DBCFE6FF020EDBCFE6FFDFCFE6FF4CECFA
:1063AA0037F097EC40F0050EE15C02E2E16AE55253
:1063BA00E16E4CD36BEC38F0E652E652FD0EDB048C
:1063CA000BE1B0CEDEFFB1CEDDFF020EB2CEDBFFB7
:1063DA00030EB3CEDBFF0AD0AECEDEFFAFCEDDFFBB
:1063EA00020EB4CEDBFF030EB5CEDBFFFB0EDBCF16
:1063FA00E6FFFC0EDBCFE6FF020EDBCFE6FF030E65
:10640A00DBCFE6FFB6CEE6FF87EC37F091EC63F020
:10641A00006E070EE15C02E2E16AE552E16E0050AD
:10642A00040EE15C02E2E16AE552E16E0FD36BEC25
:10643A0038F0E652D3DB99EC38F039E10701B45170
:10644A0056E10501D75103E0020ED75D28E1DF507E
:10645A00000821E2D75101E18D90DF0403E18D8428
:10646A008D82898C020EDF5C03E18D848D82899C8A
:10647A00030EDF5C03E18D948D82899C040EDF5C40
:10648A0003E18D848D92899C050EDF5C10E18D9469
:10649A008D92899C0CD0D7510AE18D8008D0D705FE
:1064AA0006E1DF50000802E28C9201D08C8262EC95
:1064BA0037F0010F12DB99EC38F017E10701B451FC
:1064CA0016E10501D75108E1010EDB50000802E28E
:1064DA008B920BD08B8209D0D70507E1010EDB50D6
:1064EA00000802E2899201D0898297EC40F0FAEC26
:1064FA0038F0ACD2FE0E0501D95DFF0EDA59FF0E57
:10650A00DB59FF0EDC5905E2D92B000EDA23DB2317
:10651A00DC2397EF40F00501D951DA11DB11DC11C8
:10652A0005E0D907000EDA5BDB5BDC5B97EF40F036
:10653A006BEC38F0E652E652E65250DB070E2DDAE3
:10654A008CEC37F0DB500BE1DFCFD9F5010EDBCF56
:10655A00DAF5020EDBCFDBF5030EDBCFDCF597ECC9
:10656A0040F0050EE15C02E2E16AE552E16E6ED2AC
:10657A00D9C5E6FFDAC5E6FFDBC5E6FFDCC5E6FFFF
:10658A003A0E006EB80E6FEC38F002E2E16AE5529C
:10659A0056EF37F0E66ADD0EE66E050EE66E15EC8E
:1065AA0039F00701B45101E0120097EF40F0DDC560
:1065BA0000F0016A00BE016882EC37F0330E026E09
:1065CA00B80E43DB02E2E16AE552E16E055097EF4D
:1065DA0040F0DEC500F0016A00BE016882EC37F0C7
:1065EA002D0E026EB80E31DB02E2E16AE552E16E6F
:1065FA0005500501DE6B97EF40F09DBCFED716C132
:10660A00E6FF17C1E6FF00C1E6FF01C1E6FF210E62
:10661A00006EB80E6FEC38F002E2E16AE55256EF0E
:10662A0037F06BEC38F0A1DB030EDB6A12EC38F0C2
:10663A008CEC37F094EC38F00701B45101E081D0CA
:10664A00ECEC38F0FF0ED880EE54030EED5407E25E
:10665A00010EDB68030EF36E020EF3CFDBFFDF5091
:10666A00010802E2010EDF6E030EDB50010802E2AE
:10667A0050EC37F0DF0409E1040EDB50030805E1B2
:10668A000501E16B020EE26F06D0010EDBCFE1F5E8
:10669A00020EDBCFE2F5CAB415D0CB68FC0ECA14E1
:1066AA000009CA6E9D920F0152815293F00EBA14DC
:1066BA000C09BA6E3F0EBA140009BA6E0E010E0E1C
:1066CA00CC6FCA84030EDB502AE1DF5023E0E1C518
:1066DA0000F0E2C501F0D89001320032D8900132C0
:1066EA0000320050BB6EE1C502F0E2C503F0040EB1
:1066FA00D89002360336E804FBE1300E0216000E8B
:10670A000316CF0EBA1400010210006E03C001F086
:10671A00E85003D0BB6ACF0EBA14BA6E10D0050186
:10672A002751FDE0E1C559F5E2C55AF54E6B4F6BAD
:10673A00506B516BDFCF58F5040E346F276B97EC13
:10674A0040F0050EE15C02E2E16AE552E16E7ED1BB
:10675A00120068D92B0EE12402E3E168E6528EDBCF
:10676A00F29E040E00C5DBFF050E01C5DBFF060E17
:10677A0002C5DBFF070E03C5DBFF080E04C5DBFFFE
:10678A00090E05C5DBFF0A0E06C5DBFF0B0E07C5A2
:10679A00DBFF0C0E08C5DBFF0D0E09C5DBFF0E0E75
:1067AA000AC5DBFF0F0E0BC5DBFF100E0CC5DBFFA6
:1067BA00110E0DC5DBFF120E0EC5DBFF130E0FC542
:1067CA00DBFF140E10C5DBFF150E11C5DBFF160E1D
:1067DA0012C5DBFF170E13C5DBFF180E14C5DBFF4E
:1067EA00190E15C5DBFF1A0E16C5DBFF1B0E17C5E2
:1067FA00DBFF1C0E18C5DBFF1D0E19C5DBFF1E0EC5
:10680A001AC5DBFF1F0E1BC5DBFF200E1CC5DBFFF5
:10681A00210E1DC5DBFF220E1EC5DBFF230E1FC581
:10682A00DBFF240E20C5DBFF250E21C5DBFF260E6C
:10683A0022C5DBFF270E23C5DBFF280E24C5DBFF9D
:10684A00290E25C5DBFF2A0E26C5DBFFF28E1E0E9A
:10685A00DBCF00F01F0EDBCF01F0200EDBCF02F002
:10686A00210E74EC38F002E0010EDF6E040EDB50EC
:10687A0002E0010EDF6E0501275106E1010EDF6E0F
:10688A00F36E030EF3CFDBFFDF5010E0150EDBCF04
:10689A0000F0160EDBCF01F0170EDBCF02F0180E58
:1068AA0074EC38F003E0DE52010EDD6EDF5012E0C8
:1068BA00190EDBCF00F01A0EDBCF01F01B0EDBCF77
:1068CA0002F01C0E74EC38F005E0010EF36E020EB5
:1068DA00F3CFDBFF030EDBCFE6FFE66A020EDBCF68
:1068EA00E6FFE66A010EDBCFE6FFE66ADFCFE6FFE8
:1068FA00E66A100E006EB80E9DD8036E0B0EE15CB0
:10690A0002E2E16AE552E16E03502B0EE15C02E21B
:10691A00E16AE552E16E9AD085D8080EE12402E3D5
:10692A00E168E652E16EF29E28C5DFFF010E29C535
:10693A00DBFF020E2AC5DBFF030E2BC5DBFF040EAD
:10694A002CC5DBFF050E2DC5DBFF060E2EC5DBFFB2
:10695A00070E2FC5DBFFF28E08EC39F0060E006E2B
:10696A00B80E68D8036E0B0EE15C02E2E16AE552EA
:10697A0098DA080EE15C02E2E16AE552E16E66D05D
:10698A00F29E0501286B296B2A6B2B6B2C6B2D6BE6
:10699A002E6B2F6BF28E97EF40F0E66E3FEC47F0CE
:1069AA00FAEC38F0E552120001DB1F0E3D6E050EBF
:1069BA003E6E3F6A406ACDDA2CEC6AF0A7DBD9500A
:1069CA001200C7DA040EDBCF3DF0050EDBCF3EF036
:1069DA00060EDBCF3FF0070ED8EF38F0DBCF03F01F
:1069EA00B8DADFCF3DF0010EDBCF3EF0020EDBCF8F
:1069FA003FF0030ED8DBD880190E3854C6EF38F0B2
:106A0A00040EDB6A050EDB6A060EDB6A070EDB6A1A
:106A1A00080EDB6A090EDB6A0A0EDB6A0B0EDB6AFA
:106A2A00E5EF37F0BBDBE1CFD9FFE2CFDAFF1200A7
:106A3A0073DA63D3016E026A00C0E6FFE66E02C033
:106A4A00E6FFCBEF68F0B2DA10EF39F0E552E5CFA6
:106A5A00DAFFE7CFD9FF1200DBCF3BF03D683E6893
:106A6A003F684068A2EF69F0DBCF07F004C038F056
:106A7A0005C039F006C03AF007C03BF025EC59F0E2
:106A8A001C0EDBCF3EF01D0EDBCF3FF01E0EDBCF20
:106A9A0040F01F0EDBCF41F091EC59F04CDB210E98
:106AAA003E6EE60E3F6E5B0E406E400E416E91ECFE
:106ABA0059F095EF5AF044DA00C039F0BBEF38F0DC
:106ACA0076DB1BD3D950FA0FE96EFF0EDA20EA6E95
:106ADA00D8801E0EEE54000E5BD3E66E000EDA204E
:106AEA00E66E1200D880FF0E3954FF0E3A54FF0E9C
:106AFA003B54000E3C5412000FDAEE50385CEE5054
:106B0A003958EE503A58EE503B581200F60EDBCF89
:106B1A0000F0F70EDBCF01F0F80EDBCF02F0F90E32
:106B2A00DBCF03F01200000EEE5C000EEE58000EF2
:106B3A00EE58000EEE581200DA20EA6ED890030ED4
:106B4A00EB50000A1200DBCF07F0045005100610C4
:106B5A0007101200D8900036013602360336E806CE
:106B6A001200DBCF3CF03C34000E3C181200FA0E47
:106B7A00DBCF00F0FB0EDBCF01F0FC0EDBCF02F027
:106B8A00FD0EDBCF03F0E0DAE4D9A2EF69F038C0FA
:106B9A00DEFF39C0DEFF3AC0DEFF3BC0DDFFDD525B
:106BAA00DD52120039C004F03AC005F03BC006F0CD
:106BBA003CC007F01200CDD9FA0EDBCF3DF0FB0E38
:106BCA00DBCF3EF0FC0EDBCF3FF0FD0EECDA0F0E12
:106BDA001200D880D6DA000E3C541200E66AD3EFCF
:106BEA0038F0080E34C0DBFF090E35C0DBFF0A0E91
:106BFA0036C0DBFF0B0E37C0DBFF12000C0E34C0B1
:106C0A00DBFF0D0E35C0DBFF0E0E36C0DBFF0F0EAD
:106C1A0037C0DBFF1200140E34C0DBFF150E35C07F
:106C2A00DBFF160E36C0DBFF170E37C0DBFF120084
:106C3A00F20EDBCF00F0F30EDBCF01F0F40EDBCF68
:106C4A0002F0F50EDBCF03F01200036E046A02C0F5
:106C5A00E6FFE66E04C0E6FFCBEC68F0056E050EB3
:106C6A00E15C1200D9500C0F57D90450EE24006E83
:106C7A000550EE20016E0650EE20026E0750EE20FF
:106C8A00036E1200DE6ADE6ADD6ADD52DD52120030
:106C9A0043D90C0EEECFDBFF0D0EEECFDBFF0E0E4F
:106CAA00EECFDBFF0F0EEECFDBFF120035D9140E4D
:106CBA00EECFDBFF78EF38F000C0DFFF010E01C036
:106CCA00DBFF020E02C0DBFF030E03C0DBFFDCEFBB
:106CDA0038F0000EE66EE66AE66EE66AB6CEE6FFC3
:106CEA00E66EE66A91EC63F0006E070EE15C120054
:106CFA00DA20EA6E210EEECFDBFF220EEECFDBFFAB
:106D0A00230EEECFDBFF240EEECFDBFF1200DA20DC
:106D1A00EA6E250EEECFDBFF260EEECFDBFF270E47
:106D2A00EECFDBFF280EEECFDBFF1200080EDBCF23
:106D3A0000F0090EDBCF01F00A0EDBCF02F00B0EDA
:106D4A00DBCF03F0100E1F0B120031DAEECF04F086
:106D5A00EECF05F0EECF06F0EFCF07F0100E1F0BC7
:106D6A00120024D9100E1F0B1200E652E652E65208
:106D7A00DF6A010EDB6A020EDB6A120028DAEE50C5
:106D8A00ED101200040EDBCF3AF0050EDBCF3BF01C
:106D9A000EEF59F00CDAD880FF0EEE54FF0EEE54C7
:106DAA00FF0EEE54000EEE54120001DAD880000EE7
:106DBA00EE54800EEDD1180EDBCF00F0190EDBCFAA
:106DCA0001F01A0EDBCF02F01B0EDBCF03F012002C
:106DDA000C0E38C0DBFF0D0E39C0DBFF0E0E3AC0B9
:106DEA00DBFF0F0E3BC0DBFF1200040EDBCF00F00F
:106DFA00050EDBCF01F0120008C038F009C039F0E7
:106E0A000AC03AF0120088D8A80ED880EE54610E53
:106E1A00ED54120090D9140E1200E16E0350DE6A8E
:106E2A00800EDE6EDE6ADD6ADD52DD521200CFD9D7
:106E3A00010EEE181200100EDB6A110EDB6A120E3A
:106E4A00DB6A130EDB6A120039C008F03AC009F097
:106E5A003BC00AF03CC00BF01200060EDBCF3AF042
:106E6A00070EDBCF3BF00EEF59F0FF0EEE5CFF0E84
:106E7A00EE58010EEE58000EEE581200E16EDF6A6F
:106E8A00010EDB6A020EDB6A030EDB6A1200DFEC1C
:106E9A0031F0FAEF38F0010EF36E030EF3CFDBFF99
:106EAA001200E16E035097EF40F0D76F96809482FC
:106EBA00958C958E9588958A1200010EE66ED950AA
:106ECA001200F36E010EF3CFDBFF020EDB6A120033
:106EDA00010EDBCFB2FE020EDBCFB3FE1200D8905A
:106EEA00383639363A363B36E8061200D890043638
:106EFA00053606360736E806120000C0E6FF01C06E
:106F0A00E6FF1200DECFE6FFDDCFE6FF1200E76EF6
:106F1A00040EE7CFDBFF1200E96E000EDA20EA6EFC
:106F2A001200DBDD060ED2EF34F00C0EDBCF04F0DC
:106F3A000D0EDBCF05F00E0EDBCF06F00F0E1200A2
:106F4A0039C03EF03AC03FF03BC040F03CC041F08F
:106F5A00120000C038F001C039F002C03AF003C094
:106F6A003BF01200080EDBCF38F0090EDBCF39F008
:106F7A000A0EDBCF3AF00B0E31EF35F0080EDBCFFD
:106F8A0039F0090EDBCF3AF00A0EDBCF3BF00B0EDD
:106F9A00B6EF35F00C0EDBCF39F00D0EDBCF3AF041
:106FAA000E0EDBCF3BF00F0EB6EF35F000D9EECF69
:106FBA0000F0EECF01F0EECF02F0EFCF03F01200B7
:106FCA000C0EDB6A0D0EDB6A0E0EDB6A0F0EDB6A35
:106FDA001200070EE2DCE66AD9501200DBCF0BF092
:106FEA000BDF0BC03BF025EC59F0DCDD64DD91ECE6
:106FFA0059F095EF5AF0D950080F1ADD04D9D4EC9C
:10700A002EF0006E0C0EE15C1200E16EDE6A3ADED2
:10701A0005EF35F00FDDFAEF38F0E0DD01D94DDF8D
:10702A00FEEF38F0040EDBCF39F0050EDBCF3AF075
:10703A00060EDBCF3BF0070EB6EF35F0040EDBCFC2
:10704A0038F0050EDBCF39F0060EDBCF3AF0070E2B
:10705A0031EF35F00C0EDBCF00F00D0EDBCF01F077
:10706A000E0EDBCF02F00F0EF3EF34F0140EDBCF6F
:10707A0039F0150EDBCF3AF0160EDBCF3BF0170EC8
:10708A00B6EF35F0140EDBCF00F0150EDBCF01F0B2
:10709A00160EDBCF02F0170EF3EF34F0140EDBCF2F
:1070AA0004F0150EDBCF05F0160EDBCF06F0170E37
:1070BA00A8EF35F0F20EDBCF04F0F30EDBCF05F0CC
:1070CA00F40EDBCF06F0F50EA8EF35F0ABDCE65296
:1070DA00E6521200AFDC036E070EE15C1200DBCF52
:1070EA0003F010EF39F0150EEECFDBFF160EEECFE0
:1070FA00DBFF170EEECFDBFF1200EECFE6FFEECF7F
:10710A00E6FFEECFE6FFEFCFE6FF120038C000F051
:10711A0039C001F03AC002F03BC003F01200CDDEE4
:10712A00030FDBDC15EF39F07BD8E76E020EE7CFF1
:10713A00DBFFDB50120039C000F03AC001F03BC05F
:10714A0002F03CC003F01200190E3D6E3E6A3F6A1F
:10715A00406A1200E96E000EA1EF35F0E96EFF0EEB
:10716A00A1EF35F0EECFDBFFD950120001C03AF0A3
:10717A0002C03BF003C03CF0120023DC32DD67EFB3
:10718A0035F0000E3954000E3A54000E3B541200EA
:10719A00EE54000EEE54000EEE541200D9CFE6FF64
:1071AA00DACFE6FF1200DBCF40F02CEF6AF0D9CF3E
:1071BA00E9FFDACFEAFF1200140EDB6A150EDB6A6A
:1071CA00160EDB6A170EDB6A09DDEEEF37F0D950CF
:1071DA00010F91EF37F0A5DEE66AD9501200B4DF4D
:1071EA002CEC6AF0D4DCE5EF37F0E552E552E552D3
:1071FA001200010F72DC030ED2EF34F00BDF010E26
:10720A00DE6E47EF36F0D950040F12DC65EF35F029
:10721A0064DCEEEF37F00050011002100310120088
:10722A00010ED2EF34F0D8CFE4FFE0CFE4FFE46EF2
:10723A00E9CFE4FFEACFE4FFF3CFE4FFF4CFE4FFC2
:10724A00E6524AEC4BF0B1EC4AF0030EDB6AA4A614
:10725A00A4D1A4960E01002B0E01AB510E01005DC4
:10726A0001E284D0006B0E0179EC4AF0EF6A799062
:10727A007B6A7A6A0E01A92B0E01AA510E01A95D39
:10728A0001E3A96B40EC4BF0EA22EE50ED106EE000
:10729A0009EC4CF0B6EC4BF002E14B50491847E0D0
:1072AA0054EC4BF0EA22EE50ED103AE077EC4BF05A
:1072BA0055EC4AF040EC4BF0EA22EE504A5C486E3C
:1072CA00EE504B58496E020E48C0DBFF030E49C010
:1072DA00DBFFCCEC4AF0493412E248500008000EB9
:1072EA0049540DE2CCEC4AF054EC4BF08DEC4BF0E7
:1072FA0017E2EFEC4BF0EE264950ED2218D0CCEC19
:10730A004AF0486C491E000E492254EC4BF08DECB1
:10731A004BF006E2EFEC4BF0EE5E4950ED5A07D027
:10732A0009EC4CF0EA2248C0EEFF49C0EDFF79ECC7
:10733A004AF0120EEF6EF29E0E0140EC4BF011EC89
:10734A004AF049C048F0496A4850B66E40EC4BF0E2
:10735A0011EC4AF04850B56EF00EB4140009B46E40
:10736A00F00EB4140909B46E7980F28E0701000E8A
:10737A00D880AA55000EAB552EE2B82B000EB923C1
:10738A00AA51B85DAB51B95926E3B86BB96B030E74
:10739A00AE5D1FE2AC51EA6A200FE96E010EEA22E5
:1073AA0080CFEFFFAC51EA6A230FE96E010EEA22A1
:1073BA0081CFEFFFAC51EA6A260FE96E010EEA228D
:1073CA0082CFEFFFAC2B030EAC5D01E3AC6BAE2BAF
:1073DA0002D0AA6BAB6B000ED880AF55000EB05529
:1073EA001CE2000ED880BE55000EBF5516E2BA2B1D
:1073FA00000EBB23AF51BA5DB051BB590EE3BA6B55
:10740A00BB6B030EB35D07E2B12B030EB15D01E363
:10741A00B16BB32B02D0AF6BB06BBE51BF110BE097
:10742A00050EBD5D07E3C18C9E9C9D8CC280C28205
:10743A00BD6B01D0BD2B0601005101E1AAD0DE6A65
:10744A00DD6ADECF48F0DDCF49F0040E485C000E5D
:10745A00495801E39ED0F8EC49F0010E5BEC4AF082
:10746A00FDE1010EE926060EEA22EE50ED1075E066
:10747A00F8EC49F0010E5BEC4AF0FDE1BAEC4BF096
:10748A00EE50ED1016E1BFEC4BF001E18180C3EC48
:10749A004BF003E1ED5001E18182C7EC4BF003E1CF
:1074AA00ED5001E18184CBEC4BF003E1ED5001E1B9
:1074BA008186F8EC49F0010E5BEC4AF0FDE16DECD7
:1074CA004BF05BEC4AF0FDE1010EE926060EB6EC44
:1074DA004BF019E14B50491816E1BFEC4BF001E1B2
:1074EA008190C3EC4BF003E1ED5001E18192C7ECCE
:1074FA004BF003E1ED5001E18194CBEC4BF003E159
:10750A00ED5001E18196F8EC49F0010E5BEC4AF08E
:10751A00FDE1BAEC4BF0EE2A000EEF22F8EC49F04E
:10752A00010E5BEC4AF0FDE16DEC4BF05BEC4AF0CE
:10753A00FDE1090EE926060EB6EC4BF024E14B50AC
:10754A00491821E1F8EC49F0010E5BEC4AF0FDE143
:10755A00BAEC4BF0EE6AED6A16D0BFEC4BF001E1E3
:10756A008190C3EC4BF003E1ED5001E18192C7EC4D
:10757A004BF003E1ED5001E18194CBEC4BF003E1D8
:10758A00ED5001E18196DF2A010E01E25AD7DB2A8A
:10759A0058D70501E05101E0E0079EAC3DD09E9C22
:1075AA00C1AC07D0C19C010E0701C06FC16BBC6B97
:1075BA0018D0C4504A6E4B6E4A6AC35000014A1032
:1075CA00486E4BC049F00701BC51E96EEA6AA6EC65
:1075DA004AF048C0EEFF49C0EDFFD890C037C13726
:1075EA00BC2B100EBC5D0EE2C051BE15486EC151D7
:1075FA00BF15496E4850491005E1BC2BD890C037D9
:10760A00C137EFD7100EBC5D02E39D9C05D0BC517B
:10761A00040DF328C26EC282F2A435D0D59EF2942C
:10762A00F29A040E486E0701B751B7EC4AF0EF50D0
:10763A00485C29E1080EB75D0AE2EAEC4AF004E088
:10764A00E846FE0B4806FCE1E81C891616D0100E27
:10765A00B75D0AE2EAEC4AF004E0E846FE0B4806A7
:10766A00FCE1E81C8A1609D0EAEC4AF004E0E84694
:10767A00FE0B4806FCE1E81C8B160701B751B7EC74
:10768A004AF0020EEF6E040EE15C02E2E16AE55294
:10769A00E16EE552E5CFDAFFE7CFD9FFE552E5CF54
:1076AA00F4FFE5CFF3FFE5CFEAFFE5CFE9FFE550C9
:1076BA00E5CFE0FFE5CFD8FF1000F5EC4BF0E6523E
:1076CA00896A92680701BE6BBF6B8A6A93688B6A84
:1076DA0094688C968C9495969594928E010EE36F8D
:1076EA000501F169F2690701B26BB16BB36BAD6B5E
:1076FA00AC6BAE6BAA6BAB6BAF6BB06BB86BB96BA9
:10770A00BA6BBB6BBC6B76827680769C769A7688EF
:10771A007696FA0E776EDE6ADD6A40EC4AF004E687
:10772A00100E005C000E01580BE2F8EC49F0A6ECD2
:10773A004AF0EE6AED6ADF2A010EEFE3DB2AEDD7A3
:10774A000701DD6BDE6BDB6BDC6BDE6ADD6A40EC4E
:10775A004AF004E6400E005C000E01580CE2F8EC18
:10776A0049F0000EE926020EEA22EF6ADF2A010E2C
:10777A00EEE3DB2AECD7DE6ADD6A40EC4AF004E687
:10778A00400E005C000E01580CE2F8EC49F0400E85
:10779A00E926020EEA22EF6ADF2A010EEEE3DB2A6D
:1077AA00ECD7DE6ADD6A40EC4AF004E6000E005CC3
:1077BA00010E01580AE2F8EC49F0F6EC4AF0EF6AD9
:1077CA00DF2A010EF0E3DB2AEED70701DF6BE06B5D
:1077DA00E16BE26BB56BB66BB76BDE6ADD6A40ECE8
:1077EA004AF004E6180E005C000E015812E2F8ECAA
:1077FA0049F000EC4BF0EE6AED6AF8EC49F0290E1C
:10780A00E926010EEA22010EEF6EDF2AE8E3DB2AFF
:10781A00E6D7D586D59AD59CF294F29AF1940F01BF
:10782A00498FBE0EC16ED08E7694A386A59679EC4A
:10783A0027F0C5EC62F0F28EF28C76840FEC46F0FB
:10784A00040EE15C02E2E16AE552E16EDBEF49F027
:10785A004AEC4BF0E652B1EC4AF0030EDB6A040E36
:10786A00DB6AFFEC48F00701AE5100080AE2DCECE3
:10787A0041F00701AD2B030EAD5D01E1AD6BAE0723
:10788A00F2D7B35100080AE2FEEC41F00701B22B2D
:10789A00030EB25D01E1B26BB307F3D7200E040108
:1078AA00E76E7819E8AE02D0E73402D0E750785D87
:1078BA0001E23AD16550020B01E036D1400EE66E84
:1078CA00400EE66E020EE66E5CEC61F0F9EC4BF0EF
:1078DA00E76E030EE7CFDBFFDB50000801E3E7D0DA
:1078EA00040EDB6A030EDB50F36E040E5EEC4AF004
:1078FA0001E3DDD0040EDB50EA6A400FE96E020EA6
:10790A00EA22EFCFDFFF06015D5134E10D0E1CECD8
:10791A004AF005E00A0E016EDF50015C2BE1010E10
:10792A005D6F070168EC4AF00D0EEF6EDD2B010E5C
:10793A00DB6ADD51F36E010E5EEC4AF016E2FBECF7
:10794A004AF0E9BEEA68F6EC4AF0EF50E66EFBEC64
:10795A004AF0E9BEEA68190EE926060EEA22E5525D
:10796A00E750EF6E010EDB2AE4D73BD90701DD6B46
:10797A00DE6B8DD01B0EDF5C09E1595107E1010E68
:10798A00596F1B0E5A6F5B6B5C6B81D059050BE10B
:10799A005B0EDF5C08E11B0E5A5D05E15B5103E1FA
:1079AA005B0E5B6F74D059054AE1410EDF5C47E11B
:1079BA001B0E5A5D44E15B0E5B5D41E15A6B5B6BEA
:1079CA005C6B596B010EDB6ADBCFE9FFEA6AE9BE41
:1079DA00EA68F6EC4AF0EF500D0816E0FBEC4AF0C4
:1079EA00E9BEEA68190EE926060EEA22EF50E66EAB
:1079FA00FBEC4AF0E9BEEA68F6EC4AF0E552E750D9
:107A0A00EF6E010EDB2AE0D7010EDBCFDDF70701AF
:107A1A0068EC4AF0EF6A3C0E006EBD0E36EC4BF095
:107A2A00000EE66E030EE66E390E006EBD0E3DECDC
:107A3A004BF002E2E16AE552E16E035028D0080EEB
:107A4A00DF5C0EE10701DD5100080AE2DD0768ECA0
:107A5A004AF0EF6A360E006EBD0E36EC4BF017D0C8
:107A6A000D0EDF5C14E00A0EDF5C11E0200EDF5C15
:107A7A000EE306015A6B5B6B5C6B596B070168EC92
:107A8A004AF0DFCFEFFF06015D6B0701DD2B07012F
:107A9A00DD51006E016A000E001806E1010E0118A0
:107AAA0003E1B487DD6BDE6B040EDB2A1BD707010B
:107ABA00B45139E0B4A105D0300E006EBD0E36ECDB
:107ACA004BF00701B4A305D0110E006EBD0E36ECC3
:107ADA004BF00701B4A505D0F50E006EBC0E36ECCE
:107AEA004BF00701B4A705D0D90E006EBC0E36ECD8
:107AFA004BF00701B4A905D0BA0E006EBC0E36ECE5
:107B0A004BF00701B4AD05D0990E006EBC0E36ECF1
:107B1A004BF00701B4AF05D0800E006EBC0E36ECF8
:107B2A004BF00701B46B37D8050EE15C02E2E16A5B
:107B3A00E552E16EDBEF49F04AEC4BF0DBC7DFFFC1
:107B4A00DF2A400E1CEC4AF001E1DF6A0701DC5132
:107B5A00DF5C01E120D80701DB51EA6A000FE96E18
:107B6A00020EEA22FD0EDBCFEFFFDB2B400EDB5DC0
:107B7A0001E1DB6BDC51DB5D01E1B485FD0EDBCF9E
:107B8A0000F0016A00BE016800C0F3FF01C0F4FF03
:107B9A00E552DBEF49F04AEC4BF00701DB51DC5DC3
:107BAA001DE00701905105E0E6EC61F095EC4CF020
:107BBA00F8D70701DC51D880DB5507E2DC51DB5DE1
:107BCA0032EC4AF0DBC7DCF707D0400ED880DC5530
:107BDA0032EC4AF00701DC6BE6EC61F0E552DBEFD0
:107BEA0049F0F5EC4BF0E652DE6ADD6A020EDB6A1A
:107BFA00030EDB6A0701E1EC49F00CEC4BF0020ED4
:107C0A00F3CFDBFF0701FDEC49F004E1010E011897
:107C1A0001E1DE6B020EDB50DE6EDD6AE1EC49F05B
:107C2A002C0824E0E1EC49F00D0820E0E1EC49F0F1
:107C3A000CEC4BF0030EF3CFDBFF0701FDEC49F030
:107C4A0004E1010E011801E1DE6B020EDBCF02F046
:107C5A0002C003F0026A030EDB5000010224006E28
:107C6A00000E0320016E00C0DEFFDD6E000EDFCFC6
:107C7A003AF0010EDBCF3BF0420E3A1802E1520E07
:107C8A003B1801E11FD2540E3A1802E1510E3B187B
:107C9A0001E115D2540E3A1802E1530E3B1801E1E4
:107CAA000BD2530E3A1802E1430E3B1801E101D2FE
:107CBA00530E3A1802E1510E3B1801E1F7D14D0E6D
:107CCA003A1802E1580E3B1801E1EDD1530E3A1869
:107CDA0002E1450E3B1801E1E3D1430E3A1802E1F5
:107CEA00410E3B1801E1DAD14D0E3A1802E1510E6C
:107CFA003B1801E1D0D14D0E3A1802E1520E3B1861
:107D0A0001E1C6D1320E3A1802E1530E3B1801E1E5
:107D1A00BCD1450E3A1802E1530E3B1801E1B2D12B
:107D2A00430E3A1802E1510E3B1801E1A8D14B0E5D
:107D3A003A1802E1430E3B1801E19ED14C0E3A1863
:107D4A0002E1420E3B1801E194D1440E3A1802E1D5
:107D5A004E0E3B1801E18AD1490E3A1802E14E0E45
:107D6A003B1801E180D1420E3A1802E1510E3B184C
:107D7A0001E176D14C0E3A1802E1510E3B1801E1AD
:107D8A006CD14C0E3A1802E1530E3B1801E162D154
:107D9A004E0E3A1802E1510E3B1801E158D14E0E2F
:107DAA003A1802E1530E3B1801E14ED1430E3A183C
:107DBA0002E1530E3B1801E144D14D0E3A1802E19B
:107DCA00450E3B1801E13AD1500E3A1802E1510E24
:107DDA003B1801E130D1500E3A1802E1540E3B181B
:107DEA0001E126D1500E3A1802E1530E3B1801E187
:107DFA001CD14D0E3A1802E1410E3B1801E112D195
:107E0A004D0E3A1802E1530E3B1801E108D1470E14
:107E1A003A1802E1500E3B1801E1FED0430E3A181F
:107E2A0002E1500E3B1801E1F4D0490E3A1802E182
:107E3A00430E3B1801E1EAD0490E3A1802E1520E0C
:107E4A003B1801E1E0D0490E3A1802E1530E3B1803
:107E5A0001E1D6D0530E3A1802E1520E3B1801E165
:107E6A00CCD0530E3A1802E1530E3B1801E1C2D0AE
:107E7A00530E3A1802E1420E3B1801E1B8D0430E04
:107E8A003A1802E1420E3B1801E1AED0430E3A180D
:107E9A0002E1520E3B1801E1A4D04F0E3A1802E15A
:107EAA00420E3B1801E19AD0570E3A1802E14D0EE4
:107EBA003B1801E191D0520E3A1802E14D0E3B18DF
:107ECA0001E188D0440E3A1802E1500E3B1801E154
:107EDA007FD04F0E3A1802E1500E3B1801E176D0DE
:107EEA00490E3A1802E1500E3B186EE0580E3A1845
:107EFA0002E1540E3B1865E0540E3A1801E13B507A
:107F0A005EE0410E3A1801E13B5057E0560E3A182E
:107F1A0001E13B5050E0490E3A1801E13B5049E07B
:107F2A004F0E3A1801E13B5042E0550E3A1802E171
:107F3A00430E3B183AE0580E3A1802E1430E3B183A
:107F4A0031E0430E3A1801E13B502AE0520E3A184A
:107F5A0001E13B5023E0580E3A1802E1520E3B1859
:107F6A001AE04D0E3A1802E14C0E3B1811E0030ECE
:107F7A00DB5001E0AAD0020EBDEC4AF0BDEC4AF09B
:107F8A005D0E006EBC0E7CEC4BF001E3ADD0AAD0C6
:107F9A00D0EC2BF0ABD02AEC44F0A8D0CCD8A6D0A9
:107FAA002ED9A4D02CEC44F0A1D0C9D89FD0CBD9DB
:107FBA009DD0FDD99BD018DA99D01BDA97D0F6D884
:107FCA0095D028EC44F092D03BDB90D0A7DB8ED042
:107FDA00A2DA8CD081DA8AD06DDA88D0A2EC44F0A9
:107FEA0085D02EEC44F082D0A0EC44F07FD0A4ECF3
:107FFA0044F07CD0A6EC44F079D0A8EC44F076D0DA
:10800A00AAEC44F073D0ACEC44F070D0AEEC44F07F
:10801A006DD0B0EC44F06AD00FEC45F067D066EC56
:10802A002DF064D01AEC29F061D0A0EC31F05ED0CA
:10803A0081EC31F05BD06EEC31F058D01CEC32F0B0
:10804A0055D053EC28F052D09DEC32F04FD0BDEC15
:10805A0032F04CD0CFEC32F049D0DCEC32F046D0E2
:10806A00EEEC32F043D07FEC32F040D090EC32F0BC
:10807A003DD045EC45F03AD054EC45F037D002EC0F
:10808A0033F034D016EC33F031D03CEC63F02ED020
:10809A00ADEC33F02BD0AEEC33F028D040D926D05B
:1080AA00DEEC30F023D001EC2EF020D091EC34F04D
:1080BA001DD0C5EC34F01AD076EC46F017D0BBECE4
:1080CA0046F014D04DEC45F011D093EC4BF093EC04
:1080DA004BF0350E006EBC0EC9EC49F0036E0B0E68
:1080EA00E15C02E2E16AE552E16E03500701E1EC6C
:1080FA0049F00D080DE0B4510BE1520E006E016A11
:10810A00DF50001803E1DE52DD50011801E0B48FA0
:10811A00DDC7DEF7040EE15C02E2E16AE552E16ED8
:10812A00DBEF49F00701E35105E0A00E006ED40E23
:10813A0036EC4BF0120062EC3BF097EF40F04AEC61
:10814A004BF0DEEC4BF0EAEC49F0020EE3EC4BF0BC
:10815A002BE1DF0412E198EC4BF00AE0010E006E0D
:10816A00016ADB50001808E1020EDB50011804E135
:10817A00010EDBCFE3F701D0B48D020E1CEC4AF0FE
:10818A0012E198EC4BF00AE0010E006E016ADB5036
:10819A00001808E1020EDB50011804E1010EDBCFE2
:1081AA00BFFE01D0B48DBEDF52EF4BF0D5EC49F0E3
:1081BA00B1EC4AF0E66AA80EE66E070EE66E0DEC22
:1081CA004CF01BE1020EDB500CE1A851A91103E1AE
:1081DA00AA6BAB6B11D07684A8C7AAF7A9C7ABF76D
:1081EA000BD0A851A91103E1AF6BB06B05D076840F
:1081FA00A8C7AFF7A9C7B0F795DF52EF4BF0F5EC78
:10820A004BF0DEEC4BF022EC4CF0020F22EC4CF07F
:10821A00030F22EC4CF0040F39EC4BF00FE1DF5066
:10822A00926E010EDB50936E020EDB50946E030EBB
:10823A00DB50956E040EDB50966E74DF050EE15C22
:10824A0002E2E16AE552E16EDBEF49F0D5EC49F072
:10825A00FD0EDB50100805E2100EF36EFD0EF3CF93
:10826A00DBFFFC0EDB502BE0FD0EDB50ADEC6AF0C1
:10827A00F3500701BE13F450BF13080EF36EFD0E40
:10828A005EEC4AF00DE2010EF36EFD0EDB5003E0E8
:10829A0004EC4AF0FDE1F350F31C0F0148173DD0FE
:1082AA00FD0EDB500C0839E313EC4BF004E0E84612
:1082BA00FE0B0006FCE1E81C0F0149172ED0FD0E4B
:1082CA00DB50ADEC6AF0F3CF00F0F4CF01F0001E02
:1082DA00011E00500701BE170150BF17080EF36EAA
:1082EA00FD0E5EEC4AF00CE2010EF36EFD0EDB5061
:1082FA0003E004EC4AF0FDE1F3500F0148130DD0FE
:10830A00FD0EDB500C0809E313EC4BF004E0E846E1
:10831A00FE0B0006FCE10F014913DBEF49F0D5EC37
:10832A0049F0DEEC4BF039EC4BF009E1010EDBCF02
:10833A00E6FFDFCFE6FF8ADFE552E552F3DEE552DC
:10834A00E552DBEF49F0D5EC49F0F4EC49F0010EC7
:10835A00D2EC49F047EC4AF026E1010EDB5002E18B
:10836A00DF50896E4DEC4BF01EE1010EDB5002E14D
:10837A00DF508A6E4DEC4BF016E1010EDB5002E144
:10838A00DF508B6E4DEC4BF00EE1010EDB5002E13B
:10839A00DF508C6E4DEC4BF006E1010EDB5002E132
:1083AA00DF508D6EBFDEE552E552DBEF49F08450B7
:1083BA00E66EE66A8350E66EE66A8250E66EE66A22
:1083CA008150E66EE66A8050E66EE66A180E006E26
:1083DA00BC0EC9EC49F0036E0D0EE15C02E2E16AE3
:1083EA00E552E16E03501200A80E006ED40E36EF6D
:1083FA004BF0F5EC4BF0DF6A010EF36EDB6E020E0A
:10840A00DB6A160E006EBC0E36EC4BF09DBCFED736
:10841A00DF6ADFCF00F0100EE76E0018E8AE02D078
:10842A00E73402D0E750005C3EE2010EDB50070160
:10843A00BE150001006E020EDB500701BF150001D8
:10844A00016E005001101EE0DFCFE9FFEA6AE9BEC3
:10845A00EA68A6EC4AF0EECFE6FFEFCFE6FFDFCF01
:10846A0000F0016A00BE0168CFEC4BF00B0E026E01
:10847A00BC0EC1EC4AF0070EE15C02E2E16AE55289
:10848A00E16E0550010EDBCF00F0020EDBCF01F0EA
:10849A00D89000360136010E00C0DBFF020E01C083
:1084AA00DBFFDF2AB6D7A50E006ED40E36EC4BF0F2
:1084BA0052EF4BF04AEC4BF0F4EC49F00DEC4CF077
:1084CA0009E1D8EC4AF005E2F8EC49F0020EDBCFFC
:1084DA00EFFF28DE52EF4BF04AEC4BF0F4EC49F098
:1084EA00030EE3EC4BF015E1D8EC4AF005E2F8ECA8
:1084FA0049F0020EEFCFDBFF020EBDEC4AF0010E8F
:10850A00006EBC0E3DEC4BF002E2E16AE552E16E10
:10851A00035052EF4BF026EC4CF001E08FD0020EE4
:10852A00DB50010801E287D0010EDB50070801E2A7
:10853A0082D0410E1CEC4AF016E1020EDB500AE131
:10854A000DEC4AF003E004EC4AF0FDE1F350F31CB1
:10855A00921673D00DEC4AF003E004EC4AF0FDE108
:10856A00F35092126AD0420E1CEC4AF016E1020E47
:10857A00DB500AE10DEC4AF003E004EC4AF0FDE1BD
:10858A00F350F31C931659D00DEC4AF003E004ECB7
:10859A004AF0FDE1F350931250D0430E1CEC4AF01E
:1085AA0016E1020EDB500AE10DEC4AF003E004EC9E
:1085BA004AF0FDE1F350F31C94163FD00DEC4AF05B
:1085CA0003E004EC4AF0FDE1F350941236D0440E75
:1085DA001CEC4AF016E1020EDB500AE10DEC4AF0FF
:1085EA0003E004EC4AF0FDE1F350F31C951625D0A4
:1085FA000DEC4AF003E004EC4AF0FDE1F350951269
:10860A001CD0450E1CEC4AF016E1020EDB500AE1C2
:10861A000DEC4AF003E004EC4AF0FDE1F350F31CE0
:10862A0096160BD00DEC4AF003E004EC4AF0FDE19B
:10863A00F350961202D0B48D01D074DD52EF4BF094
:10864A00D5EC49F0B1EC4AF01CEC4CF0050E32ECDA
:10865A004BF0010F39EC4BF05FE1010EDB500708DC
:10866A0047E3410E1CEC4AF009E10DEC4AF003E045
:10867A0004EC4AF0FDE1F350801433D0420E1CECB6
:10868A004AF009E10DEC4AF003E004EC4AF0FDE19E
:10869A00F350811426D0430E1CEC4AF009E10DEC8C
:1086AA004AF003E004EC4AF0FDE1F350821419D0D9
:1086BA00440E1CEC4AF009E10DEC4AF003E004EC2C
:1086CA004AF0FDE1F35083140CD0450E1CEC4AF03D
:1086DA000FE10DEC4AF003E004EC4AF0FDE1F3503F
:1086EA008414E76E020EE7CFDBFFDB5008E002D00E
:1086FA00B48D12D0010EF36E020EF3CFDBFF020E21
:10870A00BDEC4AF0F80E006EBB0E3DEC4BF002E2F7
:10871A00E16AE552E16E035052EF4BF026EC4CF061
:10872A0001E08FD0020EDB50010801E287D0010E72
:10873A00DB50070801E282D0410E1CEC4AF016E138
:10874A00020EDB500AE10DEC4AF003E004EC4AF0B9
:10875A00FDE1F350F31C891673D00DEC4AF003E0E7
:10876A0004EC4AF0FDE1F35089126AD0420E1CEC87
:10877A004AF016E1020EDB500AE10DEC4AF003E082
:10878A0004EC4AF0FDE1F350F31C8A1659D00DECC3
:10879A004AF003E004EC4AF0FDE1F3508A1250D0AB
:1087AA00430E1CEC4AF016E1020EDB500AE10DEC16
:1087BA004AF003E004EC4AF0FDE1F350F31C8B1697
:1087CA003FD00DEC4AF003E004EC4AF0FDE1F3502F
:1087DA008B1236D0440E1CEC4AF016E1020EDB5026
:1087EA000AE10DEC4AF003E004EC4AF0FDE1F35033
:1087FA00F31C8C1625D00DEC4AF003E004EC4AF089
:10880A00FDE1F3508C121CD0450E1CEC4AF016E127
:10881A00020EDB500AE10DEC4AF003E004EC4AF0E8
:10882A00FDE1F350F31C8D160BD00DEC4AF003E07A
:10883A0004EC4AF0FDE1F3508D1202D0B48D01D060
:10884A0071DC52EF4BF097EF40F097EF40F097EF63
:10885A0040F04AEC4BF0E652D8EC4BF074EC4BF09B
:10886A0062E1D950020F08EC4AF0720ED880EE5439
:10887A002E0EED543DE3D950020F08EC4AF0EE50AB
:10888A00ED101FE003680468056A2D0EE76E020EFC
:10889A00DBCF06F0030EDBCF07F0E7500626000E0B
:1088AA000722086A0650035C006E07500458016EDE
:1088BA0008500558026E020E00C0DBFF030E01C00D
:1088CA00DBFF010EDB50070813E3410E1CEC4AF0F4
:1088DA0002E1DF6A0FD0420E1CEC4AF002E1080EF8
:1088EA0005D0430E1CEC4AF003E1100EDF6E02D0F5
:1088FA00B48D19D0010EDB50DF24E96EEA6A00EC70
:10890A004BF01AEC4BF0010EDB50DF24B7EC4AF0C7
:10891A00EF0407E1010EDB50DF24B7EC4AF0020E48
:10892A00EF6E97EC40F0040EE15C02E2E16AE55278
:10893A00E16EDBEF49F097EF40F097EF40F097EFE9
:10894A0040F097EF40F097EF40F097EF40F097EF45
:10895A0040F097EF40F0D5EC49F0070EE12402E32E
:10896A00E168E652E16E1CEC4CF0030E32EC4BF07F
:10897A0074EC4BF047E1DECF01F6DDCF02F6020ED2
:10898A00DBCF09F6030EDBCF0AF6040EDB6A030E11
:10899A00F36E040E5EEC4AF033E2010E29EC4AF063
:1089AA00030ED2EC49F0E76E050EE7CFDBFF010EAE
:1089BA00E66ED95018EC4CF0D2EC49F0E76E060E90
:1089CA00E7CFDBFF0701B4511DE1050EDB5018E1CB
:1089DA00060EDB5015E106EC4BF0010EE926060EF9
:1089EA00EA22DECFEEFFDDCFEDFF06EC4BF0090EFB
:1089FA00E926060EEA221AEC4BF0040EDB2AC7D748
:108A0A0097EC40F0070EE15C02E2E16AE552E16EA2
:108A1A00DBEF49F04AEC4BF01CEC4CF0010EE3ECB6
:108A2A004BF00DE1DF5007E0F00E9314936E060150
:108A3A00010E006F02D00601006B97EC40F0E55280
:108A4A00DBEF49F0D9CFE6FFDACFE6FFE1CFD9FF76
:108A5A00E2CFDAFFE652DF6AFF0EDF5C0AE2E8687D
:108A6A00E85005E0E80600D000D000D0F9D7DF2AA8
:108A7A00F3D7E552E552E5CFDAFFE7CFD9FF120087
:108A8A00F29EF29C6592656ADDDF0FEF00F012003C
:108A9A00F29EF29C6592656AD5DFFF001200D5EC62
:108AAA0049F0100EE12402E3E168E652E16EE66A5B
:108ABA00D950010FEAEC49F0E66A9EEC4BF01CEC47
:108ACA004CF0010E32EC4BF0040FEAEC49F0020EC6
:108ADA0032EC4BF018EC4CF032EC4BF00A0FEAECAB
:108AEA0049F0060E32EC4BF0060FEAEC49F0070E9D
:108AFA0032EC4BF00E0FEAEC49F0040E32EC4BF07C
:108B0A000F0FEAEC49F0050ED2EC49F0010EDBCF6B
:108B1A0000F0016A00BE0168CFEC4BF0EC0E026E69
:108B2A00BB0EC1EC4AF0050EE15C02E2E16AE552D5
:108B3A00E16E0550DFCFE6FFE66AE00E006EBB0E7F
:108B4A003DEC4BF002E2E16AE552E16E0350040E9D
:108B5A00DBCFE6FF050EDBCFE6FFD40E006EBB0EC1
:108B6A003DEC4BF002E2E16AE552E16E0350020E7F
:108B7A00DBCFE6FF030EDBCFE6FFC80E006EBB0EAF
:108B8A003DEC4BF002E2E16AE552E16E0350D95046
:108B9A000A0F08EC4AF0E1EC4AF0BB0E006EBB0E7D
:108BAA007CEC4BF002E2E16AE552E16E0350D950E7
:108BBA00060F08EC4AF0E1EC4AF0AE0E006EBB0E6E
:108BCA007CEC4BF002E2E16AE552E16E03500E0ED4
:108BDA00BDEC4AF0A20E006EBB0E3DEC4BF002E279
:108BEA00E16AE552E16E03500F0EBDEC4AF0960EB3
:108BFA00006EBB0E3DEC4BF002E2E16AE552E16E1B
:108C0A00035097EC40F0100EE15C02E2E16AE55293
:108C1A00E16ECCD3C5DB120EE12402E3E168E65231
:108C2A00E16E110EDB6AF36EDBCFF4FFE850F45C01
:108C3A0003E259EC4BF0F7D786EC4BF002E2E16A1B
:108C4A00E552E16E0050110EDB6A100EF36E110E42
:108C5A005EEC4AF02DE281EC4BF0EF50006E016AB7
:108C6A00013404E200508008000E015421E381EC33
:108C7A004BF0EFCF04F0200E045C1AE381EC4BF0CA
:108C8A00EF50E66E180E0201016AFA25006EFB51DA
:108C9A0087EC4AF0DB50D924B6DBEF50E66E020EC1
:108CAA00016AFC25006EFD5187EC4AF0DB2ACDD71C
:108CBA00110EDB50E824180FFAC2E9FFFBC2EAFFE3
:108CCA00EF6E110EDB50E824020FFCC2E9FFFDC271
:108CDA00EAFFEF6E120EE15C02E2E16AE552E16E32
:108CEA0065D35EDB130EE12402E3E168E652E16E2E
:108CFA00110EDB6A120EDB6A110EF36E120ED9DB4D
:108D0A0008E228EC4BF0120E12EC4CF0120EDB2AA1
:108D1A00F3D7100E99DB6CD8F9EC4BF0E76E110E15
:108D2A00E7CFDBFFE668FB0EE66EE66AA3EC4BF0E4
:108D3A00B3EC67F0006E080EE15C02E2E16AE5520C
:108D4A00E16E00506FDB69EC64F0006E080EE15CC6
:108D5A0002E2E16AE552E16E005097EC40F0130E30
:108D6A00E15C02E2E16AE552E16E20D319DB120E00
:108D7A00E12402E3E168E652E16E110EDB6AF36E6A
:108D8A00DBCFF4FFE850F45C03E259EC4BF0F7D781
:108D9A0086EC4BF002E2E16AE552E16E0050DF50E8
:108DAA00006E016AD890015004E6800E005C000E45
:108DBA00015803E2200EDF5C06E2480E006EBD0E8B
:108DCA0036EC4BF00CD045EC4BF0910E006EBB0E1E
:108DDA003DEC4BF002E2E16AE552E16E035097EC9A
:108DEA0040F0120EE15C02E2E16AE552E16EDED287
:108DFA004AEC4BF0DF6A4DDBEF6AAAEC4BF002E17A
:108E0A00B4890CD0D9DA2C080BE0E7EC4BF002E27B
:108E1A00E16AE552E16E03500701B48B000E28D0D7
:108E2A00E7DA04E1010E011801E1DE6B0D0ED4EC64
:108E3A004BF009E02C0E016EBFDA015C04E0FB0E78
:108E4A00DB50DF5C02E3DF5013D0B6DAE66E21DBDB
:108E5A00E552E750EF6ECCDA04E1010E011801E1A8
:108E6A00DE6BDF2AFC0EDB2AFD0EE0E3DB2ADED70F
:108E7A00E5529CD295DA090EE12402E3E168E65252
:108E8A00E16E080EDB6AAAEC4BF005E1FA0EDB5044
:108E9A0021E1B4891FD090DA2C080EE0FA0EDB50DB
:108EAA0009E1E7EC4BF002E2E16AE552E16E0350B8
:108EBA000701B48B020E25D19BDA04E1010E0118D9
:108ECA0001E1DE6B0D0ED4EC4BF006E1FA0EDB503D
:108EDA0001E1B489030E15D12D0ED4EC4BF020E13B
:108EEA00040E5CDB1DE0050E026EFD0EDB50025C1B
:108EFA0017E0FD0EDB0401E1CAD0030E28DB01E115
:108F0A00C6D0070E4BDB01E1C2D0010EF36E080E8C
:108F1A00F3CFDBFF6DDA04E1010E011801E1DE6B2C
:108F2A00040E15DB09E0050E39DB06E00A0E8CDAC1
:108F3A00F1D8F9EC4BF036D0DE51BCDBEFCF00F0C4
:108F4A00000E00C0DFFF010EDB6A020EDB6A030EB1
:108F5A00DB6A050EFCDA1FE1000EDFCFE6FF010E29
:108F6A00DBCFE6FF06EC6AF0E552E552F3CF00F0FC
:108F7A00F4CF01F0026A036A01AE02D00268036804
:108F8A0000C0DFFF010E01C0DBFF020E02C0DBFFE3
:108F9A00030E03C0DBFF07012BDA04E1010E0118FF
:108FAA0001E1DE6B080EDB5044E0FD0EDB5007E109
:108FBA001FEC4CF0800E4BDA000EEE5414E3020E56
:108FCA00C6DA07E11FEC4CF0000EEE54800E3FDAD1
:108FDA000AE3060EE3DA09E11FEC4CF0000E37DA79
:108FEA00800EEE5402E2070152D0F4D99DDA080E3F
:108FFA00DB5055E0040EDBCF38F0050EDBCF39F03D
:10900A00060EDBCF3AF0070EDBCF3BF03D683E6839
:10901A003F684068A2EC69F0040E34C0DBFF050E1D
:10902A0035C0DBFF060E36C0DBFF070E37C0DBFF9D
:10903A0036D0FD0EDB5007E11FEC4CF07F0EEE54EC
:10904A00000E05DA23E3FD0EDB0404E139DB000E32
:10905A00FED91CE3020E7BDA04E132DB7F0EF7D97C
:10906A0015E3030E9BDA04E12BDBFF0EF0D90EE3C6
:10907A00060E026EFD0EDB50025C0CE121DBFF0ED8
:10908A00EE54FF0EEE547F0EEE5404E20701B48D47
:10909A00010E37D0070E5BDA02E09CD945DAFD0EE5
:1090AA00DB50070A21E0010A17E0050A11E0010A6C
:1090BA000FE0030A08E0050A06E0010A04E0050ACF
:1090CA0002E0040E1ED002DA040EDBCFEFFF18D046
:1090DA0042DBDBCFEDFF14D03EDBDBCFEEFF060E2B
:1090EA00DBCFEEFF070E0AD0F1D9DFCFEEFF010E7C
:1090FA00DBCFEEFF020EDBCFEEFF030EDBCFEEFF80
:10910A00000E006E090EE15C02E2E16AE552E16ED0
:10911A0000504CD1BADAE652BCD9EE6AEE6AEE6A6F
:10912A00EE6A010EDB6AFB0EDB50F36E010EC1D94B
:10913A004FE20701DE51BEDAEFCFDFFF300EDF5C10
:10914A0042E3DF5039083FE3A4D9EECF00F0EECF77
:10915A0001F0EECF02F0EFCF03F00A0E3D6E3E6A49
:10916A003F6A406A00C038F001C039F002C03AF0E4
:10917A0003C03BF0A2EC69F034C000F035C001F046
:10918A0036C002F037C003F0300EDF5C046E056AA9
:10919A00066A076AE8500026055001220650022294
:1091AA000750032276D900C0EEFF01C0EEFF02C0CD
:1091BA00EEFF03C0EEFF07011BD907E1010E0118FC
:1091CA0004E1DE6B02D0000E04D0010EDB2AABD71D
:1091DA00010EE552E552EAD00701AE51E66EE66AA3
:1091EA005E0E006EBB0E44DA02E2E16AE552E16EFF
:1091FA00035012000401785108E0010E006E655018
:10920A00020B01E0010E005C17E1E5D90BE16151A7
:10921A00621111E18C86A00E616F0F0E626F010E52
:10922A00636F12006151621152E18C96A00E616F58
:10923A000F0E626F636B1200780509E0020E785D0B
:10924A0006E0040E785D03E0100E785D17E1C3D9DD
:10925A000BE16151621111E18C86200E616F4E0E95
:10926A00626F010E636F12006151621130E18C96D8
:10927A00200E616F4E0E626F636B1200200E785DD6
:10928A0026E1A9D907E16151621121E18C86E0D971
:10929A00010E15D0630507E16151621118E18C9640
:1092AA00D7D9020E0CD0020E635D0BE16151621137
:1092BA000EE18C86A00E616F860E626F030E636FDD
:1092CA0012006151621103E18C96C2D9636B1200DC
:1092DA0067D8B2D9E8AE02D0003403D0E750D880BC
:1092EA00005423E3FC0EDB5010E0E8D8E9BEEA683C
:1092FA00A2D804E0E846FE0B0106FCE1006EDED8C7
:10930A00E9BEEA6875DAEF1210D0D8D8E9BEEA6881
:10931A0092D804E0E846FE0B0106FCE1E81C006E68
:10932A00CDD8E9BEEA6864DAEF1640D039D884D9D4
:10933A00E8AE02D0003403D0E750D880005423E3CB
:10934A00FC0EDB5011E1BAD8E9BEEA6874D804E031
:10935A00E846FE0B0106FCE1E81C006EAFD8E9BE48
:10936A00EA684CDAEF160FD0A9D8E9BEEA6863D8E2
:10937A0004E0E846FE0B0106FCE1006E9FD8E9BE58
:10938A00EA683CDAEF1212D0016E026A00C0E6FF08
:10939A00E66E02C0E6FFCBEF68F0E66E9EEF4BF09A
:1093AA006FD9E1CFD9FFE2CFDAFF1200E552E5CF5C
:1093BA00DAFFE7CFD9FF1200DE517CD9EF50120055
:1093CA00A951E96EEA6A69EF4BF0E66E000EDA20FF
:1093DA00E66E1200D9CFE9FFDACFEAFF1200E652B1
:1093EA00E6521CEF4CF0DECFE9FFDDCFEAFF1200B8
:1093FA00DE2BDE51006E016A000E00181200D890B2
:10940A00F336E8061200E96E000EDA20EA6E120060
:10941A00010EF36EDB501200EA22EECF48F0EFCFD6
:10942A0049F012002DD9100EE66EA3EF4BF0006E34
:10943A00DF50005C1200C80EE926060EEA22EF5041
:10944A00016E010E01521200E66E45EF4BF0EE542A
:10945A00000EEE54000EEE541200DF6EDFCFE6FF70
:10946A00DC51016A000F006E020E012293D99FECB3
:10947A0061F0F9EF4BF0DECF00F0DDCF01F0D890CC
:10948A0001501200E76E010EE7CFDBFF0701B4516E
:10949A001200FC0EDBCFE9FFFD0EDBCFEAFF120064
:1094AA00EA22EECF4AF0EFCF4BF012000DD9E806D0
:1094BA001200DBCFF4FFF350F45C1200FD0EDBCF99
:1094CA00E9FFEA6A1200DD515FEF4BF0FB0EDBCFDA
:1094DA00E9FFFC0EDBCFEAFF1200EA22EE50EFCFE3
:1094EA00EAFFE96E00501200A951EA6A310FE96EEB
:1094FA000E0EEA22EF500E01EA6AAC25E96EAD5172
:10950A00EA2212000122110EDB50E8240024E96E3F
:10951A00000E0120EA6EE552E750EF6E110E1200BE
:10952A00036E050EE15C1200040EEECFDBFF050EA2
:10953A00EECFDBFF060EEECFDBFF070EEECFDBFF33
:10954A001200C2D8000EE926010EEA221200006EAD
:10955A00FD0EDB50005C1200E652E652E652020EA5
:10956A00DB6A1200EA6A290FE96E010EEA2212008A
:10957A00DBCFE6FFE66A1200036E046A02C0E6FF6A
:10958A00E66E04C0E6FFCBEC68F0056E1200020E30
:10959A00DBCF48F0030EDBCF49F01200016EFD0E5F
:1095AA00DB50015C1200DECF00F0DDCF01F0000ECF
:1095BA00005C100E01581200EECFE6FFEECFE6FF78
:1095CA00EECFE6FFEFCFE6FF1200070EB715486EA3
:1095DA00010E4852120006016107000E625B6351D8
:1095EA001200000EE926030EEA221200010EDBCF5A
:1095FA00E9FFEA6A120068D8410EE926010EEA225A
:10960A001200040EDB28E96EEA6A69EF4BF0E66E97
:10961A00E66A06EC6AF0E552E5521200FD0EDB50EE
:10962A00F80F006E010E00521200020EDBCFEEFFA1
:10963A00030EDBCFEDFF1200FD0EDBCF00F0190E9B
:10964A00E76E00181200D9CF00F0DACF01F012004D
:10965A00100E616F270E626F12009FDEE66AD95004
:10966A00120092DEF9EF4BF0B0DE010EE3EF4BF0A1
:10967A008BDE95EF4AF0A4DE010EE9260E0E1200EB
:10968A00D9CFE6FFDACFE6FF12008ADEE6521200F1
:10969A00010EDADE82DE47EF4AF0A6D887D690DEE0
:1096AA00790EE9260E0E1200CEDF110EB6D8110E73
:1096BA00DB2A1200EA6A000FE96E030EEA221200A0
:1096CA00B9D8FF0EEE541200D890E936EA361200E5
:1096DA00110EE926060EA0DE86DE010E1200A3D8C0
:1096EA00E3EF4BF06DDE490EE9260E0E12004CDE5A
:1096FA00036E070EE15C1200110EDB50D92408EF4D
:10970A004AF090DE17EC69F0006E080EE15C120078
:10971A00C7DE48504A5C49504B581200030E28DFF6
:10972A00020EBDEF4AF0D950010F6DDEEE50ED107A
:10973A0012003FEC47F058D8E5521200E66AE66A92
:10974A00F80EE66EE66AE66A12000D0E006E070172
:10975A0033DE005C1200BADE040EDBCFEEFF050E2C
:10976A0012009EDE4A5048181200110EE926060E13
:10977A00EA2212002FDEEE50ED1012002BDE010E4F
:10978A00EE18120027DE020EEE18120023DE030E78
:10979A00EE18120000C0E6FF01C0E6FF1200006EDC
:1097AA000BDE005C12001BDE050E57DF010F22EFF5
:1097BA004CF015DE010E51DF010F1200EEDD07013C
:1097CA00B4511200F9DDE66EE66A6A0E006EBB0E4F
:1097DA003DEF4BF064DF20DE4EDFEA2248501200F4
:1097EA0054DFE652E6521200E552E552E552120003
:1097FA006BDF960EE926060E72EF4AF065DF640EFD
:10980A00E926060E72EF4AF06DDF06DE40EF4BF0F6
:10981A00030E23DF020F39EF4BF0DB500F01D9247F
:10982A00F2DDEF6A1200020FD0DD030E1200E66AC3
:10983A0045EF4BF0CFDDD8801200C7DD010E32EFC5
:10984A004BF023DFB0DF020F39EF4BF0DDEC51F0C4
:10985A00A098636A626A0F01266BA5EC52F002E2D5
:10986A00E16AE552E16E00500F0169EC52F0DF6ADD
:10987A00DF50006E016A0C0E005C000E015810E207
:10988A00DF50040DF3CFE9FFF4CFEAFF000EE9261B
:10989A00040EEA22EE6AEE6AEE6AEE6ADF2AE8D778
:1098AA00658C0F01386B6598659C62A607D0629635
:1098BA0004018F6B946B956B966BF7D70401010EBD
:1098CA00A86FA96FAA6BAB6B9C6BDF6A030EDF5C98
:1098DA0011E2EA6ADF34D2EC52F0EA22EE6AED6A69
:1098EA00EA6ADF34D9EC52F0EA22EE6AED6A1BEC3E
:1098FA0052F0ECD70401080E856F040E866F0F0133
:10990A00160E266F0401300E026F040E036F400E0E
:10991A00016F840E006F0401796B786BE0EF51F0F0
:10992A00DDEC51F082BE06D0656A0F01366B040188
:10993A00786B7CD0040178510CE1656A0F01366BB3
:10994A0069EC52F065B602D06586FCD70401010EB7
:10995A00786F78050AE165BA08D0626A0F01366B3A
:10996A00368136890401020E786F6250040B06E0D4
:10997A000F013651040B02E0629459DB65B256D0EE
:10998A006250010B09E00F013651010B05E05EDF61
:10999A000401040E786F62906250100B06E00F010A
:1099AA003651100B02E033DB629862AC15D00F011E
:1099BA0036AD0AD070EC52F0730EE7EC51F002E2C9
:1099CA00E16AE552E16E0050629C0401A65101E091
:1099DA00A607A65101E1F3D86250200B05E00F015A
:1099EA003651200B01E002DB6250020B14E00F013A
:1099FA003651020B10E070EC52F0E6687F0EE66E0C
:109A0A00A9EC65F0006E060EE15C02E2E16AE5523D
:109A1A00E16E0050636A040E0401E76E7819E8AE3D
:109A2A0002D0E73402D0E750785D02E2A19834D040
:109A3A000F0136A730D0DF6A040EDF5C2CE262A683
:109A4A002AD064CF9DF404019D51780BE842E84284
:109A5A00E8429E6F62969DB504D09E51E0EC52F0AA
:109A6A0003D09E51E5EC52F0EA22EF709E5102E1DA
:109A7A00F0DA0FD0000EE66EE66A9D0EE66E040E70
:109A8A00E66E720EE7EC51F002E2E16AE552E16E2F
:109A9A000050DF2AD1D7A198E0EF51F0CFEC52F075
:109AAA00FC0EDBA403D0E66A59EC52F0FC0EDBA2F2
:109ABA0004D0010EE66E59EC52F0FD0EDB50016A3D
:109ACA00260F006E0F0E53EC52F0EFEC51F0FC0E25
:109ADA00DBCFEFFFE552E0EF51F0CFEC52F0FC0E96
:109AEA00DB5003E0E2EC51F002D00CEC52F03FEC18
:109AFA0052F0D9CFE9FFDACFEAFFEE50ED1003E1D9
:109B0A00F36AF46A28D0EFEC51F0F4EC52F0FA0E52
:109B1A00DBCFEEFFFB0EDBCFEDFFEFEC51F0EE52A9
:109B2A00F90EDBCFEFFF400EEAEC52F0880EF9ECAB
:109B3A0052F0FC0EDB5003E0E2EC51F002D00CECE8
:109B4A0052F0EA22EF74DECF00F0DDCF01F000C060
:109B5A00F3FF01C0F4FFE552E0EF51F0CFEC52F011
:109B6A00FD0EDB5003E1AEEC52F009D011EC52F0DD
:109B7A0083EC52F011EC52F0010F83EC52F0E552F3
:109B8A00E0EF51F0B5EC52F065A817D0C8EC52F0EE
:109B9A00400EEE16EE6AEE6AEE6AC8EC52F0EE7C01
:109BAA00E2EC51F0EA22EF74400E006EC8EC52F07B
:109BBA000050EF16C8EC52F0EF7C9FEF52F0040110
:109BCA00A85127E1010EA86FA95123E1010EA96F3F
:109BDA00020E8C5D09E1F4EC51F0EE52EF6AF4ECFE
:109BEA0051F0C80EEF6E12008C0513E19F6B01EC69
:109BFA0052F0EE52400EEF6E01EC52F08FEC52F042
:109C0A0001EC52F0840EEF6E010E9F6FCDDB800ED9
:109C1A00EF6E12000401AA6BAB6B020E8C5D07E1BA
:109C2A00EEEC52F006EC52F07EEC52F010D090516D
:109C3A000401365D040191510401375904E236C426
:109C4A0090F437C491F45CD8CADBDBDBC8DBC80EFE
:109C5A00EF6E1200CFEC52F0000EDE6E040EDD6ED7
:109C6A00DBDB040DF4CF01F0D9CFE9FFDACFEAFF4D
:109C7A00F350EE260150ED22ADDBEF9EFC0EDB50D9
:109C8A0002E1C5DB01D099DBEA22DECFEEFFDDCFB0
:109C9A00EDFFA0DBEF9C9EDB040EE926000EEA2214
:109CAA00EF8CE55288D3659804018FBF0DD094AF2D
:109CBA0009D0020E8C6FAB5101E1ACDF0401A96B34
:109CCA00A86B1200AEEF52F0040130AF0DD00401C0
:109CDA00010E8C6FAA5101E19DDF0401A96BA86BEB
:109CEA00A7510DE1E4EF4DF00401020E8C6F5CDB2D
:109CFA00840EEF6EA96BA86BA75101E160DF120019
:109D0A0057DB400EDF6E0401905D000E91590AE2A6
:109D1A0090C4DFFF8B5102E1010E03D08B0502E1F3
:109D2A00020E8B6FDF50016AE850905D906F015010
:109D3A009159916F54DBEE52DFCFEFFF380E996FD6
:109D4A00040E9A6F8FB10DD0DF5017E08DC4F6FF65
:109D5A008EC4F7FF8D2B000E8E230800F5507DDB95
:109D6A00F3D7DF500AE08DC4E9FF8EC4EAFF8D2BDA
:109D7A00000E8E23EF5071DBF4D71DD3CFEC52F0D7
:109D8A003BDBEE52EFCFDFFFDFCF00F000500401E4
:109D9A00955D000E965902E295C4DFFFDF50006E12
:109DAA00016AE850955D956F01509659966F010EBC
:109DBA00DB6ADF50F36E010EDBCFF4FFF350F45C85
:109DCA0016E2010EDB50EA6A380FE96E040EEA2247
:109DDA00EF50E66E92C4E9FF93C4EAFF922B000E9D
:109DEA009323E552E750EF6E010EDB2AE2D7000E0D
:109DFA00D8809555000E96550DE2EBDB02DBFCDAB6
:109E0A00EF50400B03E175DBC80E02D072DB880EFF
:109E1A00EF6E12D0C9DA840EEF6E9751981107E0EF
:109E2A0005D098C4FAFF04019751F96EFADF0401CC
:109E3A00949FA75101E1C3DEE552BDD2B9DA04010C
:109E4A008F8F7EDB02E2E16AE552E16E0050300E4E
:109E5A00E66EE66AE66A000EE66E040EF1DA02E2E1
:109E6A00E16AE552E16E0050658CDF6A030EDF5C41
:109E7A0002E2DCDAFBD7010EE66EE66AE66A7A0EE1
:109E8A00E66E040EDDDA02E2E16AE552E16E0050A6
:109E9A00659C0401080E856F040E866F000E7B6FA9
:109EAA00040E7C6F7BC47DF47E6F32C479F47951E1
:109EBA0002E1100E10D0010EE66EE66A790EE66E29
:109ECA00040EE66E010E7EDA02E2E16AE552E16E06
:109EDA0000500401200E786F6ED2800E0401305DAE
:109EEA004EE10401C00E8F6F04013351030A25E0CD
:109EFA00010A09E0030A41E10401B40E8D6FD30E91
:109F0A008E6F120E34D03251F66EF76AD890F6364A
:109F1A00F736090EF626D40EF7220900F5CF8DF48E
:109F2A000A00F5CF8EF4020E0401DCDAF5CF90F4C4
:109F3A00030ED8DAF5CF91F41200040E325D1AE25C
:109F4A0004018F8104013251E96EEA6AD890E93638
:109F5A00EA36F60EE926020EEA22EECF8DF4EDCFAE
:109F6A008EF48DC4E9FF8EC4EAFFEF500401906FAE
:109F7A00916B120004018F6B120004018F6B1200A7
:109F8A0009DB0401386B396B30511F0B020A11E0EF
:109F9A00030A0CE0010A1EE104018F8F04013881D3
:109FAA0004019B0517E10401388314D004018F8F43
:109FBA0011D004018F8F040134BF02D0DADA01D044
:109FCA00DDDA58DAE3DA06E005DAEF50040B02E0EC
:109FDA00010E386F04018FAF07D0380E8D6F040E53
:109FEA008E6F8F81020E906FE552E5D10F0126A187
:109FFA000CD002DAEF50800807E1F1D9EF5084085B
:10A00A0003E1FAD98C0EEF6E2691629A12000F01C3
:10A01A003685629865820401010E9C6F31DA750EED
:10A02A00D1D902E2E16AE552E16E00501200040160
:10A03A009C6B26DA740EC6D902E2E16AE552E16E39
:10A04A00005065920F01369562A402D06294FCD743
:10A05A001200AED904012D0EA66FFD0E9D1539E131
:10A06A007E0E9D15E8407F0B040DF3CF7BF4F4CFF1
:10A07A007CF4000E7B27040E7C237BC47DF47CC415
:10A08A007EF47D75B9D9EF503C0BE842E8420D08E1
:10A09A001EE1DF6A080EDF5C16E2AED9020EE9267F
:10A0AA00000ED5D9EF50E66EDF50EA6A300FE96E3E
:10A0BA00040EEA22E552E750EF6E9ED990DAEE2AB4
:10A0CA00EF22DF2AE7D798D925DA09D807D027D887
:10A0DA0005D0FD0E9D15040801E130D86CD10401AC
:10A0EA008B6BA76BAA6BAB6B9F6B8C6B78D9EF9E54
:10A0FA00857575D9EF9E8575FCD9EF9E8F6B906B30
:10A10A00916B946B956B966B55D8BAD9030E5AD945
:10A11A0002E2E16AE552E16E005058EF4EF0020E9B
:10A12A0004018C5D02E1C3EF4EF08C6B9F5104E198
:10A13A003BD98C0EEF6E12009F6B120039D94FD9A2
:10A14A00EF50400B01E0010EDF6E04018575080E29
:10A15A00785D0BE132C438FF0F01385103E0040186
:10A16A00100E02D00401040E786F8C0513E137D962
:10A17A0048D9C6DD020E04018B5D03E130D9840E95
:10A18A0007D0DF5003E12BD9C80E02D028D9880E98
:10A19A00EF6E0FD094AF0CD09751981107E005D00D
:10A1AA0098C4FAFF04019751F96EFADF0401949FEB
:10A1BA008C6B01D104013051600BE842E842E8425D
:10A1CA00E842E842000901E0120031510C0A4AE073
:10A1DA000B0A3FE00C0A31E0010A22E00B0A1EE0FA
:10A1EA00020A1CE0030A18E0080A10E0010A0CE05F
:10A1FA000F0A08E0030A01E0120004018F8F080E1B
:10A20A00786F120072EF4FF023EF4FF00401790ECE
:10A21A008D6F040E8E6F0CD0C5EF4FF038EF51F0F2
:10A22A00345104018D6F8E6B7A0E8D27040E8E23A6
:10A23A008F81010E906F8F8F120004018F8F04019E
:10A24A003451EA6A7A0FE96E040EEA2232C4EFFF49
:10A25A00120016D9020EB6D802E2E16AE552E16EA0
:10A26A0000501200120096D9E652E652E652040154
:10A27A00320510E130511F0B00090CE104018F8FE8
:10A28A00030E0401315D04E10401010E9B6F02D04B
:10A29A0004019B6B0401325101E07FD030511F0B46
:10A2AA00020801E07AD034510F0B000901E175D0A0
:10A2BA0034510F0B020871E3200E0401785D6DE141
:10A2CA008F8F040134BF04D054D9D4D8DFD803D037
:10A2DA0055D9D0D8DFD8EA22020EEFCFDBFFECD86F
:10A2EA00010B02E1DF9401D0DF8434BF02D041D9EF
:10A2FA0001D044D9EA22DECFEEFFDDCFEDFF030E17
:10A30A00315D0CE143D907E034BF02D0BFD801D098
:10A31A00C1D8EA22EF82840E67D93FD0DF7436D9DA
:10A32A000BE058D8EF9E56D8EF8CFAD802E2E16AD1
:10A33A00E552E16E005002D04DD8EF8CDF74BCD8E4
:10A34A00020B02E123D912E0040134BF02D09ED8E5
:10A35A0001D0A0D8EA22EF923B0E006E36D9E0D89F
:10A36A0002E2E16AE552E16E005002D03B0E2DD9BD
:10A37A00040134510F0B016A260F006E0F0E0122E1
:10A38A00030E00C0DBFF040E01C0DBFF030EDBCFB0
:10A39A00E9FF040EDBCFEAFFEF90050EE15C02E273
:10A3AA00E16AE552E16EC6D014D9B4D87EEF52F014
:10A3BA00D7D8E6521200E552BDD0FD0EEA6ADB3468
:10A3CA00D2EF52F0E66EE66AA9EC65F0006E060E70
:10A3DA00E15C1200DECFE9FFDDCFEAFF120085C49F
:10A3EA00E9FF86C4EAFF120034510F0BE96EEA6AEC
:10A3FA00D890E936EA3612007BC4E9FF7CC4EAFF4A
:10A40A001200EDD8380EEE6E040EED6E1200FD0E3F
:10A41A00EA6ADB34D9EF52F0FC0EDB50E824026E14
:10A42A00FD0EDB50040DF35002241200DF50C8D891
:10A43A00EA22EF6ADF50BFD8EA22EF6ADF2A120067
:10A44A00E66E7EEC68F0006E050EE15C1200EA2210
:10A45A00EE50EFCFEAFFE96E1200E66E99C4E9FF0B
:10A46A009AC4EAFF992B000E9A23E552E750EF6E41
:10A47A00DF061200EA22EECFDEFFEDCFDDFF12008B
:10A48A00000EE66EE66AE66EE66A120034510F0BBB
:10A49A00E0EF52F034510F0BE5EF52F0012200C009
:10A4AA00DEFF01C0DDFF1200FD0EDBCFE6FF2FEC61
:10A4BA004EF0E552E5521200D950020FE96E000E35
:10A4CA00DA20EA6EEF501200160E396F9F0E376FC0
:10A4DA007B0E366F1200010EE66EE66A000EE66E1D
:10A4EA00E66A1200F76A8D25F66E8E51F722080089
:10A4FA0012007DC4E9FF7EC4EAFF1200040DF3CF07
:10A50A0000F0F4CF01F0000E0026040EC7DF840E1F
:10A51A00F9EF52F064D8300EEE6E040EED6E1200B2
:10A52A00020EE66EE66ADECFE6FFDDCFE6FF050E37
:10A53A00E7EF51F0E552E5CFDAFFE7CFD9FF120096
:10A54A00020EE66EE66AE66A270EE66E0F0E25EF43
:10A55A0052F02ADF8C0EEF6E42DF840EEF6E12008D
:10A56A00D9CFE6FFDACFE6FFE1CFD9FFE2CFDAFFB4
:10A57A0012003ADF7F0EE926040E120035DF850E3F
:10A58A00E926040E120019DF2CEF52F023DFEF50F8
:10A59A00800B12000DDFE6521200FE0BEA36E96E5E
:10A5AA00850EE926040E1200FE0BEA36E96E7F0ECE
:10A5BA00E926040E1200EA6AA30FE96E040E1200DD
:10A5CA00EA6AA00FE96E040E120004DFE850EF16E3
:10A5DA0012008FDFEE52400EEF6E7EEF52F0020E47
:10A5EA00E926000EEA221200F5DEE850EF12120008
:10A5FA0039EC58F0FB0EDBCFF3FFDB06F350000912
:10A60A000AE087EC58F0FA0EF2EC58F0F3E1011C7C
:10A61A00F1E1010E01D0000E68EF58F039EC58F064
:10A62A003B0EE12402E3E168E652E16E010EDB6AC9
:10A63A00020EDB6AF90EDBCFF6FFFA0EDBCFF7FF6D
:10A64A00FB0EDBCFF8FF0800F550DF6EDF5002E1AA
:10A65A008CEF57F0250EDF5C02E07FEF57F0030E18
:10A66A00DB6A040EDB6A050EDB6A060EDB6A070E7E
:10A67A00DB6AA1EC57F02D0EDF5C0CE02B0EDF5CE1
:10A68A0009E0200EDF5C06E0230EDF5C03E0300EFB
:10A69A00DF5C1AE1DF50300A14E0130A0FE0030A04
:10A6AA000AE00B0A05E0060AE4E1030EDB80E1D7C3
:10A6BA00030EDB82DED7030EDB84DBD7030EDB86D9
:10A6CA00D8D7030EDB88D5D72A0EDF5C1BE19DECB9
:10A6DA0057F0EBEC57F010E0030EDB803A683B686A
:10A6EA00130EDBCF3FF0140EDBCF40F0D6EC5BF05D
:10A6FA00040E38C0DBFF03D0130ED4EC57F0A1ECE4
:10A70A0057F00BD0090EDB6A42EC58F003E0B6ECC6
:10A71A0058F0FAD7090ED4EC57F0030EDBB0DB98E9
:10A72A002E0EDF5C1BE1A1EC57F02A0EDF5C0BE179
:10A73A009DEC57F0EBEC57F003E1130E26EC58F0C2
:10A74A00A1EC57F00BD0090EDB6A42EC58F003E09B
:10A75A00B6EC58F0FAD7090E26EC58F0680EDF5C12
:10A76A0007E1A1EC57F0680EDF5C1DE1030E18D07B
:10A77A00740EDF5C17E07A0EDF5C14E0480EDF5CD3
:10A78A0006E0540EDF5C03E05A0EDF5C02E1020EC3
:10A79A0007D06C0EDF5C03E06A0EDF5C04E1010E99
:10A7AA0079EC58F0C9DBDF506E0A01E17FD31E0A4B
:10A7BA0001E192D1200A01E18FD13F0A01E149D199
:10A7CA001A0A01E146D10D0A01E143D1200A01E149
:10A7DA0040D13A0A01E13DD1200A01E13AD1260AE3
:10A7EA0001E135D10D0A01E132D11A0A01E1D9D0CC
:10A7FA00200A4AE0300A1FE0460A0EE0250A01E074
:10A80A0083D3D950F90FE96EFF0EDA20EA6E010EF2
:10A81A00EE5E000EEE5AEE5A87EC58F0250EE66E02
:10A82A0095DB03E1011C01E169D383EC58F001E2F5
:10A83A006BD3DB2A69D3080EDB6A040EDB500108EE
:10A84A0006E2040EDB044BEC58F0DB508BDB080EFF
:10A85A00DB5009E0030EDB50010B05E172DB01E07E
:10A86A004DD3080EDB6A64DBEFCFDFFFFBEC58F059
:10A87A0003E1011C01E142D383EC58F001E3DB2A36
:10A88A0060DB01E141D33AD3070EDB5002080FE146
:10A89A00C7EC58F0030E8EEC58F00E0EEECFDBFF2D
:10A8AA000F0EEECFDBFF100EEECFDBFF20D0F70E40
:10A8BA00DBCF03F0F80EDBCF04F0020E035E000ECE
:10A8CA00045AF70E03C0DBFFF80E04C0DBFF03C017
:10A8DA00E9FF04C0EAFF7EEC58F0026A0E0E00C0DF
:10A8EA00DBFF0F0E01C0DBFF100E02C0DBFF0E0EF6
:10A8FA00DBCFE6FF0F0EDBCFE6FF100EDBCFE6FF66
:10A90A00A6EC68F0E552E552E552130E39C0DBFFBA
:10A91A00140E3AC0DBFF060EDB5005E0130EC2EC44
:10A92A0058F001E26ADBE6EC58F002E2130E37DB7C
:10A93A00A9EC58F006E0040EC2EC58F002E2050E4B
:10A94A002EDB030EDBB005D0FCDA01E0D7D2080E0D
:10A95A00DB6A090EDB6A0E0EDBCFF6FF0F0EDBCFCA
:10A96A00F7FF100EDBCFF8FF0800F550DF6EDF505F
:10A97A0014E0ECEC58F011E2FBEC58F003E1011C96
:10A98A0001E1BCD2BBDB01E3DB2A090EDB2AD95089
:10A99A000E0FE96E000ECBDBE7D7D3DA01E1B4D2B2
:10A9AA00ADD2C6DA110EEECFDBFF120EEDCFDBFF12
:10A9BA00110EDBCFE6FF120EDBCFE6FF98EC68F054
:10A9CA00E552E552130EF3CFDBFF140EF4CFDBFF93
:10A9DA00060EDB5004E0130ED0DB01E20EDBE6ECE0
:10A9EA0058F002E2130EDBDAAFDB05E0040EC5DB3A
:10A9FA0002E2050ED4DA030EDBB005D0A2DA01E0DA
:10AA0A007DD2080EDB6A090EDB6A110EDBCFE9FF85
:10AA1A00120EDBCFEAFFEFCFDFFFDF5014E0D7DB08
:10AA2A0012E2E4DB03E1011C01E168D267DB01E326
:10AA3A00DB2A090EDB2A110EDB2ADBCFE9FF120E15
:10AA4A00E8E3DB2AE6D77DDA01E15ED257D2030ECC
:10AA5A00DB8E070EDB0410E195DB040E5ADB0A0ECF
:10AA6A00EECFDBFF0B0EEECFDBFF0C0EEECFDBFFE4
:10AA7A000D0EEECFDBFF6CD0070EDB5003082CE186
:10AA8A00030EDBAE0DD0B2DA020E76DAEFCF00F0AB
:10AA9A00016A026A036A00AE39D00168026835D0D9
:10AAAA00F70EDBCF01F0F80EDBCF02F0020E015EEB
:10AABA00000E025AF70E01C0DBFFF80E02C0DBFFE0
:10AACA0001C0E9FF02C0EAFFEFCF00F00A0E00C0A2
:10AADA00DBFF0B0EDB6A38D0070EDB50020809E1F8
:10AAEA00030EDBAE04D059DB02AE10D00ED055DB1C
:10AAFA000DD0030EDBAE12D079DA020E3DDAF9DAA6
:10AB0A00026A036A01AE02D002680368E2DA0C0E36
:10AB1A0002C0DBFF0D0E03C0DBFF1AD0F70EDBCF3E
:10AB2A0002F0F80EDBCF03F0020E025E000E035AAB
:10AB3A00F70E02C0DBFFF80E03C0DBFF02C0E9FF1D
:10AB4A0003C0EAFFD6DAC5DA0C0EDB6A0D0EDB6A41
:10AB5A00060EDB5005E1010EF36E050EF3CFDBFFA7
:10AB6A00150EDB6A160EDB6AD950370F006E000E1F
:10AB7A00DA20016E390E00C0DBFF3A0E01C0DBFF9E
:10AB8A00380EDB6A080EDB6A0A0EAEDADF50780A84
:10AB9A0012E0200A10E0280A0CE0200A0AE03F0A24
:10ABAA0006E00D0A02E0200A08E1020E05D0080EAE
:10ABBA0003D0080EDF26100E97DA030EDBBE02D092
:10ABCA00DB92DB94DB50800B24E08ADAD890030E08
:10ABDA00EB50000A08E6000EEE5C000EEE58000E7E
:10ABEA00EE58000EEE5815E213DA3D683E683F68EB
:10ABFA004068A2EC69F00A0E34C0DBFF0B0E35C0C8
:10AC0A00DBFF0C0E36C0DBFF0D0E37C0DBFF2D0E4F
:10AC1A0008D0030EDBA202D02B0E03D0DBA408D08F
:10AC2A00200EF36E170EF3CFDBFF150EDB2A02D0D0
:10AC3A00170EDB6A050EDB5003E1B7D901E189D0B3
:10AC4A00700E006ED50E016E000E026E070EDBCF7F
:10AC5A0003F0046A056A066A03C03DF004C03EF0C8
:10AC6A0005C03FF006C040F0D3D92CEC6AF0005082
:10AC7A003424F36E01503520F46E02503620F86EFB
:10AC8A00F4CFF7FFF3CFF6FF0800090EF5CFDBFF8D
:10AC9A00580EDF5C0FE1610EF36E090E7BD90AE3F1
:10ACAA00200E006E090EDBCFE7FF0050E75E090EAB
:10ACBA00E7CFDBFF070EDBCF00F0016A026A036A07
:10ACCA000FDA00C03DF001C03EF002C03FF003C001
:10ACDA0040F0EECF38F0EECF39F0EECF3AF0EFCFCA
:10ACEA003BF02CEC6AF03BC0EDFF3AC0EDFF39C0F7
:10ACFA00EDFF38C0EFFF390EDBCFE9FFDB063A0E76
:10AD0A00DBCFEAFF01E2DB06090EDBCFEFFF150E10
:10AD1A00DB2A4BD995E1030EDBA61DD06F0EDF5C53
:10AD2A0006E1C1D918E3150EDB285BDA14D0780ED8
:10AD3A00DF5C09E0580EDF5C06E0620EDF5C03E0D0
:10AD4A00420EDF5C08E1020EF36E160EF3CFDBFF54
:10AD5A0002D0150EDB6A030EDB50100B0EE0040E58
:10AD6A00DBCF00F0050EDB50D880005406E2060E59
:10AD7A00DB5003E1040EDB5034DA95D90AE2050E02
:10AD8A00DBCFE7FF150EDB50E75E050EE7CFDBFFF3
:10AD9A0002D0050EDB6A040EDBCF00F0160E45D991
:10ADAA00D880005414E2160EDBCFE6FF150EDBCF77
:10ADBA00E6FF040EDBCFE6FF050EDB50E552E75C4B
:10ADCA00E552D880E754E552D880E7545FD9030E9C
:10ADDA00DB50010B0BE1080EDB5008E0B2D801E0B2
:10ADEA008DD0080EDB50BED8080EDB6A170EDB507A
:10ADFA0007E088D9170EF1D903E1011C01E17ED0E1
:10AE0A00160EDB5016E07ED9300EE66E9FD802E1B0
:10AE1A00011C74E077D9DFCFE6FF60EC69F0E552F8
:10AE2A00E552E552F4CF01F00001F31C02E1011CE6
:10AE3A0065E0050EDBCF00F0160EDB50D88000541B
:10AE4A0009E2050EDBCFE7FF160EDB50E75E050EC3
:10AE5A00E7CFDBFF300EE66E050ECBD94FE1390E98
:10AE6A00DB2ADBCFE9FF3A0E01E3DB2ADBCFEAFF7D
:10AE7A00090EEFCFDBFFDB500EE044D9090EADD946
:10AE8A0002E1011C3BE0390EDB2ADBCFE9FF3A0E77
:10AE9A00EDE3DB2AEBD755D831E1160EDBCFE6FF1F
:10AEAA00080EC3D8E552E7245DD82ED0070EDB5032
:10AEBA00030A1CE0010A14E0030A07E07BD9DBCF8E
:10AECA00EEFF020EDBCFEDFF1FD0F5D8056A03AE09
:10AEDA0002D0046805682CD8BCD805C0EEFF14D08F
:10AEEA00EAD803BE046824D8B4D80ED063D9DBCF1D
:10AEFA00EFFF0AD07BD905E1011C03E1F368F4688E
:10AF0A0010D0FCD801E3DB2A79D928EF53F0010EDF
:10AF1A00DBCF00F0020EDBCF01F000C0F3FF01C06F
:10AF2A00F4FF3B0EE15C02E2E16AE552E16ECBD04E
:10AF3A0029D9020E8EEF58F061D90800F550DF6E5C
:10AF4A001200200EE66E080EFEEF58F060EC69F073
:10AF5A00E552E552E552F3CF00F0F4CF01F00001DB
:10AF6A00F31C1200006E016AD950010F4DD900502E
:10AF7A00EE260150ED221200045E000E055AF70E6D
:10AF8A0004C0DBFFF80E05C0DBFF04C0E9FF05C003
:10AF9A00EAFF1200DBCFF4FFF350F45C1200DB503F
:10AFAA00E76E040EE7CFDBFF12000A0EDBCF00F0DC
:10AFBA000B0EDBCF01F00C0EDBCF02F00D0EDBCF58
:10AFCA0003F000500110021003101200130EEECF0E
:10AFDA00DBFF140EEDCFDBFF130EDBCF00F0140EF8
:10AFEA00DBCF01F00001800E01141200F70EDBCF57
:10AFFA0004F0F80EDBCF05F01200050EDB50E66E0A
:10B00A00D950130F01D9E552E750EE6EED6A1200DE
:10B01A000A0EDBCF38F00B0EDBCF39F00C0EDBCF8C
:10B02A003AF00D0EDBCF3BF01200DBCFE6FF150E38
:10B03A00DBCFE6FF050EDB50E552E724E552E724B5
:10B04A001200DB50CED8010EF36E060EF3CFDBFFF3
:10B05A001200EE50EFCFEAFFE96E02C0EEFF03C026
:10B06A00EEFF04C0EEFF1200D9CFE6FFDACFE6FF0B
:10B07A00E1CFD9FFE2CFDAFF1200DFCFE6FFE66ABF
:10B08A001AEC6AF0E552E552F3501200E76E080E28
:10B09A00E7CFDBFF1200EECF00F0EECF01F0EFCFEB
:10B0AA0002F0036A1200050EDBCF00F0150EDB502A
:10B0BA00D88000541200010EDBCF02F0020EDBCF63
:10B0CA0003F0046A1200E552E5CFDAFFE7CFD9FFB1
:10B0DA0012000A0E00C0DBFF0B0E01C0DBFF1200DC
:10B0EA00D9500A0F09EF59F0F36E070EF3CFDBFFC1
:10B0FA001200EECF00F0EFCF01F01200010EDB2AB2
:10B10A00020E1200FC0EDBCFE6FFFD0EDBCFE6FFE0
:10B11A001200005E000E015AF70E00C0DBFFF80EA7
:10B12A0001C0DBFF00C0E9FF01C0EAFF1200DA201C
:10B13A00EA6EEF2AEECFF6FF000EEF22EECFF7FF10
:10B14A00EF22EECFF8FF1200040EDBCFE6FF130E5C
:10B15A00DB50E552E75C9ADFDB5004DF060EDB507A
:10B16A001200090EDB500A0DF350DF24D00FE76EF0
:10B17A00090EE7CFDBFFA1EF57F0DB50F36E050EA8
:10B18A00CFEF57F0F70EDBCF00F0F80EDBCF01F070
:10B19A001200DFCFE6FFABEF57F028DF030EECDE3D
:10B1AA0050EF58F0FDEC52F0E552E552E552E55207
:10B1BA0000091200BDDEEE50EFCFEAFFE96E010E84
:10B1CA001200130EDB50F36E040ECFEF57F0040E8D
:10B1DA00DB50F36E090ECFEF57F0DBCFE6FFABEF94
:10B1EA0057F0E76E050EE7CFDBFF12008BDFCEEFDD
:10B1FA0058F0DBCFE6FF86DFD7EF58F0D950F90FCA
:10B20A00E96EFF0E9CEF58F0E96E000EDA20EA6E46
:10B21A001200439E08D0439E3BAE05D03A6C3B1EBB
:10B22A00E86A3B22438E3BC035F03AC034F0476AA5
:10B23A00466A8E0E366E376AE8EF5AF0439E0CD095
:10B24A00439E3BAE09D0386C391E3A1E3B1EE86A53
:10B25A0039223A223B22438E3BC035F03AC034F0C1
:10B26A0039C047F038C046F09E0E366E376AE8EFAE
:10B27A005AF0436A24EC5BF03CEC5BF043B6CCEF4B
:10B28A005AF043A205D043BACCEF5AF0D3EF5AF0A2
:10B29A0043BADFEF5AF043A005D043B8CCEF5AF0D7
:10B2AA00DFEF5AF043B8D3EF5AF0376A7F0E3C24E7
:10B2BA00366EE86A37224150365EE86A375A1A0E05
:10B2CA00446E3C6A466A476A346A356A3E50395E59
:10B2DA003F503A5A40503B5A000E3C5A09E73E50FA
:10B2EA0039263F503A2240503B22000E3C2201D0E0
:10B2FA00468AD89039363A363B363C36D890463666
:10B30A00473634363536442EE1D73B503A10391099
:10B31A00D8A4468AE8EF5AF0436A24EC5BF03CEC86
:10B32A005BF043B6CCEF5AF043A205D043B8CCEF5A
:10B33A005AF0D3EF5AF043AA05D043B0CCEF5AF0F3
:10B34A00D3EF5AF043B002D043A802D0DFEF5AF04D
:10B35A00376A41503C24366EE86A37227E0E365EE2
:10B36A00E86A375A466A476A346A356A40503B0285
:10B37A00F4CF35F0F3CF34F03F503B02F350472679
:10B38A00F4503422000E352240503A02F350472638
:10B39A00F4503422000E35223E503B02F35046262A
:10B3AA00F4504722000E342235223F503A02F3501D
:10B3BA004626F4504722000E3422352240503902E4
:10B3CA00F3504626F4504722000E342235223E50CE
:10B3DA003A02F4504626000E4722342235223F50C4
:10B3EA003902F4504626000E472234223522E8EF6D
:10B3FA005AF0417E436A24EC5BF03CEC5BF043B6C6
:10B40A00CCEF5AF043A20AD043AA03D043BECCEFF2
:10B41A005AF043A4D8EF5AF0D5EF5AF043AA05D010
:10B42A0043ACD8EF5AF0D5EF5AF043A00AD043A85C
:10B43A0008D043BE04D043A402D0E1EF5AF0E5EFAE
:10B44A005AF0466A376A41503C5C456E10E339C08F
:10B45A0047F03AC034F03BC035F03CC044F03EC03F
:10B46A0039F03FC03AF040C03BF0433A09D03EC001
:10B47A0047F03FC034F040C035F041C044F0456C5D
:10B48A00439E43BC438E44C036F043B014EF5BF096
:10B49A001A0E456014EF5BF0366A3C6A43A408D082
:10B4AA00396C3A1E3B1E3C1EE86A3A223B223C2279
:10B4BA0043AC08D0476C341E351E361EE86A342267
:10B4CA0035223622386A455207E03C343B323A325A
:10B4DA0039323832452EF9D7395047263A50342274
:10B4EA003B5035223C50362238C046F0439E36AE99
:10B4FA000BD0466C471E341E351E361EE86A47229C
:10B50A00342235223622438E36A006D0D8803532F0
:10B51A00343247324632442A44C036F0E8EF5AF011
:10B52A00436A24EC5BF043B69FEF5AF043A20FD074
:10B53A0043B407D07F0E3B6EFF0E3A6E396E386EFB
:10B54A0025D0800E3B6E01D03B6A000EF6D743B081
:10B55A00FBD7386A9F0E3C60EBD77E0E3C64F4D76B
:10B56A009E0E3C5C07E0D8903B323A323932383290
:10B57A003C2AF6D743A40AD0386C391E3A1E3B1E21
:10B58A00E86A39223A223B223BAEDED712007F0E0E
:10B59A003C6EFF0E3B6E3A6E396E12007F0E43BE52
:10B5AA00FF0E3C6E02D07F0E3C6E800E3B6E3A6AF6
:10B5BA00396AF3D743AE04D0800E3C6E3B6AF7D7A4
:10B5CA003C6A3B6AF4D73550341047104610F8E00D
:10B5DA0037BEF0D735BE0CD036503710EBE0D890D6
:10B5EA0046364736343635363606D8A03706F2D7C9
:10B5FA003750D4E13628D2E046AE11D07F0E461439
:10B60A0002E147A00CD0472AE86A3422352207E330
:10B61A00D880353234324732362A3628BFE036509F
:10B62A00C9E047C039F034C03AF035343B6E3630A1
:10B63A003C6E3B323C9E43BE3C8ED2EF5AF03B36C8
:10B64A003C3602E34384437E06E143803C6A3B6A1C
:10B65A003A6A396A12003C2803E0D8803B32120069
:10B66A00D8903B3202E143821200438612004036F0
:10B67A00413602E3438C437E06E14388416A406ACD
:10B68A003F6A3E6A1200412803E0D8804032120025
:10B69A00D8904032EAE1438A1200426A40AE5BEF38
:10B6AA005BF03F6C401EE86A4022421E3BAE63EFED
:10B6BA005BF03A6C3B1EE86A3B22421E6BEC6AF076
:10B6CA003BBE73EF5BF042AE000C3A6C3B1EE86A7D
:10B6DA003B22366C371EE86A3722000C42BE6AEFFC
:10B6EA005BF04388FF0C81EC5BF043B6000C43B07F
:10B6FA00000C43A4000C010C436A24EC5BF03CEC04
:10B70A005BF043B6120043AE08D043A004D043A86E
:10B71A0002D0438012004390120041503C5C0BE17E
:10B72A0040503B5C08E13F503A5C05E13E50395CD1
:10B73A0002E143801200D8A002D0438E10D03C50C0
:10B74A0041C03CF0416E3B5040C03BF0406E3A5025
:10B75A003FC03AF03F6E39503EC039F03E6E41501C
:10B76A003C5C10E0FF0F09E0439043B403D043AEC2
:10B77A004384120043AE43941200412AD8904032C7
:10B78A003F323E323E50395E3F503A5A40503B5A61
:10B79A003BBEEAD7D89039363A363B363C2EF8D7F4
:10B7AA00C8D73BC047F03AC046F03A503F02F4CF00
:10B7BA0039F0F3CF38F03B504002F4CF3BF0F3CFEF
:10B7CA003AF03F02F3503926F4503A22E86A3B2213
:10B7DA0046504002F3503926F4503A22E86A3B2296
:10B7EA0040AEFCEF5BF046503A5E47503B5A47AEDC
:10B7FA00000C3F503A5E40503B5A000C256C692CB5
:10B80A00256C690A0D00514D2C25692C25692C25BA
:10B81A00692C25690A0D00253034692C25303469D4
:10B82A000D0A002531690D0A00253033690D0A0019
:10B83A00253031306C750D0A0025640A0D00256427
:10B84A002C256C752C256C752C256C752C256C7526
:10B85A000A0D004D616A6F72206D616C66756E63C8
:10B86A0074696F6E2041786973322053746570432E
:10B87A006F756E746572207A65726F0A0D004D617C
:10B88A006A6F72206D616C66756E6374696F6E2083
:10B89A0041786973322053746570436F756E7465AD
:10B8AA007220746F6F2068696768203A20256C756A
:10B8BA000A0D004D616A6F72206D616C66756E6368
:10B8CA0074696F6E204178697331205374657043CF
:10B8DA006F756E746572207A65726F0A0D004D611C
:10B8EA006A6F72206D616C66756E6374696F6E2023
:10B8FA0041786973312053746570436F756E74654E
:10B90A007220746F6F2068696768203A20256C7509
:10B91A000A0D002130204572723A203C6178697321
:10B92A00323E20737465702072617465203C203148
:10B93A002E3331487A2E0A0D002130204572723A90
:10B94A00203C61786973323E20737465702072619D
:10B95A007465203E2032354B2073746570732F73E3
:10B96A0065636F6E642E0A0D002130204572723AAB
:10B97A00203C61786973313E20737465702072616E
:10B98A007465203C20312E3331487A2E0A0D00216D
:10B99A0030204572723A203C61786973313E2073D7
:10B9AA007465702072617465203E2032354B2073B5
:10B9BA00746570732F7365636F6E642E0A0D0021B0
:10B9CA0030204572723A203C6D6F76655F647572FD
:10B9DA006174696F6E3E206C61726765722074686B
:10B9EA00616E203136373737323135206D732E0A82
:10B9FA000D002130204572723A203C617869733219
:10BA0A003E20616363656C65726174696F6E20764E
:10BA1A00616C756520697320302E0A0D0021302073
:10BA2A004572723A203C61786973313E20616363E2
:10BA3A00656C65726174696F6E2076616C756520DC
:10BA4A00697320302E0A0D002130204572723A2087
:10BA5A003C61786973323E206C617267657220744A
:10BA6A0068616E2031363737373231352073746565
:10BA7A0070732E0A0D002130204572723A203C6103
:10BA8A00786973313E206C617267657220746861EF
:10BA9A006E2031363737373231352073746570731B
:10BAAA002E0A0D002130204572723A203C76656CD0
:10BABA006F636974795F66696E616C3E206C657349
:10BACA0073207468616E20342E0A0D0021302045DF
:10BADA0072723A203C76656C6F636974795F696E3D
:10BAEA00697469616C3E206C657373207468616E59
:10BAFA0020342E0A0D002130204572723A203C76FD
:10BB0A00656C6F636974795F66696E616C3E206CFF
:10BB1A006172676572207468616E20323530303028
:10BB2A002E0A0D002130204572723A203C76656C4F
:10BB3A006F636974795F696E697469616C3E206CC0
:10BB4A006172676572207468616E203235303030F8
:10BB5A002E0A0D005374617475733D25690D0A0030
:10BB6A002135204572723A204E65656420636F6DF7
:10BB7A006D61206E6578742C20666F756E643A204C
:10BB8A00272563270D0A0025730D0A00506172618B
:10BB9A006D383D25630D0A00506172616D373D2590
:10BBAA00630D0A00506172616D363D256C750D0A90
:10BBBA0000506172616D353D256C640D0A0050615B
:10BBCA0072616D343D25750D0A00506172616D33E5
:10BBDA003D25640D0A00506172616D323D25640D88
:10BBEA000A00506172616D313D25640D0A005049A9
:10BBFA002C2531750D0A004D522C253033750D0A4E
:10BC0A00002C253032753A25303475004100492C14
:10BC1A00253033692C253033692C253033692C259E
:10BC2A003033692C253033690D0A002138204572DA
:10BC3A00723A20556E6B6E6F776E20636F6D6D6111
:10BC4A006E642027256325633A2532582532582702
:10BC5A000D0A002138204572723A20556E6B6E6FBC
:10BC6A00776E20636F6D6D616E64202725633A25B8
:10BC7A003258270D0A002137204572723A2045783A
:10BC8A00747261207061726D617465720D0A0021AF
:10BC9A0036204572723A20496E76616C696420706A
:10BCAA006172616D7465722076616C75650D0A004A
:10BCBA002134204572723A204D697373696E672088
:10BCCA00706172616D657465722873290D0A0021AD
:10BCDA0033204572723A2052582042756666657260
:10BCEA00206F76657272756E0D0A002132204572D8
:10BCFA00723A20545820427566666572206F7665DE
:10BD0A007272756E0D0A002131204572723A204313
:10BD1A00616E27742073746570207468617420667C
:10BD2A006173740D0A002130200D0A0020080025D5
:10BD3A0073001B5B421B5B314B1B5B3047000D0AD8
:01BD4A0000F8
:10BD4C00D9CFE6FFDACFE6FFE1CFD9FFE2CFDAFFBA
:10BD5C00240EE12402E3E168E652E16ED950FA0FB9
:10BD6C00E96EFF0EDA20EA6E020EEECFDBFF030E59
:10BD7C00EECFDBFF040EEECFDBFF050EEECFDBFFCD
:10BD8C00E8D9F2D998EC66F0006E060EE15C02E29E
:10BD9C00E16AE552E16E0050E76E0D0EE7CFDBFF76
:10BDAC00DB50800815E0A0D93E6A3F6A406A416AC0
:10BDBC0000C039F001C03AF002C03BF003C03CF0C7
:10BDCC0078EC5BF0010A10E1210E0501EF6FF06BCE
:10BDDC00020EDB68030EDB68040EDB687F0EF36E6D
:10BDEC00050EF3CFDBFF66D10D0EDB50050B01E02A
:10BDFC0061D10A0EDBCF00F00B0EDBCF01F0830E0E
:10BE0C000026FF0E012200C0DEFF01C0DDFFD9506D
:10BE1C00060F65D976D9DF50010B0FE0DF06010E56
:10BE2C0001E2DB06D950180F5AD9D890EF36010E23
:10BE3C00EB36020EEB36030EEB36D9CFE9FFDACF39
:10BE4C00EAFF020E3F6E406AEECF3AF0EDCF3BF0C8
:10BE5C0052EC5BF03AC0EEFF3BC0EDFF140EDB6A18
:10BE6C00150EDB6A160EDB6A170EDB6A1C0EDB6A1C
:10BE7C001D0EDB6A1E0EDB6A010EF36E1F0EF3CF76
:10BE8C00DBFF010EF36E0E0EF3CFDBFF0F0EDB6A42
:10BE9C000E0EDBCF00F00F0EDBCF01F0D89001506F
:10BEAC0004E61A0E005C000E015801E398D0180E3F
:10BEBC00DBCF00F0190EDBCF01F01A0EDBCF02F056
:10BECC001B0EDBCF03F0010E1F0B07E0D8900036E2
:10BEDC00013602360336E806F9E1180E00C0DBFF26
:10BEEC00190E01C0DBFF1A0E02C0DBFF1B0E03C0D4
:10BEFC00DBFF140EDBCF08F0150EDBCF09F0160EAE
:10BF0C00DBCF0AF0170EDBCF0BF0010E1F0B07E097
:10BF1C00D890083609360A360B36E806F9E1D950BE
:10BF2C001C0FDDD80850EE24046E0950EE20056E6F
:10BF3C000A50EE20066E0B50EE20076ED950180FEB
:10BF4C00CED80450EE5C006E0550EE58016E0650D3
:10BF5C00EE58026E0750EE58036E200E00C0DBFF49
:10BF6C00210E01C0DBFF220E02C0DBFF230E03C03B
:10BF7C00DBFF200EDBCF39F0210EDBCF3AF0220EA7
:10BF8C00DBCF3BF0230EDBCF3CF03C34000E3C18F7
:10BF9C0009E6D880000E3954000E3A54000E3B547A
:10BFAC00000E3C5411E2D950200F99D8AAD8D8D8F9
:10BFBC001C0EDB50EE121D0EDB50EE121E0EDB5073
:10BFCC00EE121F0EDB50EE12D9501C0F88D8AFD8D2
:10BFDC000E0EDB2A0F0E01E25BD7DB2A59D7C9D82C
:10BFEC00100E00C0DBFF110E01C0DBFF180EDBCF03
:10BFFC003AF0190EDBCF3BF0120E3AC0DBFF130EFA
:10C00C003BC0DBFFADD893D8D950100F68D8EE5099
:10C01C00ED1012E0D950120F62D8EE50ED1006E17F
:10C02C00A8D8005001100210031006E099D8EE2A8F
:10C03C00000EEE22EE22EE220C0EDB6A91D8060EDA
:10C04C00EECFDBFF070EEECFDBFF080EEECFDBFFF4
:10C05C00090EEECFDBFF7E0EF36E0A0EF3CFDBFF85
:10C06C000B0EDB6AD950020FE66E000EDA20E66E7C
:10C07C0070D826EC67F0E552E552E552E552DECF7A
:10C08C00E6FFDDCFE6FF70D8FCEC65F0006E060E27
:10C09C00E15C02E2E16AE552E16E0050020E38C04A
:10C0AC00DBFF030E39C0DBFF040E3AC0DBFF050ECD
:10C0BC003BC0DBFF19D800C038F001C039F002C01A
:10C0CC003AF003C03BF0240EE15C02E2E16AE55277
:10C0DC00E16EE552E5CFDAFFE7CFD9FF1200E96E4A
:10C0EC00000EDA20EA6E1200020EDBCF00F0030E17
:10C0FC00DBCF01F0040EDBCF02F0050EDBCF03F03B
:10C10C001200180EEECFDBFF190EEECFDBFF1A0E6E
:10C11C00EECFDBFF1B0EEECFDBFF1200EECFE6FF08
:10C12C00EECFE6FFEECFE6FFEFCFE6FF1200D890A2
:10C13C00030EEB32020EEB32010EEB32EF32120039
:10C14C00EE500016EE500116EE500216EE5003168D
:10C15C001200D950060FE66E000EDA20E66E1200C1
:10C16C00D950140F75EF60F0D950020FB8DF94EF6F
:10C17C0060F0010E006E016A026A036AF1DFA6EF3D
:10C18C0060F0040130511F0B010801E01200305126
:10C19C00600BE842E842E842E842E842010801E06C
:10C1AC001200345103E0340501E012003151220A2F
:10C1BC0031E0030A24E0010A15E0210A0DE0010A2E
:10C1CC0001E012000401A00E8D6F070E8E6F080E99
:10C1DC00906F916B8F8121D00401A00E8D6F070E93
:10C1EC008E6F1BD036C495F437C496F40401800EC0
:10C1FC00926F070E936F976B986B948F12000401DC
:10C20C00800E8D6F070E8E6F070E906F916BC10EA7
:10C21C008F6F120032C49BF704018F8F120007013D
:10C22C00806B4B0E816F826B836B846B856B080EFE
:10C23C00866F8F6B1A0EE66E010EE66E53EC4DF0A8
:10C24C00E552E5521E0EE66E020EE66E53EC4DF014
:10C25C00E552E5522FD902E2E16AE5524FD90701C6
:10C26C00996B9A6B906B12001CD982D9050E3A18F7
:10C27C0001E13B5002E0000E18D051D90701975153
:10C28C00001808E19851011805E114D902E2E16A9D
:10C29C00E55234D944D907019951001805E19A5156
:10C2AC00011802E1906B956B010E0CD1FAD80701C5
:10C2BC008F6B9751981102E1000E05D045D9EF50C4
:10C2CC00800B01E0010E000931E1FB0EDBCF00F029
:10C2DC003BD9EE52EF50D880005405E235D9EE52DE
:10C2EC00FB0EEFCFDBFF8F6BFB0EDB508F5D19E28C
:10C2FC008F51EA6A400FE96E070EEA22EF50E66EA4
:10C30C008F51E76EFC0EDBCFE9FFFD0EDBCFEAFFB2
:10C31C00E750E926000EEA22E552E750EF6E8F2B2C
:10C32C00E3D7C8D802E2E16AE552E8D807018F5199
:10C33C00C9D0B7D80701905107E1E7D8FB0EDBCF86
:10C34C0095F7010E966F906FBDD00BD917E1C0D841
:10C35C00EDD802E101500BE0010EDBCFE9FFDB2A47
:10C36C00020EDBCFEAFF01E3DB2AEF50F1E1CDD87F
:10C37C00DFCF95F70701010E966F906FE552E552EE
:10C38C00E552A0D0EED818E1A3D8D0D802E10150E4
:10C39C000CE0010EDBCFF6FFDB2A020EDBCFF7FF42
:10C3AC0001E3DB2A0800F550F0E1AFD8DFCF95F7B9
:10C3BC000701966B010E906FE552E552E55282D063
:10C3CC0070D8E652E652070199519A1102E1000E1B
:10C3DC0008D099C7E9FF9AC7EAFFEF50800B01E03C
:10C3EC00010E00095BE1030E905D01E1906B905131
:10C3FC0055E0020E905D0DE1E66A000EE66EE66A0F
:10C40C008BD802E2E16AE55298D80701030E906FCF
:10C41C0045D0900543E1400E006E016A9551005CD9
:10C42C00000E015803E2400EDF6E02D095C7DFFF0D
:10C43C00DF50955D956F000E936F070E946F010E94
:10C44C00DFCFDBFF96510BE1010EDB5012E091C701
:10C45C00F6FF92C7F7FF0800F55043D8F5D7010E49
:10C46C00DB5007E091C7E9FF92C7EAFFEF5039D8DC
:10C47C00F6D70701955107E1400EDF5C02E1020E91
:10C48C0001D0030E906FDFCFE6FF000EE66E070EB5
:10C49C00E66E42D802E2E16AE5524FD8E552E55227
:10C4AC0011D0D9CFE6FFDACFE6FFE1CFD9FFE2CF4B
:10C4BC00DAFF1200400EE66E400EE66E070EE66ED8
:10C4CC00E66A47D0E552E5CFDAFFE7CFD9FF120095
:10C4DC00DF6A4ED8DE523AC0DEFF3BC0DDFFDD52D4
:10C4EC00120093C7E9FF94C7EAFFEF6E932B000E7F
:10C4FC009423912B9223010EDB061200E16E005067
:10C50C00F3CF97F7F4CF98F71200FC0EDBCF91F72F
:10C51C00FD0EDBCF92F71200010EE66E1AD0FA0E6A
:10C52C00DBCF00F0FB0EDBCF01F01200DF2ADF5077
:10C53C00006E016AFF0E00181200E16E0050F3CF7E
:10C54C0099F7F4CF9AF7120097C7E9FF98C7EAFF5B
:10C55C001200020EE66E72EC4DF0006E050EE15C00
:10C56C0012009FDFE652E652E6520701905112008C
:10C57C00FC0EDBCF3AF0FD0EDBCF3BF012006AD99C
:10C58C00E6520E01006BA96BDF6A180EDF5C14E239
:10C59C0083D9010EE9260E0E85D9DF5077D9EF6AC3
:10C5AC007BD9490EE9260E0E7DD976D9790EE9266E
:10C5BC000E0E78D9DF2AE9D70E01C60EAC6F0E0E1F
:10C5CC00AD6F3F0E79140009796ECF0E7914000906
:10C5DC00796E79827B6A7A6A79900F0152815293D3
:10C5EC00F00EB4140909B46E0E01080EAA6F030EF6
:10C5FC00AB6F800EAE6F3E0EAF6FE00EB06F2E0EB7
:10C60C00B16F040EB66F900EB26F010EB36F900E39
:10C61C00B46F010EB56F000EE66EE66A010EE66EA3
:10C62C00DFEC31F0E552E552E552E55229D112D951
:10C63C00E652DF6A180EDF5C0AE2DF5027D9EFCF33
:10C64C0000F0FD0EDB50005C0AE0DF2AF3D7DF6A56
:10C65C00180EDF5C08E2DF5019D9EF5002E1DF2839
:10C66C0003D0DF2AF5D7000EE5520AD1F3D8070E16
:10C67C00E12402E3E168E652E16EDE6ADD6A020E55
:10C68C00DB6A030EDB6A040EDB6A050EDB6A060E40
:10C69C00DB6A010EE66ED9CFE6FFDACFE6FF030EBA
:10C6AC00E2D8020F03D9010EDED8030FFFD8030E18
:10C6BC00DAD8050FFBD8030EFED80701B45124E1DC
:10C6CC00020EDB50180802E2B48D1ED0050EDBCF33
:10C6DC00E6FF060EDBCFE6FF030EDBCFE6FF040E14
:10C6EC00DBCFE6FF020EDBCFE6FFDECFE6FFDDCFD2
:10C6FC00E6FF11D8006E070EE15C02E2E16AE5523A
:10C70C00E16E005097EC40F0070EE15C02E2E16A4A
:10C71C00E552E16EB5D09ED8E652E652FB0EDBCF69
:10C72C00E6FF85DFE552E76E010EE7CFDBFFDB505E
:10C73C0002E1000E8CD0D950FC0FE96EFF0EDA200E
:10C74C00EA6EEE50ED101FE1010EDB049FD8EF50A6
:10C75C000E01EA6AAC25E96EAD51EA22EF6A88D87F
:10C76C00790EE9260E0E9ED883D8490EE9260E0EB8
:10C77C0099D8010EDB048AD8EF6A7AD8010EE92623
:10C78C000E0E90D862D0010EDB04006E0E01AA5181
:10C79C00005C5BE2FB0EDB50180857E3FB0EDB5032
:10C7AC00070802E10501E36B63D8010EE9260E0EC2
:10C7BC00EA22EE50ED1010E1E66AFB0EDBCFE6FF4D
:10C7CC009BEC49F0E552E552E66AFB0EDBCFE6FF47
:10C7DC006DEC49F0E552E55205012751FDE00501EC
:10C7EC00030E346FF70EDBCF4EF5F80EDBCF4FF5A3
:10C7FC00506B516B190E3D6E3E6A3F6A406A4EC5D6
:10C80C0038F04FC539F050C53AF051C53BF0A2ECA9
:10C81C0069F034C04EF535C04FF536C050F537C011
:10C82C0051F5010EDBCF55F5FB0EDBCF54F5FC0EAD
:10C83C00DBCF52F5FD0EDBCF53F5F90EDBCF56F502
:10C84C00FA0EDBCF57F50501276B010EDB50E552D5
:10C85C00E55216D0D9CFE6FFDACFE6FFE1CFD9FF0C
:10C86C00E2CFDAFF120027D8010EE66ED950120083
:10C87C00010EDB04E96EEA6AD890E936EA3612005A
:10C88C00E552E5CFDAFFE7CFD9FF1200EA6A310FA4
:10C89C00E96E0E0EEA221200EA6ADF34FE0BEA366B
:10C8AC00E96E1200EA22EE6AED6A1200E66E000EE4
:10C8BC00DA20E66E1200E66E3FEC47F0E552E552E8
:10C8CC00E552E5521200D9CFE6FFDACFE6FFE1CF11
:10C8DC00D9FFE2CFDAFF060EE12402E3E168E6526B
:10C8EC00E16EDF6A010EDB6AD950FA0FE96EFF0EBA
:10C8FC00DA20EA6E020EEECFDBFF030EEECFDBFF8B
:10C90C00040EEECFDBFF050EEECFDBFFD950FA0F96
:10C91C00E96EFF0EDA20EA6E060EE76ED890030E73
:10C92C00EB32020EEB32010EEB32EF32E706F6E1A0
:10C93C00D950FA0FE96EFF0EDA20EA6E060EE76E9A
:10C94C00D890EF36010EEB36020EEB36030EEB36BB
:10C95C00E706F6E1D950FA0FE96EFF0EDA20EA6E1F
:10C96C00400EEE26000EEE22000EEE22000EEE22FF
:10C97C00FA0EDBCF04F0FB0EDBCF05F0FC0EDBCFA9
:10C98C0006F0FD0EDBCF07F0D950020FE96E000E5A
:10C99C00DA20EA6EEE50045C006EEE500558016E23
:10C9AC00EE500658026EEE500758036E0050DF6EC4
:10C9BC00D950F80FE96EFF0EDA20EA6EEE50ED104A
:10C9CC0065E0040EDB50F86E030EDB50F76E020EC2
:10C9DC00DB50F66EDF50DF0600091AE0F60EDBCFF7
:10C9EC00E9FFDB2AF70EDBCFEAFF01E3DB2AEF508E
:10C9FC00F56E0D00F80EDB06DBCF00F0F90E01E250
:10CA0C00DB06DBCF01F00050011001E101D0E2D7D1
:10CA1C00040EDB50F86E030EDB50F76E020EDB508B
:10CA2C00F66EA684F2AE04D0F29EDE52010EDD6EDE
:10CA3C00550EA76EAA0EA76EA682A694010EDB5009
:10CA4C0003E0F28E010EDB6A400EDF6E400E006ECC
:10CA5C00016A026A036AD950020FE96E000EDA20ED
:10CA6C00EA6EEE500026EE500122EE500222EE50FD
:10CA7C000322020E00C0DBFF030E01C0DBFF040E1D
:10CA8C0002C0DBFF050E03C0DBFF92D7060EE15C94
:10CA9C0002E2E16AE552E16EE552E5CFDAFFE7CF5B
:10CAAC00D9FF120005D895EC4CF02DEC3CF0FBD7DF
:10CABC008ED8E652E6520F0148694969600ED36E72
:10CACC009B8C580EDE6E020EDD6EDFCF00F0DF06A3
:10CADC00010EDBCF01F001E2DB0600500110F5E1A5
:10CAEC00948E62EC3BF02BEC4CF0E552E55278D096
:10CAFC001200120012001200C7EF60F0120015EFC6
:10CB0C0061F004019B051EE104019C051BE1F1DFB2
:10CB1C00659204019C6B0201100EFE6F0E0EFF6FEE
:10CB2C00FE07000EFF5BFE51FF11FAE16584080E53
:10CB3C00FE6F070EFF6FFE07000EFF5BFE51FF112D
:10CB4C00FAE16594120043D8FC0EDBCF3AF0FD0EEF
:10CB5C00DBCF3BF0050E3A1801E13B5036E0E868BC
:10CB6C003A1802E17F0E3B182FE0030E3A1801E150
:10CB7C003B5028E0020E3A1801E13B5021E0010E37
:10CB8C003A1801E13B501AE0740E3A1801E13B509F
:10CB9C0013E0750E3A1801E13B500CE0730E3A1895
:10CBAC0001E13B5005E0720E3A180FE13B500DD0FD
:10CBBC00A1DF0BD09DDF09D09CDF07D0A0DF05D013
:10CBCC009DDF03D099DF01D096DF010E09D0D9CFBC
:10CBDC00E6FFDACFE6FFE1CFD9FFE2CFDAFF1200B2
:10CBEC00E552E5CFDAFFE7CFD9FF120096D8E1CFB7
:10CBFC00D9FFE2CFDAFF0C0EE12402E3E168E65242
:10CC0C00E16ED950FA0FE96EFF0EDA20EA6E080ECB
:10CC1C00EECFDBFF090EEECFDBFF0A0EEECFDBFF14
:10CC2C000B0EEECFDBFF79D8D950080FE96E000E52
:10CC3C00DA20EA6EEECFE6FFEECFE6FFEECFE6FFB0
:10CC4C00EFCFE6FF98EC66F0006E060EE15C02E2B8
:10CC5C00E16AE552E16E0050E76E070EE7CFDBFFAD
:10CC6C00DB50840B3AE1070EDB041AE1060EDB50B5
:10CC7C0006E0006A016A026A800E036E04D0006A44
:10CC8C00016A026A036A080E00C0DBFF090E01C0CC
:10CC9C00DBFF0A0E02C0DBFF0B0E03C0DBFF1DD057
:10CCAC00F80EDBCF00F0F90EDBCF01F0D950040FFA
:10CCBC00E96E000EDA20EA6E0050EE260150ED22ED
:10CCCC00D950080FE66E000EDA20E66E26D826EC58
:10CCDC0067F0E552E552E552E552080EDBCF00F065
:10CCEC00090EDBCF01F00A0EDBCF02F00B0EDBCF0F
:10CCFC0003F000C038F001C039F002C03AF003C0B4
:10CD0C003BF00C0EE15C02E2E16AE552E16EE552A9
:10CD1C00E5CFDAFFE7CFD9FF1200D9CFE6FFDACFA4
:10CD2C00E6FF1200D9CFE6FFDACFE6FFE1CFD9FF5D
:10CD3C00E2CFDAFFE652006801687F0E026E036AEA
:10CD4C00D950FA0FE96EFF0EDA20EA6EEE5000169B
:10CD5C00EE500116EE500216EE5003166AD800C0C3
:10CD6C00EEFF01C0EEFF02C0EEFF03C0EEFFFD0EB2
:10CD7C00DB50800B02E0010E01D0000EE66E59D89C
:10CD8C00060EE926000EEA22E552E750EF6EFC0E85
:10CD9C00DBCF00F0FD0EDBCF01F0D8900036013672
:10CDAC00FC0E00C0DBFFFD0E01C0DBFFDB50E66EAE
:10CDBC0040D8040EE926000EEA22E552E750EE6E4A
:10CDCC00ED6AFD0EDB50006E016AFF0E001818E1D3
:10CDDC00015016E12ED8EECF00F0EECF01F0EECFE1
:10CDEC0002F0EFCF03F0005001100210031006E028
:10CDFC00210E0501EF6FF06B800E0BD0040E09D0E5
:10CE0C00FD0EDB5008E115D8EE6AEE6AEE6AEE6AAA
:10CE1C00010EDF6E06D0020EDF6E0BD8EE52EE5214
:10CE2C00EE8EDF50E552E552E5CFDAFFE7CFD9FFC2
:10CE3C001200F80EDBCFE9FFF90EDBCFEAFF120090
:10CE4C00D9CFE6FFDACFE6FFE1CFD9FFE2CFDAFFA9
:10CE5C005BD8013411E20050FE08000E01540CE2C4
:10CE6C0076D805E06CD8800EEE6EEE6847D067D8A9
:10CE7C00800EEE6E7F0E0ED047D8D890015004E68F
:10CE8C00010E005C000E01580BE261D805E057D88A
:10CE9C00EE6A800EEE6E32D052D8EE6AEE6A2ED06A
:10CEAC0047D8EECF00F0EECF01F0EECF02F0EFCF8F
:10CEBC0003F032D800C0EEFF01C0EEFF02C0EEFF5F
:10CECC0003C0EEFF21D80050010B05E025D8020E5F
:10CEDC003AD8EF8E04D020D8020E35D8EF9E14D855
:10CEEC00D8900132003218D8030E2DD800C0EFFFB5
:10CEFC001AD804E011D8030E26D8EF8EE552E5CFF0
:10CF0C00DAFFE7CFD9FF120013D8040E1CD8EECFEE
:10CF1C0000F0EFCF01F01200FA0EDBCFE9FFFB0EB1
:10CF2C00DBCFEAFF120004D8060E0DD8EF5012002A
:10CF3C00FC0EDBCFE9FFFD0EDBCFEAFF1200ECDFCE
:10CF4C00EE6AEE6A1200E926000EEA221200220EA8
:10CF5C000501EF6FF06B99EF67F0D9CFE6FFDACFF1
:10CF6C00E6FFE1CFD9FFE2CFDAFFE652E652E65216
:10CF7C00E652E652DF6AD950FA0FE96EFF0EDA205C
:10CF8C00EA6E010EEECFDBFF020EEECFDBFF030EDF
:10CF9C00EECFDBFF040EEECFDBFFF60EDBCF00F0A7
:10CFAC00F70EDBCF01F0F80EDBCF02F0F90EDBCF82
:10CFBC0003F048D80050EE5C0150EE580250EE5889
:10CFCC000350EE5833E2030EDB50F86E020EDB50CA
:10CFDC00F76E010EDB50F66EA684A688F2AE03D077
:10CFEC00F29E010EDF6E550EA76EAA0EA76EA682DC
:10CFFC00DF5001E0F28E006A040E016E026A036AD1
:10D00C0021D8EE500026EE500122EE500222EE50B6
:10D01C000322010E00C0DBFF020E01C0DBFF030E7A
:10D02C0002C0DBFF040E03C0DBFFB7D7050EE15CCB
:10D03C0002E2E16AE552E16EE552E5CFDAFFE7CFB5
:10D04C00D9FF1200D950010FE96E000EDA20EA6EFA
:10D05C0012002A0EF66E100EF76E000EF86E050119
:10D06C000900F550EA6F0900F550EB6F03E1EA6730
:10D07C0001D03DD00900F550E56F0900F550E66F81
:10D08C000900F550E76F09000900F550E96E090039
:10D09C00F550EA6E090009000900F550E86F090027
:10D0AC00F550E96F09000900F6CFECF5F7CFEDF577
:10D0BC00F8CFEEF5E5C5F6FFE6C5F7FFE7C5F8FFD7
:10D0CC000501E85302E1E95307E00900F550EE6E63
:10D0DC00E807F8E2E907F9D7ECC5F6FFEDC5F7FF6D
:10D0EC00EEC5F8FF0501EA07000EEB5BBFD7120097
:10D0FC00FE0EE3CFE9FFFF0EE3CFEAFFE9CFF3FF2C
:10D10C00EACFF4FFFB0EE35003E1FC0EE35009E021
:10D11C00FB0EE30602E2FC0EE306FD0EE350EE6EA0
:10D12C00F1D71200FE0EE3CFE9FFFF0EE3CFEAFFCB
:10D13C00F36AF46AEE5203E0F34AF42AFBD71200C6
:10D14C00FF0EE3CFF8FFE552FF0EE3CFF7FFE552FA
:10D15C00FF0EE3CFF6FFE552E66AE66AE66A0900DF
:10D16C00F55209E0FD0EE32A05E1FE0EE32A02E189
:10D17C00FF0EE32AF4D7FD0EE3CF39F0FE0EE3CF1A
:10D18C003AF0FF0EE3CF3BF01200D9CFE6FFDACF37
:10D19C00E6FFE1CFD9FFE2CFDAFFE652E652E652E4
:10D1AC00E652D950FB0F006EFF0EDA20016E00C064
:10D1BC00DEFFDD6EDECFE6FFDDCFE6FFFB0EDBCF65
:10D1CC00E6FFFC0EDBCFE6FFFD0EDBCFE6FFF1C585
:10D1DC00E6FFF2C5E6FF13EC53F0006E070EE15CC0
:10D1EC0002E2E16AE552E16E0050020EF3CFDBFF82
:10D1FC00030EF4CFDBFF020EDBCF00F0030EDBCF10
:10D20C0001F000C0F3FF01C0F4FF040EE15C02E288
:10D21C00E16AE552E16EE552E5CFDAFFE7CFD9FFDF
:10D22C001200D9CFE6FFDACFE6FFE1CFD9FFE2CF8C
:10D23C00DAFFE652E652E652E652D9CFE9FFDACFF0
:10D24C00EAFFFA0EDBCFEEFFFB0EDBCFEEFFFC0EA0
:10D25C00DBCFEEFFFD0EDBCFEEFF020EDB50F86EE8
:10D26C00010EDB50F76EDF50F66EF80EDBCF00F0E0
:10D27C00DB06F90EDBCF01F001E2DB0600500110FA
:10D28C000DE00900F60EDBCFE9FFDB2AF70EDBCF52
:10D29C00EAFF01E3DB2AF5CFEFFFE7D7040EE15CF1
:10D2AC0002E2E16AE552E16EE552E5CFDAFFE7CF43
:10D2BC00D9FF1200D9CFE6FFDACFE6FFE1CFD9FFD5
:10D2CC00E2CFDAFFFB0EDBCF00F0FC0EDBCF01F080
:10D2DC000001800E01141AE1FB0EDBCFE9FFFC0EFE
:10D2EC00DBCFEAFFEECFF3FFEDCFF4FFEE2A000E1B
:10D2FC00EF22F3CFE9FFF4CFEAFFFD0EDBCFEFFF18
:10D30C00EF50016AF36E01C0F4FF10D0FB0EDB503E
:10D31C00FE0806E1FD0EDBCFE6FF9FEC6AF005D0C0
:10D32C00FD0EDBCFE6FFA1EC3DF0E552E552E5CF7B
:10D33C00DAFFE7CFD9FF120038503D02F3CF34F0BB
:10D34C00F4CF35F03E02F3503526000EF420366E45
:10D35C0038503F02F3503626000EF420376E38500A
:10D36C004002F350372639503D02F3503526F45025
:10D37C003622000E372239503E02F3503626F45036
:10D38C00372239503F02F35037263A503D02F350C2
:10D39C003626F45037223A503E02F35037263B5093
:10D3AC003D02F35037261200120100020200004029
:10D3BC00D80492FD8201010203010902430002011B
:10D3CC0000C0320904000001020201000524001013
:10D3DC0001042402020524060001052401000107B2
:10D3EC0005810308000209040100020A000000077D
:0FD3FC0005020240000007058202400000C6D370
:10D40C00FF0EE124E96EFF0EE220EA6EEDCFF4FF91
:10D41C00EFCFF3FFF46607D0600EF36404D07B0EFD
:10D42C00F36001D0F39A1200F36AF46AFF0EE12460
:10D43C00E96EFF0EE220EA6EED6607D02F0EEF6468
:10D44C0004D03A0EEF6001D0F32A1200376A366A24
:10D45C00356A346A200EE76ED890383639363A364B
:10D46C003B3634363536363637363D50345C3E50E6
:10D47C0035583F5036584050375809E33D50345ECC
:10D48C003E50355A3F50365A4050375A382AE72EBC
:10D49C00E4D712004F4B0D0A000D0A0045424276AC
:10D4AC0031335F616E645F61626F76652045422047
:10D4BC004669726D776172652056657273696F6E1D
:09D4CC0020322E352E350D0A0028
:10D4D600376A366A100EE76ED8903A363B363636DD
:10D4E60037363F50365C4050375805E33F50365E7E
:10D4F6004050375A3A2AE72EF0D71200C00EF36E84
:10D5060000EE00F00E0E01D81200EA6002D0EE6ABC
:10D51600FCD7F350E9601200EE6AFCD71DEE00F06E
:10D526002DEE00F0F86A439C2FEC68F0C1EC6AF02F
:10D5360058EC65F0FBD71200FF0EE350ADBA04D0ED
:10D54600B06AAC8EAD8A949CADA2FED7AE6EF36E79
:10D55600F46A1200F36AF46AF32A0F0B05E0D89016
:10D56600F336F436E804FBE1120030313233343559
:0BD57600363738396162636465660077
:10D5820012000403090418035300630068006D00CD
:10D5920061006C007A004800610075007300380376
:10D5A2004500690042006F00740042006F00610094
:10D5B200720064002C0020002000200020002000C7
:10D5C2002000200020002000200020002000200059
:10D5D2002000200020002203200020002000200044
:10D5E2002000200020002000200020002000200039
:10D5F2002000200020002000800284029C02D4022D
:10D60200FEFF00000000000000000100000000001A
:10D612000000000000000000000000000000000008
:10D6220000000000000000000000000000000000F8
:10D6320000000000000000000000000000000000E8
:10D6420000000000000000000000000000000000D8
:10D6520000000000000000000000000000000000C8
:10D662000000000000000000000000000000009226
:10D672000F920F920F930F930F930F930F930F939A
:10D682000F930F930F940F940F940F940F940F9482
:10D692000F940F940F950F950F950F950F950F956A
:10D6A2000F890F890F890F8A0F8A0F8A0F8A0F8AB3
:10D6B2000F8A0F8A0F8A0F8B0F8B0F8B0F8B0F8B9B
:10D6C2000F8B0F8B0F8B0F8C0F8C0F8C0F8C0F8C83
:10D6D2000F8C0F000105000102030405060700017B
:0CD6E20002030405060702030405060706
:08FFF800ACF70AFF63F801F009
:00000001FF
